:1000000000400020D16F000011700000137000004C
:1000100000000000000000000000000000000000E0
:10002000000000000000000000000000157000004B
:1000300000000000000000001770000019700000B0
:100040001B700000595100004D7400001B7000002F
:100050001B700000000000001B7000001B700000FF
:100060001B7000001D770000C93000001B700000ED
:100070001B7000001B7000001B7000001B70000054
:100080001B700000B57800001B7000001B700000A2
:100090001B7000001B7000001B7000001B70000034
:1000A0001B7000001B70000000000000000000003A
:1000B0000000000000000000000000000000000040
:1000C00010B5064C2378002B07D1054B002B02D02E
:1000D000044800E000BF0123237010BD640200202B
:1000E00000000000E0E20000044B10B5002B03D03C
:1000F0000349044800E000BF10BDC04600000000F6
:1001000068020020E0E20000164B002B00D1144BE7
:100110009D46402292029A1A924600218B460F4633
:100120001348144A121A0BF06DF90F4B002B00D034
:1001300098470E4B002B00D0984700200021040068
:100140000D000D48002802D00C4800E000BF0BF065
:1001500019F92000290007F097F90BF0EDF8C046D7
:100160000000080000400020000000000000000027
:1001700064020020B82F00200000000000000000F2
:1001800002000120104011D1042A0ED91368180969
:1001900080B2002809D001388000031D11180979A8
:1001A000002902D001309842F8D170470020FCE7C6
:1001B0000378002B03D05AB2002A01DB01307047CC
:1001C0003F229343C03B59424B41C01803789343AD
:1001D000802BF4D10130F9E710B500240378002B0F
:1001E00001D1200010BDFFF7E3FF0134F6E770B541
:1001F000002204000D00411C092003F081FA0028B0
:1002000006D001236200134343600023A34200DBB6
:1002100070BD9A00A958821891600133F6E770B555
:10022000012803DC1C2001F047F870BD01230D6894
:1002300011201D42F7D04868184206D1042804D97D
:100240000F2302681340042B01D00E20EBE703F0CC
:10025000B5F86D100400002D03DDFFF7BDFFA842C7
:1002600006DA1220DFE72000FFF7A2FF0400013DBD
:10027000012DF8D120787F2809DDDF280BDCF82359
:100280003F22DB00800118406378134018430123AC
:1002900040001843C9E7EF280BDCFC226378120109
:1002A0009B0113403F220007000C0343A07810403D
:1002B000ECE7F72812DCFC22637892021B03134060
:1002C000E0228004520310403F221843E378134099
:1002D000FC220343A07812018001E8E7012040429C
:1002E000D5E7F8B54D680F00EB0706D4042D04D907
:1002F0000F232E683340092B03D00B2000F0DCFFC6
:10030000F8BD6B683609B6B25C10731EA3420FD8F5
:100310000321200008F032FF6421642803DC01007F
:10032000032800DA03212800891903F01BFA0500CD
:100330002B6800201B099BB2013B9C42E0D23A682B
:10034000A31C9B005A510123013464001C436C60C0
:10035000D6E7F0B585B0012803DC1C2000F0ACFF27
:100360002CE001274B683A000093022806D08B68E6
:100370003B4203D05F10002F00DC17000124009BDC
:10038000234200D0B2E0042B00D8AFE01B680D6818
:100390000F2619003140042925D1254205D1042D0D
:1003A00003D92B681E40042E01D00E20D6E70098FA
:1003B000FFF7E6FEB84203DA0120404205B0F0BD87
:1003C000009802F0FBFF0600280002F0F7FF010092
:1003D000781E30180BF0CCFB0028EDD0801B0130CC
:1003E00040002043EAE709293DD1009B5B685B1090
:1003F00001939F42E0DC25422CD1042D2AD92B68A1
:100400003340042B26D1280002F0D8FF0396029037
:100410007E1C009AB300D058854201D17800E0E7F5
:1004200020420ED104280CD90368039A1340042BF0
:1004300007D102F0C3FF010002980BF063FB002814
:10044000ECD0019B37009E42E2DDB5E71F00019B27
:100450009F42B1DC7B1C00999A008A58AA42F5D1D0
:1004600078000124BDE7032940D11A0992B25B0F3D
:1004700092000B40D31A01939F429DDC254229D163
:10048000042D27D92A681640032E19D1100980B2ED
:10049000520F800032402C1D801A019B26181B1A17
:1004A0000193009B781E0433019A904200DD83E79C
:1004B00022001918B2420FD316D101304000D0E704
:1004C000042E07D1280002F079FF04002800FFF76E
:1004D00057FEE2E70F2041E70D78AC461578AC45B2
:1004E00002D101310132E5E70130DDE7212035E7B6
:1004F00010B502F047FF43000120184310BD000073
:10050000C30711D404280FD90F2302681340032B0B
:100510000AD119400133591AC0234907DB05194094
:10052000024B1A40114301607047C046FFFFFF9F16
:10053000F7B507000E001C20012F06DD4C680123D3
:1005400022001A40009203D10D2000F0B5FE53E0C6
:10055000022F02D08A681A42F6D0012335681D4264
:1005600000D0A9E0042D00D8A6E01C41002C00DC3E
:100570001C000F2029680840092828D16B685B10EF
:100580000093022F05D0B368009A5B109A4200DDF9
:100590000093009B01221D1B0135EB43DB171D401F
:1005A000691C092003F0ACF8071E09D001236D0077
:1005B0001D4303003268083345600099A14201DA07
:1005C0003800FEBD0134A100515802C3F5E70428EC
:1005D00045D1280002F0F2FEFFF7FEFD0190022F48
:1005E00004D0B3685B10984200DD0193019BA342E5
:1005F00004DA002003F0F6F80700E1E7280002F033
:10060000DDFE0700009BA34221DB2800009702F0DB
:10061000D5FE05003800FFF7CBFD019B0134070034
:10062000A342F7DA009BC41A200003F0DBF8071E90
:10063000C6D002F0C3FE0190306802F0BFFE220077
:10064000009B591B411801980AF0C0FEB8E738001A
:10065000FFF7AEFD009B070001330093D2E70328AC
:100660002AD10B099BB2490F9B000140591A022F56
:1006700004D0B2685210914200DD1100A14205DAA7
:1006800000220320110003F03BF8B5E703200E1B06
:10069000331DD9170140C9188910002203F030F822
:1006A000071E00D18CE7013631000334FFF728FF25
:1006B000381D29193200C7E7212046E7F8B5002880
:1006C00005DC1C2000F0F8FD05002800F8BD01261F
:1006D0000C6826400FD06410E343DB171C40E11C7C
:1006E00089100022032003F00BF8051EEDD0210035
:1006F000FFF706FFE9E7042C01D80025E5E70F2303
:1007000022681340042B1BD12000FFF739FDC31CC6
:1007100007000320D9170140C9188910320002F0E0
:10072000EFFF051ED1D03900FFF7EAFE200002F0EE
:1007300045FE2B1D01003A0018000AF047FEC4E7F1
:10074000092BDAD10320636832005F10FB1CD91734
:100750000140C918891002F0D3FF051ECDD0390021
:10076000FFF7CEFEFF20BE42AFDA0122B300E3184E
:100770009B68134208D01341FF2B00DD0300D943CF
:10078000C917AA190B4013710136ECE710B57F2980
:1007900002DC0170013010BD1A4B99420CDC402381
:1007A0008A115B42134303703F230B40802149426F
:1007B000194341700230EEE7134B994210DC2023BD
:1007C0000A135B4213433F24802203708B11524271
:1007D0002340214013430A43437082700330DAE719
:1007E0000A4B9942D7DCF0230370603B4370113B06
:1007F0008A11FF3B1A4382703F2211401943C17096
:100800000430C8E7FF070000FFFF0000FF0F0100F2
:10081000F0B50D0085B0002803DC1C2000F04CFD75
:100820000DE009680122080010400AD002AC114115
:100830002000FFF7ABFF011B200002F0DFFF0400E8
:100840001AE004293FD90F230C682340092B3AD121
:100850004B685B10019303239C46019B9A420EDD7B
:1008600002F0C0FF041E07D02E68012502F0A6FD8D
:100870002F00019B9D421DDD200005B0F0BD01321F
:100880009300CC580123234001D10D20C6E764100A
:100890007F2C0DDD0D4E0223B44209DD0C4E634664
:1008A000B44205DD00270B4EE30FA6427B419B00BF
:1008B000C018D2E70135AB00F1583942E5D04910F4
:1008C000FFF764FFD5E72120A8E7C046FF07000037
:1008D000FFFF0000FF0F010010B5040001200840D9
:1008E00010D104290DD90F230A681340042B08D115
:1008F000080002F063FD010020000BF003F9434201
:10090000584110BD0020FCE7F7B50F00012803DCBB
:100910001C2000F0D1FCFEBD01264D682E4006D102
:10092000042D04D90F222B681A40092A01D00B206C
:10093000EFE76A681B099BB25410A34200D85C1E03
:1009400039681E48FFF7C8FF01230190002813D122
:1009500039681B48FFF7C0FF002811D0002C0DD0CC
:100960000123621C013C9C409200535123436B6065
:1009700004E00136B200AB50B442FADA0020CAE714
:100980003B680D20DA07C4D55B10002B11DD9C42BB
:100990000FDB9B00A200291DEB1889180433994234
:1009A00009D10123013C9C40AA181C4353606C6090
:1009B000E4E71220ADE758681860EFE797CA000037
:1009C0009BCA0000002310B50C000B70C30705D5AF
:1009D0000D49421020000BF059F808E00B4900289F
:1009E00002D0042804D10A4920000BF06FF810BD92
:1009F0000428FCD90F2302681340042BF7D102F01E
:100A0000DDFC04490200E5E794D40000A0CA000020
:100A1000A6CA0000ABCA0000F0B593B00600029170
:100A20001C20012E1DDD029B01251B681C002C4093
:100A300000D0ADE0042B00D8E6E01A680F231A407E
:100A4000092A4AD10394039A029992008A581700FE
:100A50002F4005D1042A03D910681840092806D070
:100A6000222000F029FC0190019813B0F0BD5268DB
:100A70005210A418039A013203929642E3D1611CEA
:100A8000012202F03DFE0190002802D100230193D3
:100A9000EAE7019B6400190025435D600831029A72
:100AA000BB00D05802684368120992B25B109A42A8
:100AB00000D8531E0022934209DCDA43D2171340B8
:100AC0009B00C918039B01379F42E8DBCCE79400E9
:100AD0000519AD6801320D51EDE72700032A59D100
:100AE0000193029ABB00D3582B42B9D1042BB7D93A
:100AF000186801990140032939D1020992B2430FC4
:100B000092000B40D31A1C190137BE42E9D10320D1
:100B1000E31CD9170140C9188910002202F0F0FD2A
:100B200001900028B2D000252100FFF7E9FC019BCD
:100B30001E1D029AAB00D45801231C421FD1042C65
:100B40001DD90F2123681940032918D1180980B233
:100B50005B0F80000B40C01A0023834213DBC343AA
:100B6000DB17184001353618BD42E2DB7CE704296B
:100B700000D075E71800FFF703FB2418C4E7200036
:100B8000FFF7FEFAE8E7E2181279F2540133E4E7DE
:100B900000273C000F25029ABB00D35801221342C4
:100BA00034D1042B32D9186801002940042935D1E9
:100BB0001800FFF7E5FA24180137BE42EBD12000F8
:100BC00002F010FE0190002800D15FE7029FB600FE
:100BD000BB19041D029301233D681D4229D1042D38
:100BE00027D90F262B681E40042E37D12800FFF787
:100BF000C7FA0600280002F0E1FB010020003200E5
:100C00000AF0E4FBA41922E02700C3E7180005A9B5
:100C1000FFF7D8FE05A80AF07FFFCCE7032900D034
:100C20001EE7020992B2430F92000B40D31A1C191F
:100C3000C2E705A92800FFF7C5FE05A80AF06CFF6A
:100C400005A90500020020000AF0C0FB6419029B00
:100C50000437BB42BFD10023237005E7032EF6D132
:100C60001A0992B25B0F92001E40961B291DC5E720
:100C7000F0B50D0095B0002806DC1C2000F01CFB30
:100C80000400200015B0F0BD0C68012123000B40CA
:100C9000009306D1042C04D922680F331A40092A84
:100CA00001D00B20EAE7626852100392002A03DCAD
:100CB000009802F097FDE3E73F4A019201280BD02C
:100CC0006868084208D1042806D902681340042B3A
:100CD00002D102F073FB019001980AF01DFF06009B
:100CE0000F27039B0834013B04935E43039B029050
:100CF0009B001B19059301232068184251D1042839
:100D00004FD903683B40042B52D1FFF739FA059BBA
:100D100004343618A342EED1300002F063FD041E05
:100D2000AFD02B680593029B002B03D0686802F0BC
:100D300045FB0190200002F041FB0500009B059A55
:100D40009B00D3189F68380002F038FB012306008F
:100D50001F4201D1042F04D807A93800FFF732FE43
:100D600007AE30000AF0D8FE07000200310028006C
:100D70000AF02CFB029BED19002B0AD0049B009A71
:100D8000934206DD2800029A01990AF01FFB029B9C
:100D9000ED18009B01330093009A039B9342CDD141
:100DA0006FE707A9FFF70EFE07A80AF0B5FEAEE74A
:100DB00002F004FBF9E7C04638CF000010B500246C
:100DC000A04207DD0B6801341C4003D05C10E343F4
:100DD000DB171C40611C0122092002F091FC002855
:100DE00003D0012364001C43446010BD0A6870B541
:100DF00010000125284034D1042A32D90F24136869
:100E000049681C40092C17D154681B099BB22C411E
:100E1000A34200D85C1E844205DC022001339842C4
:100E200006DB00200FE085005519A9600130F2E7CC
:100E3000840011510130F2E7032C12D1294203D171
:100E4000132000F039FA70BD4910FF29F8D81B09AA
:100E50009BB204329B00D3189342E2D91170013245
:100E6000FAE70B2000F028FADBE700000123F7B5D2
:100E700000254E680F0033400093AB420ED11D0099
:100E8000042E0BD90F2233681A40092A10D1726838
:100E90001B099BB25510AB4200D85D1E3968CB07C9
:100EA00017D54C10002C01DDA5421DDA122032E0CE
:100EB000042A04D13000FFF763F90500EEE7009D36
:100EC000032AEBD11D09ADB25B0FAD001340ED1A43
:100ED000E4E72E48FFF700FD002814D00AF072FD69
:100EE000290008F031FA4C1C009B002B4CD1042E39
:100EF0004AD932680F331340092B10D10134A400B2
:100F0000A4592000FEBD39682148FFF7E5FC2C00FC
:100F10000028E9D1113000F0CFF90400F1E7042BEB
:100F20002AD1300002F04AFA0500FFF755F9A04235
:100F3000BCDB012C1ADC300002F040FA00902800E3
:100F4000FFF736F9461B300002F04CFC041ED8D0E7
:100F500002F034FA0190786802F030FA009B320017
:100F6000E91A411801980AF031FACAE72800FFF798
:100F70001FF9013C0500DCE7032B05D13419E478A7
:100F8000023B64001C43BCE70B20C4E790CA00008E
:100F90009BCA0000F7B54D680F002A0001210A40E6
:100FA0002FD1042D2DD90F242B68BE681C40092C8D
:100FB00014D169681B099BB24C100192A34200D85E
:100FC0005C1E39682A48FFF787FC00282DD00F23C4
:100FD0002A681340092B1DD1012317E0032C10D1DF
:100FE0000E4203D1132000F067F9FEBD721001928A
:100FF000FF2AF7D81A0992B25B0F92001C40141B0B
:10100000DFE70B20EFE701339A00AE509C42FADA9B
:101010000020EAE7032BFBD12B0001335A1BA2422D
:10102000F6DC6A461279DA70F7E73968CB0706D53D
:101030004910002901DD8C4209DA1220D3E70D485E
:10104000FFF74AFC2100002801D11130CBE70F2324
:101050002A681340092B03D1013189004E51D7E78B
:10106000032BD5D16B461B796D18EB70D0E7C046CA
:1010700097CA00009BCA000010B5012408682042EE
:101080001AD1042818D90F2102681140092901D169
:10109000406810BD032908D113099BB2500F9B0073
:1010A0000840181A40002043F3E7042904D102F055
:1010B00085F9FFF791F8F5E70B2000F0FDF8E8E778
:1010C00010B5034A0B21034804F03EF910BDC04699
:1010D00038CA000030CA0000002070470420704762
:1010E0000120704710B5002002F07CFB10BD0020ED
:1010F0007047002070470020704700207047002094
:1011000070470020704700207047002070470000A3
:1011100010B5034A0C21034804F016F910BDC0466F
:1011200020CB000080CB000010B50124044002D089
:101130004410200010BD042810D90F23026813406A
:10114000042B07D102F03AF921000A220AF0ACFD83
:101150000400EEE7032B01D10430F5E70D22014B2B
:101160001A70E6E7A4020020012210B5024018D14F
:10117000042802D903681A0992B201230B4012D144
:10118000042902D90B681B099BB20024934206D1A3
:1011900004309B000431C318984206D30124200078
:1011A00010BD0022E9E70023EFE704780A78002C5D
:1011B00001D1002AF2D0013001319442ECD0002458
:1011C000EDE70000F7B50700009101933049314B7E
:1011D000002A02D002220A70013A00261A601B6817
:1011E000CE54BE4200DBF7BD009AB300D058294B65
:1011F000274D1C68C8239B0065191C1B012318423E
:1012000006D0254A4310210028000AF00DFC09E011
:10121000224A002802D004281BD1214A210028009C
:101220000AF002FC1A4C20000AF076FC194A019BD5
:101230001060002B0BD07B1EB34208DD194B984287
:1012400005D8431C1360202222540022E2540136A8
:10125000C7E7042819D90F2301680B40042B04D1D8
:1012600002F0ACF8104A0300CDE7092B03D1436824
:101270000E4A5B10C7E7032B08D10A0992B2490F47
:1012800092000B40D31A0A4ABDE70123094ABAE784
:10129000A5020020C805002094D40000A0CA0000C8
:1012A000A6CA00001F030000BFDA0000F0CD000056
:1012B000FFCD00000ACE0000014B187000207047DF
:1012C000A402002070B501F0EDFD094C0100251DC0
:1012D0001F2228000AF038FC28000AF01DFC042315
:1012E00004308008000118432060200070BDC04613
:1012F00080020020C368F0B59D00836889B05D1945
:101300000300183306930369069A9F00069B029018
:10131000DF19436901939B00D3180393CD4B1B78CE
:10132000002B26D17F222B68CB491C1213409B0037
:101330005B58043501929F46029B587804F020FCCC
:101340000023029A137027E0C24B1B78002B10D1A8
:101350002B68019A1C121340BF4A9B009B5804350E
:10136000E9E7069B3A1DD11ABA4BD82928DD1A2283
:101370001A70029BB74C9B6821780193EA1A029B72
:1013800092109B7812021A43029B587804F000FCDA
:101390000023029A23701370029B069A9B680193A4
:1013A000ED1A029BAD10DD60069BFE1A029BB61083
:1013B0001E61039B9B1A029A9B10536109B0F0BDFA
:1013C0001B783C60002B01D01700D2E72B680199F5
:1013D0001C120B40A0499B005B5817000435AAE77C
:1013E000069B3A1DD11A9B4BD82902DD1A221A708E
:1013F000BFE728681B78291D3860002B02D0170032
:101400000D00B6E76B6801991C120B4092499B00D6
:101410005B58170008358EE7069B3A1DD11A8D4B95
:10142000D82902DD1A221A70A3E7A4001B782C1910
:101430003C60002B01D017009BE72B6801991C1220
:101440000B4085499B005B581700043573E7069BEA
:101450003A1DD11A7F4BD82902DD1A221A7088E76B
:101460007E49A40061581B783960002B01D0170019
:101470007FE72B6801991C120B4077499B005B5852
:101480001700043557E7043F744B3A68A400E25054
:10149000704B1B78002B00D06BE72B68019A1C1255
:1014A00013406D4A9B009B58043544E76B4BA400E6
:1014B000E058FFF739FE043F06003868FFF734FEB6
:1014C00036180120654B76000643E650614B1B78C9
:1014D000002B00D04DE72B68019A1C1213405E4A86
:1014E0009B009B58043526E7069B3A1DD11A594BA1
:1014F000D82902DD1A221A703BE70698039C0121C5
:10150000A04202D221000C3909681B783960002BF7
:1015100001D017002DE72B6801991C120B404E4992
:101520009B005B581700043505E7069B3A1DD11A4E
:10153000484BD82902DD1A221A701AE70699039837
:1015400081420FD203000C3B1B6845495B106418B5
:10155000E41AA40023583B603E4B1B78002B05D0B7
:10156000170006E7182119700023F4E72B6801998A
:101570001C120B4038499B005B5817000435DAE613
:10158000069B039A934219D213000C3B1B68344A02
:10159000043FA4185B10E31A039A39689B00995022
:1015A0002C4B1B78002B00D0E3E62B68019A1C1211
:1015B0001340294A9B009B580435BCE61822254B52
:1015C0001A70EDE7069B039A93422DD2244B3E1FDF
:1015D000E31814000C3C04932368049A5B10D31A9C
:1015E000039A9B009858FFF79FFD07903068FFF71C
:1015F0009BFD2468049B64101C1B079BA4001F1800
:1016000001207F00039B0743E7503700114B1B78F5
:10161000002B00D0ADE62B68019A1C1213400E4A35
:101620009B009B58043586E618220A4B1A70EDE79A
:10163000069B3A1DD11A074BD82902DD1A221A70CF
:1016400097E60399A40061581B783960002B09D0F4
:1016500017008EE6A4020020F0CB0000842D0020AD
:10166000FDFFFF3F2B6801991C120B40D9499B00DD
:101670005B58170004355EE6043F039B3A68A400FC
:10168000E250D54B1B78002B00D072E62B68019AF4
:101690001C121340CF4A9B009B5804354BE6039B1A
:1016A000A4001C192368043F38685E10FFF73CFD56
:1016B00036180120C84B76001B7806432660002BA5
:1016C00000D056E62B68019A1C121340C14A9B00B9
:1016D0009B5804352FE6069BA4003F1BBE4CBB4223
:1016E0000CD82378002B00D043E62B68019A1C12FB
:1016F0001340B84A9B009B5804351CE6B74801F0DC
:101700004DFE2378002B00D033E62B68019A1C1283
:101710001340B04A9B009B5804350CE6A300ED181B
:10172000002C00DA38E6AC4B1B78002B00D020E60A
:101730002B68019A1C121340A64A9B009B58043543
:10174000F9E5043F3B68042B04D1A300ED18002CFD
:1017500000DA21E6A04B1B78002B00D009E62B68AD
:10176000019A1C1213409B4A9B009B580435E2E5EA
:10177000043F3B68042B04D0A300ED18002C00DAD2
:101780000AE6954B1B78002B00D0F2E52B68019AF6
:101790001C1213408F4A9B009B580435CBE53A1F1F
:1017A00013685B10013B06D401215B00A4000B43CE
:1017B0002D191360F0E5884B17001B78002B00D023
:1017C000D7E52B68019A1C121340824A9B009B5854
:1017D0000435B0E53A00069B0C32D31AD82B03DD52
:1017E0001A227D4B1A70C4E5FF2361005B0019408B
:1017F000FE3BFF3B19433960029906988968241221
:1018000004916D1A0299AD1089782D020D43039948
:101810009D40091A891099401D430B43BB60029BF0
:101820007D609C70E4B26E4BE4000392E358029A30
:101830009360694A1278002A03D008331D00039F81
:1018400097E51D00019A9B680C351C121340614AF4
:101850009B009B58039F6EE53B1F1C68039A069BE9
:1018600093422DD10A20E3070CD4042C13D90F2363
:1018700022681340042B11D1200001F09FFD0AF0D3
:101880004BF90630643003F099FD00280FD1043D78
:10189000069B039380E50720042CF3D02000431E11
:1018A0009841FA234042FF3318400730EAE7029B91
:1018B0002100587804F07EF90023029A1370E7E7BC
:1018C000039B039A0C3B1B6802995B109B00D31A85
:1018D0000C3B1C601F1D1300083B1B685A108A70CC
:1018E000D2B23F49D2005B0055589B0A029A9B0036
:1018F0009560ED18039B069A043B1B685B109B00E8
:10190000D3180393344B1B78002B00D031E52B68A0
:10191000019A1C1213402F4A9B009B5804350AE57C
:101920003B1F1868FFF700FCA40006003F1B1E28A1
:1019300027DC00280DDC284B1B78002B00D018E595
:101940002B68019A1C121340224A9B009B580435B5
:10195000F1E401F095FA033E361801F091FA214BBB
:10196000801B9842F9D81C4B1B78002B00D000E557
:101970002B68019A1C121340164A9B009B58043591
:10198000D9E40123029A137001F07AFA029B0A3813
:1019900086195E6000E53B1F1868FFF7C5FBA400D1
:1019A00006003F1B00280DDC0B4B1B78002B00D0E2
:1019B000DFE42B68019A1C121340064A9B009B58D7
:1019C0000435B8E4084B984210DD1D22024B1A7012
:1019D000CFE4C046F0CB0000A40200201CCE0000E3
:1019E0008C2500203F420F0080EE36000123029A32
:1019F000137001F045FAFA239B005E43029B0A3EF6
:101A000030185860C8E4A300FF1A002320001A0011
:101A10003900FFF7D7FBCC4ECC4C3168200001F0E9
:101A2000EDFECB4B31681860200003F077FF316882
:101A3000200004F0C6F8C74B1B78002B00D098E4B8
:101A40002B68019A1C121340C34A9B009B58043513
:101A500071E4C04BA4001B783F1B002B00D088E42E
:101A60002B68019A1C121340BB4A9B009B580435FB
:101A700061E4029803F006FDB64B1B78002B00D002
:101A800077E42B68019A1C121340B34A9B009B58C1
:101A9000043550E43B1F1B68002B3ED13B000C3B40
:101AA0001B68DA072CD5390001225B105800083971
:101AB00002430A60002B44DD012259001143381F04
:101AC00001603900083909681141CB1A39000C3915
:101AD0000968114224D09B189340A4001343039A31
:101AE000A3509C4B1B78002B00D042E42B68019A3A
:101AF0001C121340984A9B009B580435FFF71BFCAF
:101B0000042B06D90F211A680A40092A01D15B6803
:101B1000C9E719228F4B1A702BE45B10013BC9E710
:101B2000042909D90F200A680240092A04D1023386
:101B30009B005B58A400D2E71922864B1A70FFF76E
:101B400018FC0435CDE7A300069AFB189B1AD82B86
:101B500013DC0122631E002C14DC7E4B1B78002B4F
:101B600001D0FFF706FC2B68019A1C1213407A4A39
:101B70009B009B580435FFF7DEFB1A22754B1A7049
:101B8000FFF7F7FB3A601C000437E3E7069A3B1DBA
:101B90009B1A704ED82B03DD1A233370FFF7E9FB35
:101BA000069B039AA40093422AD23B1F1868FFF7B2
:101BB000BBFA011E21DD039B0C3B1A6852108242C6
:101BC0001BDB9007801A654B4018C018039B8000F0
:101BD000C2583B1B1A605F4B3F1B1B780437002B1E
:101BE00001D0FFF7C6FB2B68019A1C1213405A4A1A
:101BF0009B009B580435FFF79EFB20233370EAE7D8
:101C00001823FBE7524BA4001A683B1B1F001A6005
:101C1000504B04371B78002B01D0FFF7AAFB2B6831
:101C2000019A1C1213404C4A9B009B580435FFF745
:101C300082FBA3009C46FE1A002C17DC1C22454B9D
:101C40001A70002333606346FF1A424B04371B7837
:101C5000002B01D0FFF78DFB2B68019A1C1213405B
:101C60003D4A9B009B580435FFF765FB0020336815
:101C70005A108300F15801230B4003D10D21354A3E
:101C80001170DFE749108A4200DD0A00013084420A
:101C9000EFDC012352001343D4E7A3009C46FE1A55
:101CA000002C17DC1C222B4B1A7000233360634678
:101CB000FF1A284B04371B78002B01D0FFF759FB84
:101CC0002B68019A1C121340234A9B009B58043531
:101CD000FFF731FB002033685A108300F1580123CD
:101CE0000B4003D10D211B4A1170DFE749108A42D6
:101CF00000DA0A0001308442EFDC01235200134372
:101D0000D4E73B00083B1868FFF70EFA3B1F0600BC
:101D10001868FFF709FA0023864200DA0433A400AA
:101D20003A1B170013600B4B04371B78002B01D0B4
:101D3000FFF71FFB2B68019A1C121340064A9B00F9
:101D40009B580435FFF7F7FAC8050020A5020020CC
:101D500008000020A4020020F0CB0000FCFFFF3FA1
:101D60003B00083B1868FFF7DFF93B1F06001868C7
:101D7000FFF7DAF9F30FC217B0425341A4003A1B40
:101D800017009B001360E34B04371B78002B01D036
:101D9000FFF7EFFA2B68019A1C121340DE4A9B00F2
:101DA0009B580435FFF7C7FA3B00083B18683B1FF8
:101DB0001968A600BE1B0423814202D0042802D861
:101DC0000023336018E001239C461842F8D10F230A
:101DD00002681A40042AF3D163461942F0D104295B
:101DE000EED90B680B321340042BE9D1FFF7BCF995
:101DF000431E984180003060C64BA4001B783F1BF7
:101E00000437002B01D0FFF7B4FA2B68019A1C129B
:101E10001340C14A9B009B580435FFF78CFA3B00E6
:101E2000083B18683B1F1968A600BE1B00238142AF
:101E300002D0042802D80423336018E001239C4612
:101E40001842F8D10F2302681A40042AF3D16346DE
:101E50001942F0D10429EED90B680B321340042B40
:101E6000E9D1FFF781F94342584180003060A94B26
:101E7000A4001B783F1B0437002B01D0FFF779FA31
:101E80002B68019A1C121340A34A9B009B580435EF
:101E9000FFF751FA3B00083B1868FFF745F93B1F75
:101EA00006001868FFF740F9F317C20F8642534146
:101EB000A4003A1B17009B001360964B04371B7855
:101EC000002B01D0FFF755FA2B68019A1C12134022
:101ED000914A9B009B580435FFF72DFA3B00083BC5
:101EE0001868FFF721F93B1F06001868FFF71CF977
:101EF0000023864200DD0433A4003A1B1700136060
:101F0000844B04371B78002B01D0FFF732FA2B6883
:101F1000019A1C121340804A9B009B580435FFF71E
:101F20000AFA3B1F1B68A400043B5A1E93413A1B4C
:101F300017009B001360774B04371B78002B01D0F0
:101F4000FFF717FA2B68019A1C121340724A9B0084
:101F50009B580435FFF7EFF93B00083B1868FFF783
:101F6000E3F83B1F06001868FFF7DEF8321801207F
:101F7000A4003B1B1F00520002431A60654B04374C
:101F80001B78002B01D0FFF7F4F92B68019A1C1283
:101F90001340614A9B009B580435FFF7CCF93B0086
:101FA000083B1868FFF7C0F83B1F06001868FFF7EA
:101FB000BBF8321A0120A4003B1B1F005200024351
:101FC0001A60544B04371B78002B01D0FFF7D1F96E
:101FD0002B68019A1C1213404F4A9B009B580435F2
:101FE000FFF7A9F93B00083B1868FFF79DF83B1F76
:101FF00006001868FFF798F802000120A4003B1BB8
:102000001F007243520002431A60424B04371B7890
:10201000002B01D0FFF7ADF92B68019A1C12134079
:102020003D4A9B009B580435FFF785F93B1F186814
:10203000FFF77AF8061E17D11F23364A1370A40043
:102040003B1B1F001E60334B04371B78002B01D055
:10205000FFF78FF92B68019A1C1213402E4A9B0040
:102060009B580435FFF767F93B00083B1868FFF7FA
:102070005BF8310007F082F8012640000643DEE7F6
:102080003B1F1868FFF750F8061E17D11F23214A7F
:102090001370A4003B1B1F001E601E4B04371B78EF
:1020A000002B01D0FFF765F92B68019A1C12134031
:1020B000194A9B009B580435FFF73DF93B00083B4C
:1020C0001868FFF731F8310007F03EF901264900A2
:1020D0000E43DEE73B1F1868FFF726F8C21780188B
:1020E00050400122A4003B1B1F0040001043186019
:1020F000084B04371B78002B01D0FFF73AF92B6807
:10210000019A1C121340044A9B009B580435FFF7A8
:1021100012F9C046A4020020F0CB0000A300FE1A72
:102120003068012C24D1FEF7FFFF0494079009F0DA
:1021300049FC0799002900DC012107F005F9049BFF
:10214000A400C918012349001943EA4B3F1B1B781F
:1021500031600437002B01D0FFF70BF92B68019A8F
:102160001C121340E44A9B009B580435FFF7E3F828
:10217000FEF7DAFF04907068FEF7D6FF049B01308B
:10218000C31A0793D3E7A300FE1A3100200004937B
:1021900001F0BAFC049B3060FF1AD64B04371B7861
:1021A000002B01D0FFF7E5F82B68019A1C121340B1
:1021B000D14A9B009B580435FFF7BDF83B00083B14
:1021C0001868FEF7B1FF3B1F06001868FEF7ACFF6A
:1021D00002000120A4003B1B1F00324052000243BA
:1021E0001A60C44B04371B78002B01D0FFF7C1F8ED
:1021F0002B68019A1C121340BF4A9B009B58043560
:10220000FFF799F83B00083B1868FEF78DFF0600C2
:102210003B1F1868FEF788FF320002430120A4002C
:102220003B1B1F00520002431A60B24B04371B785D
:10223000002B01D0FFF79DF82B68019A1C12134068
:10224000AD4A9B009B580435FFF775F83B00083BEF
:102250001868FEF769FF06003B1F1868FEF764FF69
:10226000320042400120A4003B1B1F0052000243E9
:102270001A60A04B04371B78002B01D0FFF779F8C8
:102280002B68019A1C1213409B4A9B009B580435F3
:10229000FFF751F83B1F1868FEF746FFC0430122C5
:1022A000A4003B1B1F00400010431860914B0437F3
:1022B0001B78002B01D0FFF75CF82B68019A1C12E9
:1022C00013408D4A9B009B580435FFF734F83B00C0
:1022D000083B1868FEF728FF06003B1F1868FEF74A
:1022E00023FF3200824051000122A4003B1B1F004B
:1022F0000A431A607F4B04371B78002B01D0FFF78D
:1023000038F82B68019A1C1213407B4A9B009B589B
:102310000435FFF710F83B00083B1868FEF704FF90
:1023200006003B1F1868FEF7FFFE32000241510015
:102330000122A4003B1B1F000A431A606D4B0437A7
:102340001B78002B01D0FFF714F82B68019A1C12A0
:102350001340694A9B009B580435FEF7ECFF3B0095
:102360000C3B1868FEF7E0FE3B00083B06001868CF
:10237000FEF7DAFEF1170200C317300007F036F857
:102380003B1F049005911868FEF7CEFE02000498EA
:10239000059906F0DFFF43000120A4003E1B370033
:1023A0001843544B30601B780437002B01D0FEF7E4
:1023B000E0FF2B68019A1C1213404F4A9B009B5868
:1023C0000435FEF7B8FFA300FE1A31002000049385
:1023D000FEF7F4FC049B3060FF1A464B04371B7871
:1023E000002B01D0FEF7C5FF2B68019A1C12134089
:1023F000414A9B009B580435FEF79DFFA300FF1A3E
:1024000039002000FEF7F2FC3A4B1B78002B01D07C
:10241000FEF7AFFF2B68019A1C121340364A9B004F
:102420009B580435FEF787FFA300FE1A31002000F9
:102430000493FEF71BFD049B3060FF1A2D4B0437FD
:102440001B78002B01D0FEF794FF2B68019A1C1219
:102450001340294A9B009B580435FEF76CFFA300EC
:10246000FF1A39002000FEF795FD224B1B78002B48
:1024700001D0FEF77EFF2B68019A1C1213401E4A02
:102480009B009B580435FEF756FFA300FE1A31004F
:1024900020000493FEF7F0FD049B3060FF1A154BFB
:1024A00004371B78002B01D0FEF763FF2B68019ADD
:1024B0001C121340104A9B009B580435FEF73BFF4B
:1024C0003B1F186800F07AFF3A00083A12680300D0
:1024D000A400D1072DD4042A10D910680F2210406F
:1024E0000138082813D806F0ABFD09242A26121259
:1024F00012122800A4020020F0CB0000F1491800BD
:1025000009F000FB434258413B1B80001860EE4B32
:102510003F1B1B780437002B01D0FEF72AFF2B68E6
:10252000019A1C121340E94A9B009B580435FEF7A0
:1025300002FFE749E3E7E749E1E7E749DFE7E74982
:10254000DDE7069B3E1DF31ADF4CD82B03DD1A2373
:102550002370FEF70EFF00F09DFC4300012018439E
:1025600023783860002B02D03700FEF702FF2B687B
:10257000019A1C121340D54A9B009B583700043522
:10258000FEF7D9FE069B3E1DF31ACF4CD82B03DD78
:102590001A232370FEF7EDFE00F072FCD04B4000D2
:1025A00018400123184323783860002B02D03700ED
:1025B000FEF7DFFE2B68019A1C121340C34A9B00F2
:1025C0009B5837000435FEF7B6FE0123A600BE1B5C
:1025D00020001A003100FEF7F5FDC24C206864307F
:1025E00002F0ECFE002802D1043DFEF7D5FE029B6E
:1025F00021685A78BC4803F0F2FA0123029A3700A6
:10260000137000F03DFCB94B22681B68063253433F
:102610001818029B5860FEF7BFFEA600BE1B2000E4
:10262000012300223100FEF7CDFDAE4C206864305E
:1026300002F0C4FE0028D7D0AB4803F05FF8DCE717
:10264000A4003E1BFEF73EFE37009F4B30601B7818
:102650000437002B01D0FEF78CFE2B68019A1C1268
:1026600013409A4A9B009B580435FEF764FEA40071
:102670003E1B300000F03DFC3700934B30601B7870
:102680000437002B01D0FEF774FE2B68019A1C1250
:1026900013408E4A9B009B580435FEF74CFEA40065
:1026A0003E1B300000F027FC3700874B30601B7862
:1026B0000437002B01D0FEF75CFE2B68019A1C1238
:1026C0001340824A9B009B580435FEF734FEA3005A
:1026D000FE1A31002000049300F010FC049B3060CF
:1026E000FF1A794B04371B78002B01D0FEF741FE0F
:1026F0002B68019A1C121340744A9B009B580435A6
:10270000FEF719FEA4003F1B380000F029FC6E4BB9
:102710001B78002B01D0FEF72CFE2B68019A1C12AF
:1027200013406A4A9B009B580435FEF704FEA30041
:10273000FE1A31002000049300F03AFC049B306044
:10274000FF1A614B04371B78002B01D0FEF711FEF6
:102750002B68019A1C1213405C4A9B009B5804355D
:10276000FEF7E9FDA4003F1B380000F063FC564B68
:102770001B78002B01D0FEF7FCFD2B68019A1C1280
:102780001340524A9B009B580435FEF7D4FD0121AB
:10279000200000F037FC4C4B1B78002B01D0FEF7DB
:1027A000E8FD2B68019A1C121340484A9B009B5875
:1027B0000435FEF7C0FD0021200000F023FC424B51
:1027C0001B78002B01D0FEF7D4FD2B68019A1C1258
:1027D00013403E4A9B009B580435FEF7ACFDA40015
:1027E0003E1B300000F048FC3700374B30601B7850
:1027F0000437002B01D0FEF7BCFD2B68019A1C1298
:102800001340324A9B009B580435FEF794FDA40008
:102810003E1B300000F044FC37002B4B30601B782F
:102820000437002B01D0FEF7A4FD2B68019A1C127F
:102830001340264A9B009B580435FEF77CFDA400FC
:102840003F1B380000F006FC1F4B1B78002B01D00B
:10285000FEF78FFD2B68019A1C1213401B4A9B0048
:102860009B580435FEF767FDA4003F1B380003F0BA
:10287000D1FC154B1B78002B01D0FEF77AFD2B689D
:10288000019A1C121340114A9B009B580435FEF715
:1028900052FDA4003E1B300003F056FD37000A4BEA
:1028A00030601B780437002B01D0FEF762FD2B68E7
:1028B000019A1C121340054A9B009B580435FEF7F1
:1028C0003AFDC0462CCE0000A4020020F0CB000050
:1028D00034CE00003BCE000042CE000047CE0000C8
:1028E000FEFFFF7FC8050020A50200200400002095
:1028F000A4003F1B380003F03DFCC24B1B78002BAB
:1029000001D0FEF736FD2B68019A1C121340BE4A17
:102910009B009B580435FEF70EFDA4003E1B3000C3
:1029200003F03EFC3700B74B30601B780437002BB8
:1029300001D0FEF71EFD2B68019A1C121340B24A0B
:102940009B009B580435FEF7F6FCA300FF1A3900E4
:10295000200001F0F7FBAB4B1B78002B01D0FEF7FA
:1029600008FD2B68019A1C121340A74A9B009B5834
:102970000435FEF7E0FCA300FF1A3900200001F047
:1029800017FAA04B1B78002B01D0FEF7F2FC2B6846
:10299000019A1C1213409C4A9B009B580435FEF779
:1029A000CAFCA300FF1A3900200001F003FB954B7D
:1029B0001B78002B01D0FEF7DCFC2B68019A1C125F
:1029C0001340914A9B009B580435FEF7B4FCA300CA
:1029D000FF1A3900200001F015FB8A4B1B78002BF1
:1029E00001D0FEF7C6FC2B68019A1C121340864AE0
:1029F0009B009B580435FEF79EFCA300FE1A310095
:102A00002000049303F038FD049B3060FF1A7D4BD7
:102A100004371B78002B01D0FEF7ABFC2B68019A22
:102A20001C121340784A9B009B580435FEF783FC28
:102A3000A300FE1A31002000049303F025FD049B3F
:102A40003060FF1A6F4B04371B78002B01D0FEF764
:102A500090FC2B68019A1C1213406B4A9B009B58F8
:102A60000435FEF768FCA300FE1A31002000049331
:102A700003F012FD049B3060FF1A624B04371B7891
:102A8000002B01D0FEF775FC2B68019A1C12134035
:102A90005D4A9B009B580435FEF74DFCA300FE1ACF
:102AA00031002000049303F01DFB049B3060FF1AEB
:102AB000544B04371B78002B01D0FEF75AFC2B68CF
:102AC000019A1C121340504A9B009B580435FEF794
:102AD00032FCA300FF1A3900200001F0A1F9494B94
:102AE0001B78002B01D0FEF744FC2B68019A1C12C6
:102AF0001340454A9B009B580435FEF71CFCA3007D
:102B0000FF1A3900200001F0A5FA3E4B1B78002B7C
:102B100001D0FEF72EFC2B68019A1C1213403A4A92
:102B20009B009B580435FEF706FCA300FE1A3100FB
:102B30002000049301F00AFA049B3060FF1A314B25
:102B400004371B78002B01D0FEF713FC2B68019A89
:102B50001C1213402C4A9B009B580435FEF7EBFBDC
:102B6000A300FF1A3900200001F0B8F9254B1B78AB
:102B7000002B01D0FEF7FDFB2B68019A1C121340BD
:102B8000214A9B009B580435FEF7D5FB069B029A11
:102B9000FB1A9B101361A300FF1A3900200002F0FA
:102BA000EBFD184B1B78002B01D0FEF7E2FB2B68E6
:102BB000019A1C121340144A9B009B580435FEF7DF
:102BC000BAFB069B029AFB1A9B101361A300FE1A24
:102BD00031002000049302F0CFFD049B3060FF1A07
:102BE000084B04371B78002B01D0FEF7C2FB2B6883
:102BF000019A1C121340044A9B009B580435FEF7AF
:102C00009AFBC046A4020020F0CB00000023F7B5D9
:102C10005A1E0192002B07DA01F0AAFA02F0DCFE3C
:102C200003F03CF81923019300263000194B196872
:102C3000B14212DD184B1A6801328A420FDAF024D1
:102C40001A601D68154F6C43E35D002B1FD0E4191B
:102C5000022B06D12000FEF74DFB019BD8E7002296
:102C6000EDE7012B0DD1002801D100F009F9F02288
:102C70006A43BB185B680A49C31A8B4201D8022316
:102C8000BB54F0235D43054BEB5C022BE2D00136D5
:102C9000CCE7C046CC050020000000202C1C002002
:102CA0003F420F00012200210A4B0B481A611950C4
:102CB00004301950A2210420C9005850C121C0205D
:102CC0008900800258501A60044BFC311960044B93
:102CD0001A70704700A000400405000000E100E009
:102CE000F305002004207047F8B550C901232200E5
:102CF0001A40101E2DD03340181E2AD06410002018
:102D00001C2C26D81D4B761035009E4200DD1D0080
:102D10001B4F3B5D012B05D00121200004F04AFD33
:102D200001233B55174B1B78002B01D1FFF7BAFF4E
:102D30000023154A9E420DDCFF2514491448D65C39
:102D4000B44202D15E007052D5540133042BF6D147
:102D50000420F8BDD15C8C4203D10C4A5B009D522B
:102D6000F6E70133042BF5D10023D15CFF2901D113
:102D7000D454F2E70133042BF7D1E9E788130000BC
:102D8000D4050020F30500201C0000200E000020C8
:102D9000DC050000F8B530C9012623003340181EB9
:102DA0001BD02B003340181E17D0344100201C2CA0
:102DB00013D8174F3B5DB34204D03100200004F01C
:102DC000F9FC3E5569100800124A1038124B904227
:102DD00004D9012252421A600420F8BD1C600F4839
:102DE00006F0CCF90E4B18800E4B1B78002B02D14D
:102DF000FFF758FFF0E701220B4B9A64A922D2009B
:102E00009A588018A82280B2D2009850E4E7C046B1
:102E1000D4050020908601001800002020A10700A2
:102E20000C000020F305002000A00040030010B5B6
:102E30000120002B02DC1B30FEF73EFA10BD0420FF
:102E4000704710B5002803DC1C20FEF735FA10BDD2
:102E50000B680020DB07FAD40D30F6E701220020D2
:102E6000054B06491A615850043103305850083157
:102E7000801858501A607047008000400405000018
:102E80000122034B1A64A822D20098587047C0460A
:102E90000080004010B5FFF7F3FFFA21890006F02B
:102EA000E3F810BD00487047A4CE00001D20704715
:102EB00070B5054E0400335C0D008B4202D004F067
:102EC00079FC355570BDC046D405002070B500248E
:102ED000064D635D012B05D10021200004F06AFC42
:102EE0000023635501341D2CF2D170BDD4050020A0
:102EF00070470D2070473B2070470000F8B5012453
:102F00000B6806000D00234204D10D20FEF7D4F912
:102F10002000F8BD5B102000052BFAD80E4A9B005C
:102F20009C580E4F3B5D002B05D00021200004F083
:102F300041FC00233B55012E06DD6B68042B03D1B9
:102F40000221200004F036FC200004F0E1FA012404
:102F500040002043DDE7C0468CCE0000D4050020B1
:102F6000F8B501260568354202D04468344203D1E1
:102F70000D20FEF7A1F9F8BD6D101C2DFBD80A4FEE
:102F80007B5D012B04D03100280004F013FC7E553A
:102F9000064964108C4202DCE143C9172140280035
:102FA00004F03CFBE7E7C046D4050020FF03000027
:102FB00070B501240D68254204D10D20FEF77CF97F
:102FC000200070BD6D101C2D17D80024012804DDD1
:102FD0004C68043C63425C416400094E735DA3424B
:102FE00004D02100280004F0E5FB7455280004F00B
:102FF00015FC03000420012BE3D00020E1E7C046CC
:10300000D405002070B504000D001C280ED8084E11
:10301000335C012B04D0012104F0CCFB0123335598
:10302000290020004D1EA94104F0E2FB70BDC046FE
:10303000D4050020036810B5DA0703D40D20FEF78D
:103040003BF910BD4168581004394A425141FFF71D
:10305000D9FFF6E737B569460A00064B30CB30C2D8
:1030600003680220042B02D100F0A4FF37BD00F05A
:10307000C9FFFBE754CE000010B5084C6379002B64
:1030800005D00021052004F095FB00236371052085
:1030900004F0C4FB43425841800010BDD405002019
:1030A00010B5084CE37A002B05D000210B2004F06A
:1030B00081FB0023E3720B2004F0B0FB4342584134
:1030C000800010BDD4050020F7B5304D304E6B6C3C
:1030D000002B15D0A8240023E40037596B642D4B36
:1030E000186800280CDB2C4B19784A425141C9B2B0
:1030F000197004F07DFB294B1B88DF19BFB23751D3
:10310000AB6C002B39D00021254B264FF458A96415
:103110003A780C340193244D8A4206D02B68032B55
:1031200003D8224AD05C04F063FB2B68204A0133A9
:10313000134004D50422013B5242134301331B497F
:1031400000228C462B60042B18D06046C05C591CB2
:10315000FF2802D10B000122F5E7002A00D02B60E6
:10316000012104F045FB01233B702B68114A5B00F1
:103170009B5AE418019BA4B2F450F7BD01235B42B3
:103180002B6000233B700C4BF3E7C046FCA00040D3
:1031900000A0004018000020F20500200C000020D4
:1031A00044050000F1050020D00500201C0000208F
:1031B000030000800E00002050460000084B094A22
:1031C000FF201A805A809A80DA800023064A074935
:1031D0001370074A087048708870C8701360704791
:1031E0000E000020DC050000F10500201C0000207E
:1031F000D00500200122024B52421A607047C0469F
:103200001800002010B5034A0621034802F09CF87C
:1032100010BDC0465CCE0000C6D50000E12170B5EF
:103220004902144803F06CFFFFF718FE0A2004F06F
:1032300069F90023FF21104A995401331D2BFBD15A
:10324000012200200D4B01001A6004230C4A0D4D91
:103250001468002CFCD02C680002013B2043116054
:10326000002BF5D10122084B1A6004F005F901F09A
:10327000CBF870BDB41B0020D405002000D0004066
:1032800000D1004008D5004004D00040F8B50B4EF6
:10329000070030000D0003F07BFF0400A84200DDB2
:1032A0002C003D00EB1B9C4205DD300003F07AFF53
:1032B00028700135F6E72000F8BDC046B41B002099
:1032C00010B50100014803F023FF10BDB41B00201E
:1032D00010B5054C200003F029FFE1212000490230
:1032E00003F00EFF10BDC046B41B0020C3070CD472
:1032F000064B1B68834208D8054B1B68984204D8CC
:10330000031F1B68002B00D018007047FC0500202D
:10331000F80500200023012210B50A489900013366
:103320004250642BFAD1084C084B00211A6020004F
:10333000074A08F067F8074B074A6360074B1A60B3
:1033400010BDC046842D002000060020080000208B
:10335000D40900003027000004060020F4050020F6
:1033600010B5044B044A1A60044B054A1A60FFF773
:10337000D1FF10BDFC05002000060020F80500204C
:10338000D40F0020044B1B681868000980B2023873
:10339000C343DB1718407047F405002000B59BB00D
:1033A0000200054901A808F071FB01A802F0C2F96A
:1033B00002F074FCFCE7C04628CF00000B4BC207AC
:1033C00004D4042804D80A4B00D00A4B18007047D4
:1033D0000F2203681A40031D042AF7D0064B092A5E
:1033E000F4D0064B032AF1D0054BEFE702CF0000E3
:1033F000A6CA0000A0CA00000CCF00001CCF00002D
:1034000013CF00000020064A0649131F18601368F6
:103410001B099BB202339B00D2188A42F5D3704736
:1034200004060020D40F0020F7B50F240126314BED
:10343000314A1968314B324D186813681F00274014
:10344000072F26D813681B099BB202339B00D218A2
:10345000AA42F2D300242B4EA500AD192868FFF72D
:1034600045FF01342860642CF6D1274C2068FFF713
:103470003DFF2060254C2068002802D0FFF736FF72
:1034800020600025224B1B680093009B9D4214DBAB
:10349000F7BD1B099BB29B00D3189A42D2D01F687C
:1034A000374208D1B94206D2B84204D3043F3F683C
:1034B000002F00D01F60043BEFE7F0236B43154A59
:1034C0009B181A78002A01D10135DEE71F693C23D9
:1034D00000266B43DB199B0001930136BB1BF3D421
:1034E000019BB4001C1B0B4B1C19A069FFF7FEFECF
:1034F000A061F2E7FC05002004060020F80500208A
:10350000D40F0020842D002008000020D40F0020BC
:10351000CC0500202C1C0020F7B50124204246D108
:10352000234B1B689C46984241D3224B1B68019356
:1035300098423CD8031F1B68002B38D10200036857
:1035400000941B099BB2002B0FD10099131F196027
:1035500090422CD015682B1F1B68990069180C68C5
:10356000013B14600A602A00EDE79D0055192968A7
:10357000009C214219D18C4517D8019C8C4214D350
:103580000E1F3468002C10D10F680F343C40072CFC
:1035900008D92F60151F2B600B680A601B099BB2AE
:1035A0000A00D0E700993160CDE7013BCBE7F7BDDA
:1035B000FC050020F80500200D4970B50A000D4DEE
:1035C0001368141F1B0926689BB2981C002E0BD091
:1035D00000238A4200D00B0023608300C9188000BA
:1035E0001218AA42ECD370BD1B011360F7E7C04666
:1035F00004060020D40F0020F8B5124C27000F223B
:103600003B681D09ADB213420DD06E1CB600A74237
:1036100004D032003900200007F0E1FE0022A31997
:103620000436A4191A600235AD00074B7F199F427A
:10363000E5D31B1B9B10013B1B012360034B1C604C
:10364000F8BDC04604060020D40F0020F405002079
:10365000F0B59BB0FFF714FC00240700214AA3003B
:10366000D0580134FFF758FF642CF7D11E4B18686F
:10367000FFF752FF1D4B1868002801D0FFF74CFFE1
:1036800000261B4B1B689E4217DBFFF795FFFFF7D9
:10369000CBFEFFF7B1FFFFF7F3FB164BC21B1B6816
:1036A00015491B6801A81B099BB2023B08F0EEF903
:1036B00001A802F03FF81BB0F0BDF02575430F4B99
:1036C000ED182B78002B01D10136DAE72B695C1E4F
:1036D000002CF9DBA300EB189869FFF71DFF013CF4
:1036E000F6E7C046842D002008000020D40F0020FB
:1036F000CC050020F4050020E2CE00002C1C0020A8
:10370000F7B5174D4F1C2B6806001B680C001B09F2
:103710009BB201929F420BDBFFF79AFF2B681B685D
:103720001B099BB29F4203DB0A20FDF7C5FDFEBDCE
:103730002868A71CBA00DB1B81181B010B602960DD
:103740000021031F19600F231E400300240126439C
:1037500040C3083A9A189A42E9D9019902C3FAE794
:10376000F4050020F7B503000122134004000D000A
:103770000193002B2BD1174B1B68834227D8164B84
:103780001B68834223D90F23144F38600068184008
:10379000FFF7B6FF019B3C68061E3B6017D023680D
:1037A00004301B099BB29D4200DD1D00AA00211DB3
:1037B000251F07F00BFEFFF725FE2E60FFF734FEF6
:1037C00000232B602268064B134023603400200046
:1037D000FEBDC046FC050020F8050020D40F0020E7
:1037E000F0FF0F000323043010B5C117194009186A
:1037F000891000220420FFF783FF10BD70B505007B
:1038000008000C00FFF7EEFF0023002804D170BD74
:10381000E95CC21811710133A342F9DBE343DB1702
:103820001C40002304192371F1E7F0B50C009BB094
:10383000022804DC1C20FDF73FFD1BB0F0BD012376
:103840000868184206D1042804D90F2601683140BF
:10385000042901D00E20EEE761680D001D40F9D16A
:103860000429F7D90A683240042AF3D1A2681A421F
:1038700001D10D20DFE7FFF7A1FD06006068FFF72B
:103880009DFDA768010001AC7F103000257002F09B
:10389000E2FF39006423220003F042F8200008F020
:1038A0003BF901002000FFF7A9FFC6E710B51C4C4B
:1038B000A544041E02D1FFF795FF0BE002F0E4FEE1
:1038C0000138062828D805F0BBFB0909111829047E
:1038D000240000208023DB009D4410BD200002F066
:1038E0004FFF011B2000FFF789FFF3E7200002F0E4
:1038F000F5FE430001201843ECE780226946D20020
:10390000200002F002FF684608F006F90100684650
:10391000E9E704210348E6E70020CCE70420D9E7E3
:1039200000FCFFFF70CF000070B50C00022803DC24
:103930001C20FDF7C1FC70BD01230868184206D1A8
:10394000042804D90F2501682940042901D00E203C
:10395000EFE761681942FAD10429F8D90A682A40C8
:10396000042AF4D1A2681A4201D10D20E1E7FFF741
:1039700025FD05006068FFF721FDA46801006410C3
:10398000280002F068FF210002F0A5FFFFF78EFF7C
:10399000D1E770B50D00012803DC1C20FDF78CFC7D
:1039A00070BD01240868204206D1042804D90F21E3
:1039B00002680A40042A01D00E20EFE76A6822421A
:1039C000FAD1042AF8D913680B40042BF4D1FFF77D
:1039D000F5FC06006868FFF7F1FC0100300002F01A
:1039E0003AFF02F0BCFF40002043D9E7F8B50700DA
:1039F0000C001C20012F0BDD01250868284206D190
:103A0000042804D90F2102680A40042A03D00E209A
:103A1000FDF752FCF8BD62682A42F8D1042AF6D9B3
:103A200013680B40042BF2D1FFF7C8FC0600606856
:103A3000FFF7C4FC0100022F14D0A4682C4211D05F
:103A40006410300002F007FF050002F01DFE01289F
:103A500011D1002C02DD0135012C06D12800FFF721
:103A600025FFD7E701246442EBE7280002F094FE2B
:103A7000013C0500F0E70228F0D1002CEEDD013515
:103A8000012CEBD000222800110002F0B7FE02F05A
:103A900083FE013C0500F3E710B5012408680440EB
:103AA00016D04410200005F0FDFD154905F0C8FCB6
:103AB00007F0AEFB03F0F6FF0022124B06F062FDAA
:103AC00003F098FF07F034FB43000120184310BDBA
:103AD000042810D90F2302681340042B07D1FFF7E5
:103AE0006DFC21000A2208F0DFF80400DAE7032B5E
:103AF00001D10430F5E70D20FDF7DEFBD2E7C0462B
:103B0000D30237390000D040086870B501240500A1
:103B1000254006D1042804D90F2302681340042B42
:103B200003D00E20FDF7C8FB70BDFFF747FC0378FC
:103B30002900233B5A4253411022C01808F0B4F820
:103B400080239B05C218044B9A4201D91420E9E74F
:103B500040002043E8E7C046FFFFFF3F10B5034A9F
:103B60000621034801F0F0FB10BDC04640CF000025
:103B700039CF00000020704710B51E20FDF79CFBD8
:103B800010BD10B51E20FDF797FB10BD10B51E200F
:103B9000FDF792FB10BD10B51E20FDF78DFB10BD8B
:103BA00010B51E20FDF788FB10BD10B51E20FDF7D7
:103BB00083FB10BD10B51E20FDF77EFB10BD10B5B8
:103BC0001E20FDF779FB10BD10B51E20FDF774FB1C
:103BD00010BD10B51E20FDF76FFB10BD10B5034AD8
:103BE0000B21034801F0B0FB10BDC046ACCF000074
:103BF00004D000000120034B1860034B1B68834076
:103C000018437047F80F0020D80F0020F0B5EFF3ED
:103C100010810123194083F31088134C134AA446E2
:103C20001268134E013A9340124F134A002B17D0DB
:103C3000146803420FD03D682C60C046C046C046A1
:103C4000C046C046C046C046C0460C4C15682468F5
:103C500025605B08EAE765462C6014683460F8E785
:103C600081F31088F0BDC0460805005020000020F8
:103C70000C050050E40F0020EC0F0020E00F0020A6
:103C800030B585B001AD0C220649280007F09EFB37
:103C90000024285D01210134FFF70AF90C2CF8D12A
:103CA00005B030BD99D00000F7B56A46394B01AD7B
:103CB00013801C239370384B2B800A23AB70FFF7C3
:103CC000DFF8364B364CC0182368984201D20023E7
:103CD00023602668002E3DD16B469F5D0121380090
:103CE000FFF7E6F801360021380003F081FD032ECE
:103CF000F2D10026AF5D01213800FFF7D9F8013677
:103D00000121380003F074FD032EF3D1C8200138DF
:103D1000C046C046C046C046C046C046C046C04673
:103D2000C046C046C046C046F1D100212878FFF702
:103D3000BFF868780021FFF7BBF8A8780021FFF7EB
:103D4000B7F8FFF79DF8FA2300251B01C018206083
:103D50002800FEBDFFF794F8236800259842F7D3AA
:103D6000032003F0D5FB0600042003F0D1FB361836
:103D70000A2003F0CDFB0B4B9B1B181A0A4BA842E1
:103D800006DB18600023094A236013600125DFE782
:103D90001D60F7E71A1B0000030400001027000055
:103DA000F00F0020E3030000D80F0020F80F0020E0
:103DB0000022054B10B51A60044B1B68934201D0DA
:103DC00002F002FC002010BDF40F0020D81A0020E1
:103DD00010B5041E10DA00240A4BA400E258012397
:103DE0009340094A09491360094A1160094A0A497E
:103DF00011600A4A136010BDFFF758F8A042EADDCF
:103E0000EAE7C0469CDD0000EC0F002008050050EA
:103E1000E40F0020E00F00200C05005018050050B2
:103E20002B4BF7B51B680C00002B03D1012040423F
:103E3000FFF7CEFF24680126250035401AD0FF2267
:103E40006310120260121040DAB21043FF221B020C
:103E50001204134018431F4B1B68202B06D1B4409B
:103E60001D4BA40EA400E35800021843FFF7CEFE3A
:103E70000020FEBD042CFBD90F2322681340092B20
:103E8000F6D1FF2763683F025B100193019B9D42BF
:103E9000EEDAAB00E3189B68334216D05A10581282
:103EA000D1B238400843FF21120209040A401043EE
:103EB000084A1268202A06D15B009B0E06499B0027
:103EC000020258581043FFF7A1FE0135DEE7C04655
:103ED000EC0F00202000002080D2000002000868C3
:103EE00010B5C3070FD540101823012A03DD4A6817
:103EF000042A00D10833054A1360FEF7F9FFFFF7E3
:103F000067FF002010BD01204042EDE720000020A7
:103F100010B50124044002D04410200010BD042834
:103F200010D90F2302681340042B07D1FFF746FA7C
:103F300021000A2207F0B8FE0400EEE7032B01D1AE
:103F40000430F5E70D20FDF7B7F9E6E70868F8B5A6
:103F5000C3071AD5FFF7DCFF0300203B5E2B25D8F3
:103F60000520434301221D180020114E9D4219D007
:103F700005211024F75C3C4200D080180139520022
:103F800064100029F7D10133F0E704280ED90F227D
:103F900003681A40042A09D11B099BB2002B05D0E3
:103FA0000379DAE7012340001843F8BD0120FCE75C
:103FB000A5D0000070B508680D00FFF7A9FF040048
:103FC0006868FFF7A5FF621E0100042A14D8451E89
:103FD000042D11D805236B439B18012215009D4029
:103FE0002B00064805682B430360054B1B68002B1C
:103FF00002D0200002F0E9FA002070BDF40F00208A
:10400000D81A002070B508680D00FFF781FF040082
:104010006868FFF77DFF621E0100042A13D8451E61
:10402000042D10D805236B439B1801229A400748A2
:10403000036893430360064B1B68002B03D00022E8
:10404000200002F0C2FA002070BDC046F40F00202C
:10405000D81A0020F0B5050089B008680C00FFF7F9
:1040600057FF0690022D36DD6068FFF751FF019083
:10407000A068FFF74DFF04000127231D661E07936C
:10408000731C0293079B9E4235D00523734305930F
:10409000019B019D05330493049BAB421ED0042E6B
:1040A00016D86B1E042B13D80122059B2349013B14
:1040B0005B199A409446224A0B681068069A3A4067
:1040C00003920DD062461A430A60012200280DD1E6
:1040D0007F000135E0E701240194CDE7029ECFE7A0
:1040E000624693430B600028F2D0039A029928009D
:1040F00002F06BFAECE7019B1E1D042E1AD8012C6E
:1041000018D1002505273B0021006B439B199940DE
:104110000B000A4A013511689943094B11601B686D
:10412000002B05D0019B0022581D290002F04DFAFA
:10413000052DE8D1002009B0F0BDC046F40F0020E5
:10414000D81A0020086810B5C30703D5FFF7E0FEB2
:10415000054B1860054B1B68002B03D0024B1868F9
:1041600002F034FA002010BDF40F0020D81A00200D
:104170007FB5A04C2368002B0AD19F4A1268002A01
:1041800006D19E4B1B68002B01D0FFF78DFD7FBD34
:104190009B4D2A68002A26D1984A1268002A1BD013
:1041A000FFF782FD0028F2D0FFF76AFD924B2468EA
:1041B0001A681C60002A16D0002C14D101AD0C2204
:1041C0009049280007F002F9285D00210134FEF72C
:1041D0006FFE0C2CF8D1DAE7874A1268002AE5D185
:1041E000002BE3D0E0E700211A2003F001FB0021BF
:1041F0001B2003F0FDFA00211C2003F0F9FA2E68C1
:10420000012E5CD0022E00D1A2E0002E50D101364A
:104210003100794C03202368994303F0E9FA042024
:10422000216801404B42594103F0E2FA1021236812
:104230000A2019404B42594103F0DAFA80212368E1
:10424000090119404B425941062003F0D1FA80215F
:104250002368090219404B425941072003F0C8FA6C
:1042600080212368490219404B425941092003F03B
:10427000BFFA80212368890219404B425941192015
:1042800003F0B6FA80212368C90219404B42594114
:10429000182003F0ADFA802321681B0319404B421C
:1042A0005941172003F0A4FA31001A2003F0A0FAB4
:1042B0002B680321581C05F047F8296067E70221A5
:1042C0004D4C1720236819404B42594103F090FA96
:1042D00008212368182019404B42594103F088FAFD
:1042E00080212368C90019404B425941042003F042
:1042F0007FFA80212368490119404B4259410A2025
:1043000003F076FA80212368C90119404B425941D4
:10431000032003F06DFA80212368890319404B4282
:104320005941092003F064FA802321681B041940D5
:104330004B425941192003F05BFA3100062003F08B
:1043400057FA3100072003F053FA31001B20ADE784
:104350002021294C1720236819404B42594103F072
:1043600047FA40212368182019404B42594103F075
:104370003FFA80212368192019404B42594103F02C
:1043800037FA80212368490019404B4259410920DE
:1043900003F02EFA80212368890019404B425941CD
:1043A000072003F025FA80212368890119404B4238
:1043B0005941062003F01CFA802123684903194063
:1043C0004B4259410A2003F013FA80212368C903A4
:1043D00019404B425941032003F00AFA8023216817
:1043E0005B0419404B425941042003F001FA0121BA
:1043F0001C205BE7F40F0020E80F0020F80F0020DE
:10440000DC0F002099D00000012010B54042FFF7DA
:10441000DFFC10BD10B5034A0921034800F094FFEA
:1044200010BDC04680D30000C8D3000030B50224C0
:104430008025094B094AED009C505C59002CFCD0AA
:10444000A124E400884202D30021995030BD802588
:10445000ED0018514019F5E700E0014004050000A7
:1044600010B5002806D1C020B02140028902FFF714
:10447000DDFF10BDB02080218002C902F7E70000F7
:1044800043425841064B40421840B0239B02C0189B
:10449000036800201A0E532A01D11B02180A704724
:1044A00000C0FEFF30B501248025054B054AED0014
:1044B0009C505C59002CFCD001600021995030BD0B
:1044C00000E001400405000043425841074B4042D0
:1044D0001840B0239B02C018A62310B50902DB05C3
:1044E000090A1943FFF7DEFF10BDC04600C0FEFFFA
:1044F00070B5012480250D4B0D4EED009C515C598B
:10450000002CFCD0002902DC00229A5170BD5578A5
:1045100014782D0225439478013924042543D47856
:10452000043224062C4310C0ECE7C04600E00140F2
:104530000405000070B505004B680A009C1C2100B2
:10454000A400FFF7D5FF281970BD0000134B1B68AE
:10455000002B0CD08022B023D2029B0200280BD16A
:104560001A1D5B681B0E522B00D110007047B02241
:10457000C02392025B02F1E782420DD903681B0E51
:10458000522B09D1436802339B00C018824203D9E1
:1045900003681B0E522BE9D00020E7E7FC10002037
:1045A000F0B50020B7B00024FFF7D0FF27000500CA
:1045B0002600002D2ED1284D2868FFF761FF32001C
:1045C0003B0001900094254904A807F05FFA04A875
:1045D00001F0B0F8224B64201C682B68A0215A42DD
:1045E0005341204A5B421340B02292029B18E41AC6
:1045F0006043490204F0C2FDA0225202030000926F
:104600001949220004A807F041FA04A801F092F821
:1046100037B0F0BDFF226B6829689C460233FF1853
:104620000B12013613409C4200DA1C00FF200A14D2
:10463000024003926246014001920091039A0B49A5
:1046400004A807F023FA04A801F074F82800FFF783
:104650007DFF0500ADE7C046FC100020D2D400006D
:104660000011002000C0FEFF7CD40000BED400007A
:1046700070B50020FFF704FF04000120FFF700FFE2
:10468000844200DA04000A4B1D686A425541280042
:104690001D60FFF7E5FEA0226B4252021340054A5F
:1046A00028009B18044A611C1360FFF70DFF70BDC2
:1046B000FC1000200480010000110020F8B500204B
:1046C000FFF7DEFE07000120FFF7DAFE3E00204D77
:1046D0000643204C0DD18021C020C9024002FFF7C3
:1046E000A5FE01213000FFF7EFFE1B4B2E6023607B
:1046F0001DE0874209DD0023B0212B60164B8902A3
:10470000236023680020012517E0012380212B600E
:10471000124BC9022360F4E7120E522A08D0002877
:1047200000D023600E4801F005F8FFF7A1FFF8BDA7
:1047300028005A68023292009B188B4205D21A68F0
:10474000561CE9D10028F2D0D1E72160EFE7C0463E
:10475000FC100020001100200480010004C00200B1
:1047600097D4000070B50020FFF7F0FEFF2605008B
:10477000002801D1280070BD03681C143440FFF7E5
:10478000E5FEDA2CF4D10500F2E700008022F0B556
:104790005200A1B00021674806F034FE80220021BB
:1047A0005200654806F02EFE644BFF271B681A0076
:1047B000049353425A4110000592FFF751FE049CA6
:1047C0000020631E9C415E4B64421C405D4BE4181C
:1047D000FFF7C8FF0600002E2DD10498FFF750FE0A
:1047E000411C0598FFF770FE059A574D534B2C60FE
:1047F0001A60FEF76DFD514B64201B68A0215A42E0
:1048000053414F4A5B421340B0222C6892029B18DE
:10481000E41A6043490204F0B1FCA02252020300F2
:1048200000924A49220007A807F030F907A800F0D3
:1048300081FF21B0F0BD3268131412123A403B40A0
:1048400003921A000A3A092A49D83A4B039A995C0A
:10485000002931D110223E4806F0D4FD35002B68E6
:1048600003991A123A40914209D11A143A400B2A7C
:1048700027D0132A2DD00A2A01D1354B1D602800DC
:10488000FFF764FE051EEAD1314B196800290FD0ED
:104890002000FFF74FFE04002D4B5B1959680029DB
:1048A00003D02000FFF746FE040004350C2DF3D1A1
:1048B000204B0121039A99543000FFF747FE060070
:1048C00089E73B40022BDADC214A9B00D3185D606C
:1048D000D5E7102200211E4806F094FDCFE71A000C
:1048E000153A082AE8D8144A0399525C002AE3D101
:1048F0003500152B00D01500300003681A143A401B
:10490000152A0FD01D2A00D10025FFF71FFE002811
:10491000F3D1002D04D020002900FFF70BFE040086
:10492000054BC6E7039A1B123B409A42EDD10500A6
:10493000EBE7C046FC0F002004110020FC10002013
:1049400000C0FEFF04C002000011002061D400007E
:10495000142F002010B5FFF719FF10BDF0B585B07A
:10496000039203220333DC17294D1440E4182B680B
:10497000284F5A42534180225B42D202A4103B404E
:104980009B18A21C0291244E910000910190316865
:1049900000980A18934215D2FFF7F8FE2B685A4286
:1049A000534180225B421F40D202BF183368009AF5
:1049B0009B189F4206D2194800F0BCFE0025280033
:1049C00005B0F0BD029B356819066B461A7BA4231F
:1049D000DB051343FF222F00090C1943019B12042E
:1049E0001B04134019432800FFF75CFD0837281DFE
:1049F00021003760FFF756FD002C04D00A9A2100F1
:104A00003800FFF775FD009B083BFF183760D6E7BD
:104A1000FC10002000C0FEFF001100203BD400006D
:104A200070B59AB0FFF74AFEFF221E4CD20000215B
:104A3000200006F0E7FCFF25FFF794FE0026002883
:104A400014D10200C300E3580130591E8B41D21823
:104A5000FF28F7D1144901A807F018F801A800F0C1
:104A600069FE124800F066FE1AB070BD03681A14A1
:104A70002A400A2A0AD11A122A40FF2A03D0D20059
:104A8000A1180B71A050FFF761FDD8E7132AFAD1E6
:104A90001B122B40FF2BF6D0DB00E2181671E650FC
:104AA000F1E7C0468C25002007D500001BD500008B
:104AB0000021094B094A59600131516059680029A8
:104AC000FCD000211961012393600222044B813143
:104AD000FF315A501A607047FC100040001000402F
:104AE00000E100E00222064B0121DA670022054BBB
:104AF0005A61054A11615A69002AFCD07047C046C4
:104B000004E100E0FC1000400010004010B5044C2F
:104B10002378002B01D0FFF7E5FF0020207010BDA7
:104B200005120020802301205B055B6E5B001843AB
:104B3000704700000120024B1B685B001843704760
:104B4000881200200120024B1B685B00184370474D
:104B5000240000200120024B1B685B0018437047B3
:104B60008C12002070B504000D001600FEF792F9BB
:104B7000802301215B055A6E267000265300617068
:104B8000E1706272010A5A0A6071A171A272010C8D
:104B90005A0C000E5B0EA6702571E1712072E27254
:104BA000237370BD10B5044C200006F0B5FF010062
:104BB0002000FEF723FE10BD911200200E4B10B511
:104BC0001B680E4C5A1C0FD00D4C002B0CD00D4CFA
:104BD000012B09D00C4C022B06D0094C042B03D01E
:104BE0000A4C052B00D1074C200006F095FF010070
:104BF0002000FEF703FE10BD28000020ACD5000009
:104C000034CE0000B7D500003BCE0000B1D5000087
:104C100070B5214C2278002A3DD1204B01215A60E9
:104C20008022D20511605A68002AFCD00022072099
:104C30001B4B1C4901255A500439585008315A5011
:104C400019481A4958501A491A485A501A495A507C
:104C5000A622D2009D50082218495A5004315850BB
:104C60000220174958501749174858501748043917
:104C70005850182016495850C12189005A500539FA
:104C8000FF395858921802435A501249124A995003
:104C9000FFF70EFF257070BD05120020FC000040DC
:104CA000001000400C050000746962751C050000CE
:104CB00024050000200004022C050000140500005B
:104CC000340500003C050000FFFF0000211001003A
:104CD00054050000061200200405000070B50E4BBC
:104CE00006001B78002B01D1FFF792FF00200B4D2F
:104CF0002C7884420ED00A4B202219780323091BFA
:104D00001940084B4901C918300006F05FFB01202B
:104D1000013C2C7070BDC04605120020901200208E
:104D20000412002006120020002370B588B09842BB
:104D300035DD0D6801262C0034409C422FD1230024
:104D4000042D2CD90F222B681A402300092A26D1C2
:104D50006A683F2A23DD6846FFF7C0FF230000286A
:104D60001DD06B4619783300A14203DB6B461B5DF7
:104D70005B003343A200AA1801349360202CF2D1C7
:104D8000092169444A780B7812021A438B781B0474
:104D90001A43CB781B061343024A136004231800FE
:104DA00008B070BD8C12002070B5454B8AB01B78DE
:104DB000002B01D1FFF72CFF02AC2000FFF78EFF84
:104DC000002802D100200AB070BD23780B2BF9D93E
:104DD0006378012BF6D1E378012BF3D10023112066
:104DE000384E394D33602B7068442379374A417807
:104DF0001360027809021143827812041143C278C9
:104E000012060A4332490A60002B0ED1152169446B
:104E10004A780B7812021A438B781B041A43CB781A
:104E20001B0613433360002318E0012B1AD1152110
:104E300069444A780B7812021A438B781B041A4390
:104E4000CB781A211B06134333600E23627C69441E
:104E5000934200DD130000229A422CD1002204204C
:104E6000EA54B0E7022B03D1627B10331621EEE740
:104E7000042B0DD1152108226944684606F0A6FAD4
:104E80000098019902F026FD06F052F93060CAE759
:104E9000052BC8D1152108226944684606F096FA08
:104EA0000098019902F016FD06F042F93060627D2B
:104EB0000A231E21CBE7885CA8540132CCE7C04608
:104EC00005120020881200209112002028000020E6
:104ED0008C12002010B5134B04001B78002B01D15D
:104EE000FFF796FEFFF7FEFD00200F4A0F49104B1B
:104EF000545058600130106058680028FCD00020E1
:104F000018610130906018690028FCD0094B0A48EC
:104F10001B785B011B185350FFF7E4FDFFF7C8FD3A
:104F200010BDC0460512002000100040040500001E
:104F3000FC100040041200200612002010B588B0BA
:104F400000281DDD0A68012113000B4018D1042A36
:104F500016D90F2014682040092811D150683F2825
:104F60000EDD9800101880680024084201D040101F
:104F7000C4B26846C4540133202BF2D1FFF7AAFF14
:104F8000002008B010BD000010B5002813DD0C682B
:104F9000E30710D56410532C0DD8084B1B78002B59
:104FA00001D1FFF735FEFFF79DFDA123044ADB0089
:104FB000D450FFF77DFD002010BDC0460512002033
:104FC0000010004010B500280EDD0C68E3070BD57B
:104FD0006410FF2C08D8054B1B78002B01D1FFF77C
:104FE00017FE034A034BD450002010BD05120020C9
:104FF000001000402405000013B5002814DD0C68E3
:10500000E30711D5094B64100093094B0193072C5A
:105010000AD8084B1B78002B01D1FFF7F9FD6B462E
:10502000054A1957054BD150002016BDE2ECF0F4AB
:10503000F8FC000405120020001000400C050000E0
:1050400070B588B0002820DD0124086804401CD118
:1050500004281AD90F2302681340042B15D1FEF738
:10506000ADF9060006F058FD0500122800D91225FA
:105070002A0002210D326846FFF774FD6B465D730E
:10508000A54205DC6846FFF725FF002008B070BD8B
:105090002300325D6B449A730134F1E7F0B50D00E3
:1050A0008BB0012832DD08680122040014402DD1A4
:1050B00004282BD90F2301680B40042B26D16B68E1
:1050C000134223D0FEF77AF96E680700731001933C
:1050D00006F022FD05000E2800D90E252A00012128
:1050E000113202A8FFF73EFD6A46127902AB5A73ED
:1050F00002AA73129373019B76141B0ED67313745A
:105100005574A54205DC02A8FFF7E4FE00200BB0B1
:10511000F0BD3A5D02A963189A740134F1E730B525
:1051200089B0002814DD0C68E30711D51022684609
:105130000021FFF717FD6B466A4665105D736846F0
:1051400063122D0E64149373D4731574FFF7C2FEAB
:10515000002009B030BD0000174B184A59680029DB
:1051600003D00021596001319160196900291FD0D5
:10517000002018618023DB00D3581149012B18D17E
:10518000A923DB00D3585B420B600E490B78032B3D
:1051900001D801330B7003200B490B780133034016
:1051A0000B700A495B015B18094953500123936056
:1051B00070470860FAE7C046FC100040001000404D
:1051C000240000209012002004120020061200206B
:1051D0000405000010B5034A1021034800F0B4F89C
:1051E00010BDC0462CD5000023D50000044A054957
:1051F0001368C85401339B059B0D13607047C0466C
:10520000C0160020C012002070B5114C114A23684E
:10521000834202DC0023236016E0155C411C2E0053
:10522000FA3E012E05D899420FDA555C013D1F2D3B
:1052300001D90800ECE70100151A565C6E540131E3
:105240008B42FADC181A206070BD1570FAE7C04670
:10525000CC1A0020CC16002010B5FDF711FE064B2D
:105260001A68824201D900221A601B68C31A0348D7
:1052700098428041404210BDBC120020204E0000E8
:1052800010B5094C094A23681268934200D110BD39
:10529000074AD05CFEF714F80028F8D023680133E1
:1052A0009B059B0D2360ECE7C4160020C016002070
:1052B000C012002010B50400064B074A1B68126894
:1052C0009B1ADB439B059B0DA34200DB10BDFFF740
:1052D000D7FFF1E7C0160020C4160020F7B505007F
:1052E00056680191B000441C06301700FFF7E2FF3A
:1052F000FB20FFF77BFF1C20FFF778FFE8B2FFF7EA
:1053000075FFE0B22412FFF771FFE0B2FFF76EFF06
:105310006B461879FFF76AFF0025AE4200DCF7BD47
:10532000AB00FB189C680135E0B2FFF75FFF20126D
:10533000C0B2FFF75BFF2014C0B2FFF757FF200E8B
:10534000FFF754FFE9E7000070B5074E33680B2BF9
:1053500008DC0C255D43054C01332851641961605C
:10536000A260336070BDC046C8160020242F002004
:1053700010B5FBF7A5FEFFF74DF8FBF7C9FEFDF7EB
:1053800041FFFEF7EBFBFEF729FCFFF723FF00F0E0
:1053900015FF01F01DF901F067FB10BD962210B555
:1053A00012010021034806F02DF80022024B1A607A
:1053B00010BDC0462C1C0020CC050020064B074A1F
:1053C0001B6812689B1ADB439B059B0D01228342DD
:1053D00000DC002210007047C0160020C416002018
:1053E000F8B505000C0016001F1E0ED10320FFF7B4
:1053F000E5FF002808D0FA20FFF7F8FEE8B2FFF733
:10540000F5FEE0B2FFF7F2FEF8BD501DFFF7D6FF44
:105410000028F9D0FB20FFF7E9FEE8B2FFF7E6FE2F
:10542000E0B2FFF7E3FEF0B2FFF7E0FE3012C0B2E9
:10543000FFF7DCFE3C00E31B9E42E5DD2078FFF732
:10544000D5FE0134F7E7000070B50024F0250B4BC2
:105450001B68A34202DCFFF7A1FF70BD2B00634372
:10546000074A9B181A78002A05D059780023112082
:105470001A00FFF7B5FF0134E9E7C046CC0500206C
:105480002C1C0020F8B507000024F0252B006343F6
:105490000C4A01349E18B74211D0317800290BD044
:1054A0000133D15C002311201A00FFF799FF2A0075
:1054B0000021300005F0A6FF0A2CE7D1F8BD024B11
:1054C0001C60F9E72C1C0020CC050020F0B515006D
:1054D00001222F00754C1740A54401900291002F26
:1054E00011D005AB1A706A105A70120E1A7105228B
:1054F000691299706D140299DD70FFF771FFCF2367
:105500009B009D44F0BD042D1ED90F202A68104039
:10551000042826D1022304AA28001371FDF74EFFA8
:10552000040006F0F9FA624B984200D91800B8421C
:1055300004DC421C05AB02990198DEE701377B1EB3
:10554000E35C05AAD355F2E7042D00D0A9E00323BC
:1055500004AA043D13716B425D4105AB55710222F3
:10556000E9E709287ED1042205AB1A706A68511058
:1055700000916946521209789A70009A59701F2A50
:1055800001DD202200926A46127806ACDA70009B98
:10559000BB4202DC05ABE21ACDE70126BB00EB18EB
:1055A0009868064006D1042837D90F2103681940AE
:1055B00002290CD1012323704310637042121B0E89
:1055C0004014A270E070237105340137DFE704292D
:1055D00021D102232370FDF7F1FE039006F09CFA1F
:1055E000A31C0C2809D86070864201D19C19ECE7F5
:1055F000039A925D9A550136F6E70C226270039A7F
:10560000925D9A550136092EF9D12E23E372237348
:1056100063730E34D9E7012907D1032304382370BB
:105620004342584160700234CFE7092909D104236D
:10563000237043685A1062705B12A370E6700434E2
:10564000C3E703290BD1052323700068020992B236
:10565000430F92000B40D31A63701B12EDE72670C4
:105660000134B2E7032800D049E7052105AB1970E2
:10567000110989B2520F890002408A1A11129970D9
:105680005A701100642A00DD64210420D970C9B267
:10569000041FA14201DC04324DE72C5C1C54013094
:1056A000F6E7002D00D02AE751E7C046C4FCFFFF13
:1056B0002303000070B502000024F0210D4E080005
:1056C000604380194578954203D001340A2CF6D105
:1056D00070BDF022002105F095FE074A1368013BDA
:1056E000A34200D11460002329001A001120FFF703
:1056F00077FEEDE72C1C0020CC05002010B5B2B0E1
:1057000002236A460400137006F006FAC72800D97F
:10571000C7200023984207DC421C6B46FE21142060
:10572000FFF75EFE32B010BD694601335A1EA25C1F
:10573000CA54EFE730B5B3B002236A4605001370D0
:1057400006F0EAF90400C72800D9C72400239C42C8
:105750000BDC20003230FFF7ADFD621C6B46FF21F1
:105760001420FFF73DFE33B030BD694601335A1EA9
:10577000AA5CCA54EBE70000F0B5BBB004900C0083
:10578000012803DC1B20FBF797FD51E02A4B08683A
:105790000293C30709D4042807D90F2302681340D2
:1057A000042B02D1FDF70AFE0290234B606803939D
:1057B000C30709D4042807D90F2302681340042B18
:1057C00002D1FDF7FBFD039000271C4B1B680693DD
:1057D000069BBB420BDC039B194A0093C821029B2A
:1057E00008A806F021F908A8FFF7A4FFCAE70C26CD
:1057F0007E43144B0299F618306806F083F9051EB3
:1058000005D17368B6680793079B9D4201DB01379A
:10581000DEE730680399059606F074F9083600282B
:1058200008D121000498059B083102385B6898472D
:105830003BB0F0BD0135E7E738CF0000C8160020C7
:1058400088D60000242F0020F7B5234B06001B68E4
:10585000F02100930023009A9A4211DC0024F023E7
:105860001A006243019201991C4A55182F78002FA3
:1058700012D001340A2CF3D11948FFF75BFF29E05D
:105880000A005A43154882185078B04202D1127863
:10589000002A1FD10133DEE7F0223900280005F08D
:1058A000B1FD02230D4A0199EB6053540D4AF100FA
:1058B0008A58009B6E70AE70AA602F616F61A34220
:1058C00002DC054B01341C60002331001A0010205B
:1058D000FFF786FDF7BDC046CC0500202C1C00203C
:1058E000D1DA00008C25002010B5FFF7ADFDFF24B4
:1058F000084AE3005B429B18074AD35C043B012B38
:1059000003D8E043C0B2FFF79FFF013C002CEFD16A
:1059100010BDC046FC0700008C250020F7B50F0025
:10592000FF247F2501901E4AE300D31A1D4A9A18CE
:105930001278062A01D0032A20D1FF22D2009B1818
:10594000186883682B401C2B18D1C3681A002A40A2
:10595000042A13D102692A40192A0FD11B0A0133E4
:105960009B000C30C018FDF729FD03780600002BC2
:1059700010D006F0D1F80023B84209D0013C002C29
:10598000D1D1F7BD019AF15CD25C9142F6D10133DD
:105990009F42F7DCE043C0B2FFF756FFEEE7C04698
:1059A0008C250020FC07000070B50500FF24084A84
:1059B000E3005B429B18074AD35CAB4203D1E04350
:1059C000C0B2FFF741FF013C002CF0D170BDC046D2
:1059D000FC0700008C250020F7B5FDF751FA514B6C
:1059E0001A68824201D900221A601A684E49821A46
:1059F0008A4200D883E01860FDF74CFA071E00D1F8
:105A000001370020FDF738FB01900020FDF748FB2F
:105A1000019B0090454C464D002B14D02368002B71
:105A200000D07AE02B682760002B00D171E0414B59
:105A300001261B78002B63D10920FFF7B5FF3E4BF1
:105A40001E703C4B1E70009B002B12D02B68002B4D
:105A50000FD123682F60002B1ED0374B01261B78F7
:105A6000002B52D10920FFF79FFF334B1E70314BA3
:105A70001E702368002B0FD02F4E3278002A0BD1D6
:105A80009F4200D227602368FB1A312B04D90720DC
:105A9000FFF78AFF012333702B68002B0FD0254EB0
:105AA0003278002A0BD1BB4200D92F602B68FF1A35
:105AB000312F04D90820FFF777FF012333702368C3
:105AC000002B0CD0019B002B09D11B4E3378002BEF
:105AD00002D10720FFF768FF0023236033702B6893
:105AE000002B0CD0009B002B09D1124C2378002BEB
:105AF00002D10820FFF758FF00232B602370F7BD69
:105B00000720FFF751FF0C4B9CE70820FFF74CFFE5
:105B1000ADE7009B002B9CD1ABE7009A002A95D102
:105B2000AAE7C046B81200200F270000A8120020E4
:105B3000B0120020B4120020AC12002037B50024AF
:105B40000500FFF781FC01A80194FDF783FA21000D
:105B50002000FEF72DF9FEF70BFBFDF72FFBFDF7FD
:105B600049FBFEF751FCFDF7B1F9A54204D0FDF762
:105B7000D1FB0248FFF7DEFD37BDC046C2DA0000A8
:105B8000002310B501001A001120FFF729FC10BDF9
:105B900007B56B46197069465A7013128B7013144F
:105BA000120ECB700A716B46010005221320FFF71D
:105BB00017FC07BD10B50A0001001220FFF786FC94
:105BC00010BD70B5050008000C003230FFF772FB05
:105BD0002B00220000211B20FFF702FC70BD10B536
:105BE0000C000300110014202200FFF7F9FB10BD88
:105BF000012370B5FF24084A41185B42884201D353
:105C0000D84370BD06781D0A234073409B009B5803
:105C100001306B40F2E7C046A4D6000013B5040083
:105C2000FE2813D80A4BC200D05800280ED0436873
:105C300008309900FFF7DCFF01900920FFF73AFBDD
:105C400001AB042221001720FFF7CAFB13BDC04699
:105C50008C250020F7B50190FEF784FD0125040096
:105C6000FF276D42002C01D12800FEBD26683314A9
:105C70003B40152B0DD121000198083105F042FF62
:105C8000002801D135123D402000FEF75FFC0400E2
:105C9000E8E71D2BF8D101256D42F5E7F0B5802727
:105CA0009DB0FFF7EDFAA54CA54D2068FF00391A0D
:105CB0004019FDF7EBFA23680600C3182360002B98
:105CC0000ED11DB0F0BD2068391A2818FDF7DEFA94
:105CD000236806001B182360FDF7D2F8994B186063
:105CE000002EF0DC2B78FA2B00D037E12368022B52
:105CF00007DCFFF7B1FA0028E3D00120FFF784FAB0
:105D0000DFE76878AC78023818282BD803F0A2F9BE
:105D100019002C0030003400370040002A004A00EF
:105D20007C0086008A00A000F10002012A002A00FF
:105D30002A002A002A002A002A002A002A002A0013
:105D40001001FF2C0ED02000FFF7B4FC00227E4B88
:105D5000E100CA505B181A71210000921300132051
:105D6000FEF7FCFD0320C9E72000FFF76DFDF9E712
:105D70002000FFF79FFCF5E7FFF7B6FDF2E7FFF71E
:105D800063FB0020FFF7DAFE7048FFF7D3FCE9E77A
:105D9000632CE7D86E4BA200D25821001520FFF7E4
:105DA00095FBDFE7FEF7DEFCFF270400002CD9D0CF
:105DB00025682B143B40152B04D02000FEF7C6FBB2
:105DC0000400F3E72000083005F0A6FE06000530C9
:105DD000FFF770FAFB20FFF709FA2D121D20FFF7DD
:105DE00005FAE8B2FFF702FAF0B2FFF7FFF9301256
:105DF000C0B2FFF7FBF925002B1B9E42DDDD287AA0
:105E0000FFF7F4F90135F7E700211D2000910B00A1
:105E10000A00FEF7A3FDFDF77DFAA3E72000FFF7D8
:105E2000FDFE9FE7FDF73EF803AC4A4A642100906F
:105E3000494B200005F0F8FD02232000237005F0F7
:105E40006BFE2300020000211620FFF7C9FA89E744
:105E500000243D4AE300D558002D27D06B689E00F2
:105E6000701DFFF727FA2B000025320008332100B0
:105E70000120FFF7B5FA2F00FEF774FC2E00002872
:105E800018D1002F04D03A0001212000FFF726FA94
:105E9000002D04D02A0002212000FFF71FFA002E57
:105EA00004D0320000212000FFF718FA0134FF2C43
:105EB000CFD157E7FF2103681A120A40A24209D145
:105EC0001A140A400B2A08D10B400CD0012B0CD01D
:105ED000022B0CD0FEF73AFBD1E7132AFAD10025AA
:105EE0002F002E00F6E70600F4E70700F2E70500B2
:105EF000F0E70024FFF7A8FA220021000094230015
:105F0000DA20FEF72BFDFF222100D2000E4805F01B
:105F100079FA80E7012C02D1FEF742FB22E7022C3E
:105F200002D1FEF717FD1DE70120FFF707FE19E775
:105F3000002321001A001A2087E7C046CC1A00204F
:105F4000CC160020BC1200208C250020A4DA000012
:105F5000842D0020BBDA0000B6DA0000FB2B00D055
:105F6000CBE62268042A00DCC3E62E79E878574B9A
:105F7000360206439E4200DDBFE6331D9A4200DC36
:105F8000B7E6EB5CFE2B00D0B7E66B78AC78771EFB
:105F90001B2B61D019D8072B47D0082B1CD0012B05
:105FA00018D1FF2C16D02000FFF784FB6D79484AEA
:105FB000B31E009221002A000A20FEF7CFFC454BB9
:105FC000E400E0501B191D7104E01D2B56D048D38E
:105FD0001E2B6AD0701D91E6632CFBD86A79022AC9
:105FE00013D0032A1BD0012AF4D1E979AB79090235
:105FF00019432B7AA4001B0419436B7A1B060B432D
:106000005B001343344AA350E4E7002FE2DDB11EE6
:106010002F48FDF7F3FB304BA400E050DAE7AB79F3
:10602000A4005A1E93419B00ECE7632FD2DC03AD22
:106030003A002A49280005F0C9F900232800EB5549
:10604000FFF708FE0028C5DB234B8000C258210063
:106050001520FFF73BFABDE739002048FFF75EFC4B
:10606000B8E7FF2CB6D06A79022AB3D818490B20BA
:1060700000912100B31EFEF771FCABE7632F00DD3A
:106080006327002303A99F420ADCFB430022DB179E
:106090003B40CB181A70152000917B1C2100EAE7C9
:1060A000EA185279CA540133EDE7012C92D1002F3E
:1060B00090DD6B79002B03D01C00322B00DD3224E5
:1060C00064235C43064B1C6084E7C046F603000073
:1060D000D21600208C250020842D0020D11600200F
:1060E000040000200122094B1A60094A1368002BA2
:1060F000FCD00322074B1B68D8171040C01801239F
:1061000080100638400018437047C04600C0004069
:1061100000C1004008C500400120704710B5064C82
:10612000200000F0D7FD0549200000F0FBFD012212
:10613000034B1A6010BDC046FC1A0020801A0600EE
:10614000D01A002010B501210D20FCF7B1FE01216D
:106150000E20FCF7ADFE00210F20FCF7A9FE044C39
:10616000200000F0F3FC1021200000F00BFD10BD1A
:10617000DC1A002010B504680D20E30703D5641075
:10618000FF2C03D91720FBF797F810BDFFF7DAFFB4
:10619000E1B2024800F018FD0020F6E7DC1A00200A
:1061A00010B5FFF7CFFF0021034800F00DFD4300BD
:1061B0000120184310BDC046DC1A002010B5034A68
:1061C00008210348FFF7C0F810BDC046E8DA000018
:1061D00028DB00000D4B70B51B6804000E00150095
:1061E000002B01D1FFF79AFFE1B2094C200000F02B
:1061F00030FEF1B2200000F033FDE9B2200000F0E3
:106200002FFD200000F090FE70BDC046D01A002087
:10621000FC1A002010B501240368234205D0416810
:10622000214202D08268224203D10D20FBF744F8BC
:1062300010BD5810802801D91520F7E74910FF2913
:1062400001D91620F2E75210FF2A01D91720EDE7F5
:10625000FFF7C0FF0020EBE7F7B5012214009042E2
:1062600022DD0D682A421FD01D4B15411B684C686A
:10627000002B01D1FFF752FFE9B201272500194E8B
:106280003D40300000F0E5FD002D0FD03C413000D6
:10629000E1B200F0E5FC300000F046FE0024A04230
:1062A00002D02320FBF708F82000FEBD042CF2D911
:1062B0000F2322681340092BEDD163685B10019313
:1062C000019BAB42E7DDAB00E3189968394204D08B
:1062D0004910C9B2300000F0C3FC0135F0E7C046F8
:1062E000D01A0020FC1A0020154B70B51B68050061
:1062F0000E00002B01D1FFF711FF124CEDB2290067
:10630000200000F0A6FDF1B2200000F0A9FC002161
:10631000200000F0A9FD002801D0404270BD72B6F7
:1063200001222900200000F08FFD62B6200000F05D
:1063300088FC0028F2D0200000F088FCEEE7C04680
:10634000D01A0020FC1A002010B501240368234253
:1063500002D04168214203D10D20FAF7ADFF10BDF4
:106360005810802801D91520F7E74910FF2901D9D5
:106370001620F2E7FFF7B8FF40002043EFE70000E8
:1063800010B50D211D20FFF7AFFF164C5A2809D17B
:1063900001222A2122703D38FFF71CFF0122124BF7
:1063A0001A6010BD0F211920FFF79EFF332805D179
:1063B00002235F22237020211A38EDE70D211E20D1
:1063C000FFF792FFC7280AD1032300222A21A93808
:1063D0002370FFF7FFFE1B222A211E20DCE700238B
:1063E0002370DBE72C000020D41A0020204B10B5CE
:1063F0001B680400002B01D1FFF7C2FF1D4B1B7867
:106400005BB2022B0AD0032B29D0012B2CD1210007
:106410001D200124FFF768FF644205E0012C13D121
:1064200029211920FFF760FF7F2801DD0138FF389F
:1064300003007F3301DA7F204042C8237F21584385
:1064400002F09CFE604310BD032C0BD12B211920C0
:10645000FFF74AFF043CE7E72D211920D9E7210087
:106460001E20D6E7052CF7D0012400206442E4E783
:10647000D41A00202C00002010B50120FFF7B6FF31
:1064800043000120184310BD10B50320FFF7AEFFF5
:1064900043000120184310BD10B50520FFF7A6FFEB
:1064A00043000120184310BD144B70B51B68002B2E
:1064B00002D10120FFF79AFF114B1B785BB2013329
:1064C00001D1FFF75DFF0120FFF790FF04000320DB
:1064D000FFF78CFF05000520FFF788FF6D4364433D
:1064E00040436419201804F059FE01F023FB04F026
:1064F0001FFE43000120184370BDC046D41A00207F
:106500002C000020F8B501231C0098422BDD0F68F9
:106510003B4228D04E6835001D4024D1042E22D99C
:106520000F2231680A40092A1DD173685C10202CA3
:1065300000DD2024144B1B68002B01D1FFF7EEFD7A
:1065400072B67F10F9B2114F2200380000F07CFCC7
:1065500062B6A54214DA380000F073FB002804D1BB
:1065600001246D002C432000F8BD380000F06EFBC4
:106570000122AB004000F31810439860AD18E8E723
:1065800064000125EEE7C046D01A0020FC1A002066
:10659000002070470120704700207047002070479E
:1065A000012070470020704700207047002070478E
:1065B000002070470020704700207047002070477F
:1065C00000207047002070477047704770470000F8
:1065D00010B5034A0E210348FEF7B6FE10BDC046B3
:1065E00078DB0000E8DB00000378013B1F2B00D9BB
:1065F00070470130F8E710B5FFF7F6FF0378002B7E
:106600000BD00130222B11D10378002B03D0421C78
:10661000222B03D11000FFF7E7FF10BD5C2B03D145
:106620004378002B00D0821C1000EDE73A2BF2D00B
:106630002C2BF0D07B2B0BD1FFF7D6FF0378002B50
:10664000E9D07D2B01D10130E5E7FFF7D4FFF5E775
:1066500020225B2B14D1FFF7C7FF0378002BDAD081
:106660005D2BF0D0FFF7C7FFF7E7202BD3DD2C2BF6
:10667000D3D0190091435D29CFD0222BCDD001304A
:106680000378002BF1D1C6E7002210B5904216D056
:10669000FFF7AAFF03780422222B10D0023A7B2BAB
:1066A0000DD0013A5B2B0AD019003039023209298A
:1066B00005D92D2B05D14178303909290AD8100088
:1066C00010BD0522742BFAD00132662BF7D00132AF
:1066D0006E2BF4D0581E83415A42F0E770B5FFF795
:1066E00083FF037801222D2B01D18018023A002369
:1066F0000A2502E06B430130CB1801783039CCB267
:10670000092CF7D95A43100070BDF8B50C001500DC
:10671000FFF76AFF0378222B02D000232370F8BD15
:106720000D236A1E210008250C260A279C460130ED
:106730000378222B02D100230B70F0E7002BFAD054
:10674000441C5C2B0BD14378841C622B0ED0662B2F
:106750000ED06E2B0ED0722B0ED0742B0ED0002AC2
:10676000E9DD0B70013A01312000E1E72B00F6E78B
:106770003300F4E73B00F2E76346F0E70923EEE776
:1067800010B50400FFF737FFA04202D90378202B91
:1067900000D910BD0138F7E710B5002815D00378EF
:1067A000002B13D0FFF720FF2021037802008B433A
:1067B00000205D2B09D01000FFF71DFF03782C3B54
:1067C0005A425341C018FFF70FFF10BD1800FCE7F5
:1067D0000300002070B50C0081420EDD1A785B2AA0
:1067E0000BD1581CFFF700FF0125AC4205D0FFF785
:1067F000D3FF002801D00135F7E770BD70B50C005C
:106800001500002901D000230B70002820D0037848
:10681000002B1ED0FFF7E8FE037806002C2B03D1D7
:106820000130FFF7E1FE0600337800207D2B0FD00A
:10683000844204D02A0021003000FFF766FF3000B8
:10684000FFF7D9FE03783A2B02D10130FFF7CCFED7
:1068500070BD1800FCE7F0B50D0004009DB02E7867
:10686000002E35D02E21280005F03EF9071E14D049
:10687000431B0193303E092E14D82800FFF72EFF4A
:1068800001002000FFF7A4FF0400002C20D0002FFF
:106890001ED0019B0133ED18E1E7280005F03CF91B
:1068A0000190E7E723787B2B11D1601C642203A9B8
:1068B000FFF7A4FF041E0BD0019A290003A805F0DE
:1068C00032F90028E1D02000FFF795FEEEE7002422
:1068D00020001DB0F0BD70B5050000200C00814205
:1068E0001DDD2800FFF7D0FE0300681C012B14D02B
:1068F0000020022B13D10022681C1100FFF77EFF3D
:10690000012C0CD0FFF748FF00221100FFF776FFA3
:10691000013CF5E7FFF740FF013C012CFAD170BDC7
:10692000F8B5050000200C0016001F0081420DDDA7
:106930002800FFF7A9FE03000020022B06D1681CE7
:106940003A003100FFF75AFF012C00D1F8BDFFF7E4
:1069500023FF3A003100FFF751FF013CF4E710B587
:106960000024A04218D0FFF73FFE03787B2B0AD10A
:10697000013000221100FFF741FF00280CD0FFF783
:106980003AFE0134F5E75B2B06D10130FFF704FF37
:10699000002801D00134F9E7200010BDF8B5002827
:1069A00016DD0D68EB0713D56D10013D0124FDF7D1
:1069B000D9FE0026FF27644200280CD1002E21D0EA
:1069C000300005F0A9F801003000FCF717FFF8BD12
:1069D00001256D42EAE703681A143A40152A0BD1E3
:1069E0001B123B409C4200DA1C009D4201D1060074
:1069F0000836FDF7ABFDDFE71D2AFAD1012400269A
:106A00006442F6E70120013464002043DFE7000020
:106A100010B508680C00FCF7D1FCFFF71BF9002843
:106A200003DB6268024B8000C250002010BDC046EC
:106A3000842D002010B50868FCF7C0FCFFF70AF9A8
:106A40000123002802DB024B8000C358180010BD50
:106A5000842D002010B50868FCF7B0FCFFF7FAF8A9
:106A6000C043C00F800010BD10B5034A0421034885
:106A7000FEF76AFC10BDC04678DC000071DC000047
:106A800010B5FCF7CBFBFCF76BFCFEF771FC044880
:106A9000FEF750FEFDF7C4FFFEF726FF10BDC0460F
:106AA000C7DC000010B5FCF7B1F810BD70B50025CB
:106AB00004AC24780573A94205D10A4B0A4A232164
:106AC0000A4804F015FC01600949920052589B00E5
:106AD00002715B58A400837163588560437102237F
:106AE000C37170BDDFDC00003EDD0000EDDC0000A6
:106AF0009CDD0000037B002B04D14373837303618F
:106B000001330373704700001FB50191A0210024D9
:106B10000068C900D2B24450012A10D0A24209D064
:106B2000032A0AD0074A8350074B019AC250012317
:106B300043501FBD02221343F4E70422FBE7062261
:106B4000F9E7C046540500002405000010B5040014
:106B5000FFF7D0FFA1222368A179D2009950617973
:106B6000064A20009950217904329950044B196843
:106B70005A689B68FFF7C8FF10BDC0460C050000AF
:106B8000F01A00204BB2002B0FDB80233F290FD8D7
:106B90001F290FD80F290FD807290FD803290FD87D
:106BA0001B060168074A8B50704780239B04F8E757
:106BB000DB04F6E71B05F4E75B05F2E79B05F0E76E
:106BC000DB05EEE7240500000368074A99501A0028
:106BD000FC32D1680029FCD0A321C90058580023F9
:106BE000C0B2D3607047C0461C05000007B58022C4
:106BF000074BD2051A6000229A6002321A710F23E5
:106C00000C3200930349023B0348FFF74FFF07BDD7
:106C1000F01A002000300040DC1A0020F8B5050012
:106C20000E0017000024BC4208D02B68315D1B68A1
:106C300028009847002801D00134F4E72000F8BD6F
:106C4000704710B51C3000F0A9F910BD10B51C300C
:106C500000F096F910BD10B51C3000F0A5F910BD7C
:106C600070B5437E0D00002B01D1002070BD643053
:106C7000040000F0A2F90028F7D12000290000F05C
:106C800070F90120F2E70000F7B50193FA2300251F
:106C900004009B0083600D4B4560083303601C308B
:106CA0000F00160000F052F92000643000F04EF999
:106CB000074A2761B600B35820006375019B9B000B
:106CC0009B586576A576A375FEBDC0467CDD0000A9
:106CD0009CDD00000123A022C375837D0E49C133D2
:106CE000FF33D2059B009950437DC133FF339B0096
:106CF0009950CC220169094B5204CA5005220169FE
:106D0000243BCA50827D01690833CA500269417D23
:106D1000034BD1507047C0460C060000240500000C
:106D20000C050000A022002310B50469D200A35076
:106D30000A4CA1420FD90A4C8C425B4109495B4283
:106D40000B40CD21C9045B18046907496350052134
:106D50000369995010BDCC235B04F5E7A0860100C0
:106D600090D00300000098FD24050000F7B5040052
:106D700000200D000193824265D01600402A00D900
:106D8000402627001C37380000F0F6F8B1232269AE
:106D9000DB00D55080220123216992008B50A27E16
:106DA000002A03D122691362226913600025731E31
:106DB000AB4207D1019B002B04D080220221236922
:106DC00092009950012223691A622369FC33DA6820
:106DD000002A02D19A6A002AF9D09A6A002A0BD1B5
:106DE000DA60A3232269DB00D1583800C9B201352B
:106DF00000F0B7F8B542DAD3019B2269002B0FD11E
:106E00001300FC339B6A002B0AD10133A376D361B4
:106E10002369FC33DA6C002AFCD00022DA640AE031
:106E200000230121A37651611A002369FC3399687C
:106E30000029FCD09A602369FC339A6A002A01D0A9
:106E400000229A62E8B2FEBD10B50123FFF78EFF63
:106E500010BD0300AC3310B504001970643000F0AD
:106E60008BF80123637610BD0023020070B5AC32AD
:106E700043760D001178B12204000069D2008150E0
:106E80008022216992008B502269013313622269AA
:106E9000936026006436300000F080F8002812D09D
:106EA000300000F06DF81E4B2269D0502369FC338E
:106EB0001A6A002A02D19A6A002AF9D09A6A002A2C
:106EC00001D11A62E5E723690122002D0DD11900D5
:106ED000FC31896A002908D1DA612369FC33DA6C54
:106EE000002AFCD00022DA6407E05A612369FC33EF
:106EF0009A68002AFCD000229A6000202369FC33A3
:106F00009A6A82420BD098622169064A8B588B504C
:106F10001800022B03D0181F431E9841033070BD88
:106F20001C050000C404000010B50121FFF79CFF00
:106F300010BD000010B51323142202490248FFF7C8
:106F4000A3FE10BD00400040FC1A002010B54022F6
:106F50000021040004F056FA002320002364636437
:106F600010BD10B53F24026C531C2340446C9C425E
:106F700001D08154036410BD00230364436470474F
:106F8000436C026C934206D03F21C25C01330B403C
:106F900043641000704701204042FBE7036C406CE3
:106FA000181A00D540307047436C026C934201D0F0
:106FB000C05C704701204042FBE73F22036C406CFD
:106FC00001331340181A43425841C0B270470000C1
:106FD00003210A4802680A430260094802680A431A
:106FE00002600849084A094B9B1A03DD043BC85854
:106FF000D050FBDC00F012F8F9F786F824050040C9
:1070000054050040ECE20000000000206402002073
:10701000FEE7FEE7FEE7FEE7FEE7FEE72D4B10B5D5
:107020001A68D2B2012A0FD12B4A126812070BD16B
:107030002A4AE0241168F0220800104021422DD194
:107040002749096811422CD01A68D2B2012A12D1FC
:107050002149096809070ED1F0202049096801403B
:10706000402908D11E490968014204D18020C1216C
:10707000C005C90042501B68DBB2012B0DD1164B75
:107080001B681B0709D1154B1A68F0231A40A02A68
:107090000FD1134A12681A420ED010BD3028CFD03B
:1070A000D2E7104A104911608021104A090211608C
:1070B000CAE7D02AF1D1ECE70D4B1A68012A04D0B7
:1070C0000C4A1A601A68012AFCD1C0220A4B1A60C5
:1070D000E3E7C046E00F00F0E40F00F0E80F00F037
:1070E000EC0F00F004050040DFFF07C0186C004003
:1070F00000EC06407593000014EC06400120704738
:1071000010B503681322DB69984710BD7047000073
:10711000054B0269D1500369FC331A6A002AFCD07E
:10712000002201201A6270471C050000030010B500
:107130005C331A781F231A401E3B19009140114AF4
:10714000D167C222042104699200A15002695360F0
:107150000269D360A02300220169DB00CA50012329
:107160000169094A5B428B500169084A8B500169E9
:107170000C3A8B50016908328B501430FFF7FCFE3B
:1071800010BDC04604E100E00C050000140500003D
:1071900010B51430FFF702FF10BD10B51430FFF723
:1071A00003FF10BD10B51430FFF7EAFE10BD00005C
:1071B000030070B55E331A780469724BE250030025
:1071C0005D331A780469704BE250030061331C7818
:1071D00002696E4B012C00D09EE005005F352E78D1
:1071E000A225ED005651020060321578A1220669F1
:1071F000D200B5500269D4509623DB00994200D8E2
:107200008CE096231B01994200D88AE096235B010B
:10721000994200D888E096239B01994200D885E0E6
:10722000E1239B01994200D882E09623DB01994239
:1072300000D880E0E123DB01994200D87DE096236D
:107240001B02994200D87AE0E1231B02994200D840
:1072500077E096235B02994200D874E0E1235B0259
:10726000994200D871E0E1239B02994200D86EE078
:10727000474B994200D86CE0E123DB02994200D8E9
:107280006AE0E122002312038A425B41414A5B42E9
:107290001340802252059B1801693F4A8B50A0235E
:1072A00004220169DB00CA5000210369FC33D96064
:1072B0000369FC331962012301690B6001698B606A
:1072C000C1210469890062501F215C3002780A40A4
:1072D00093406231314AFF31535000214156002919
:1072E0003CDA0F230B40083B2D4C9B089B001B19DD
:1072F00003242140A140FC348C40DD69A5432C00CF
:10730000C0258D4029002143D9611F2301781940F0
:107310001E3B8B40136070BD00246CE79E23DB0294
:10732000BAE79D231B03B7E71E4BB5E71E4BB3E738
:10733000EC239B03B0E71D4BAEE71D4BACE71D4BA9
:10734000AAE71D4BA8E71D4BA6E71D4BA4E71D4B65
:10735000A2E78023DB049FE71B4B9DE78C080F4BC4
:10736000A400E41803230B40FF21C025DB00994053
:10737000AD0066598E433100C0269E4033000B435A
:107380006351C2E70C050000140500006C05000005
:1073900090D0030000D0BEFE2405000000E100E014
:1073A00000ED00E000B013000050270000A04E00E8
:1073B00000F0750000509D0000F0EB0000903A01D5
:1073C00000E0D70100B0AF0300705F07F7B500938E
:1073D00008AB1B7800250193FA2304009B0083600F
:1073E0000E4B45600833036014300F001600FFF7A2
:1073F000ADFD23005C3327611E70009B084A9B0093
:10740000995823005D331970019B20009B009A5806
:1074100023005E33DD701A70FEBDC04620DE000022
:107420009CDD0000036910B51A00FC32D26804002C
:10743000002A0AD0A322D20099581430C9B2FFF70B
:1074400090FD00222369FC33DA6010BD10B50248BC
:10745000FFF7E8FF10BDC046B41B0020162307B598
:10746000022200930249013B0248FFF7AFFF07BD2C
:1074700000200040B41B002010B5002801D004F00B
:107480007DFA10BD7047000010B500F011F8FFF74D
:10749000F9FF012000F000FAFFF7F2FAFFF702FB14
:1074A000024B002BFAD000E000BFF7E7000000001D
:1074B000C420114B80001A5810491140C0221202FA
:1074C0000A431A50C0218022490092025A501A6081
:1074D0008023A3220021DB05D20099500122F9303C
:1074E0009A60074BFF301950C120023180001950BB
:1074F000403019501A60704700E100E0FF00FFFFC4
:1075000000100140014B18607047C0467800002011
:10751000F7B5002320285AD8384B8000C258042AD7
:107520005BD007D8022A54D055D80423012A09D0A9
:1075300000234CE0062A54D051D31A2A53D00223F8
:107540001B2AF5D12E4A116808294ED909294FD096
:107550000A240226A02001252A4AC00015502A48E4
:107560002A4D07681C20BF00074029480197006882
:107570005759009027481B0207401F43C02300981B
:107580009B020340FF2057515759000207401F43F9
:10759000019B1F43009B58016023184007433E4353
:1075A000565101251C4B156058680028FCD000205E
:1075B0005860A1230125DB00D3585560A025ED00BC
:1075C00050511BB2A14202D015D2611ACB40180013
:1075D000FEBD0823B6E71023B4E72023B2E740231B
:1075E000B0E78023AEE70123ACE708240026B1E72B
:1075F0000C000126AEE7091B8B40E8E79CDD00008C
:1076000074000020007000403000002004050000DD
:1076100034000020FF00FFFFFC700040F0B5202880
:107620005BD8364B8000C258354B1E68002E30D1D7
:10763000C227344BBF00D859334C03250440C02027
:1076400000022043D851C0248020640080001851DB
:107650002E4F18602E4B803CD859FF3CA043D85188
:107660000437D859A8432043D8510837D8590C3586
:10767000A8438446072065462843D851A820C00067
:107680001E50C1208026800076021E501C601C4BBC
:107690001C60142500202B001E4C2E00464336593A
:1076A000771C1BD14343E250A0230325C132FF3294
:1076B0009200DB05D550184B1A68082A14D1142300
:1076C0004343E3189A6812485132FF3292005960DE
:1076D0001150DA68C1239B00C250F0BD9642E1D040
:1076E00001300328D9D1F8E7082A02D9083AD14055
:1076F000E5E708239A1A9140E1E7C0469CDD0000C7
:10770000181C002000E100E0FF00FFFF040500005E
:107710000090004038000020780000202149F0B59A
:107720004A6C2148002A14D0A025A1260023012458
:10773000ED05F600C258571C06D0C7187F68002F09
:1077400002D027009740AF5114333C2BF2D10023D5
:107750004B64A0230121DB0500260F009C46142367
:107760004B43C3181A1F1268104C0E4D9200141987
:107770005219526C002A10D01A00143A1268551C83
:1077800009D0103B1B68FF2B05D03B00934065469A
:107790001A00074BEA50FC34666401310429DED13B
:1077A000F0BDC046FC900040380000200090004032
:1077B0000C05000000B5202810D80C4A8000835822
:1077C00003290BD8A0220800C133FF33D2059B0048
:1077D00001F036FC020905070021D15000BD0C2143
:1077E000FBE70421F9E70321F7E7C0469CDD000031
:1077F00020280AD8074B8000C25801239340A022BA
:10780000D205002902D1044953507047A121C90073
:10781000FAE7C0469CDD00000C05000003000020D4
:10782000202B0AD8A021A222C905D2008858034AD9
:107830009B009B58D8400123184070479CDD0000F6
:10784000F7B506000D000C008B180193019B671B18
:107850009C4207D0336821781B6830009847013478
:107860000028F3D13800FEBD0849094A094B10B57C
:107870001B688858FA22190A1B0618439200002335
:1078800001F0B4FD4904C00B084310BD00100140D5
:10789000040500001C1C002070B5041E09D0FFF771
:1078A000E3FF050000F014F8FFF7DEFF401BA042E5
:1078B000F8D370BD0022044B9A60044A1368013368
:1078C000DBB213607047C046FC1001401C1C002056
:1078D00070470000F0B5C64600B5CB0F9846404A49
:1078E0004B005B0D9A1882B00D000400132A2FDCA8
:1078F000002A49DB3B4F17413E000E40064323D090
:107900007F08390029400C430AD03749BD438C46D3
:1079100063445C425C418023DB021341E4071D4366
:107920004146CE0031492B008E192200346875681B
:107930002000290001F000FF0090019100980199BA
:1079400022002B0003F090F802B004BC9046F0BD7A
:10795000332A08DD8023DB009A42F5D102000B00B8
:1079600001F0EAFEF0E7224A9446012263445242C3
:10797000DA400242E8D052080242D1D09443802239
:10798000D2051A411443CBE74B005B080343DBD01D
:107990000B031B0B1C436342234380244D0C240325
:1079A0001B0B23406D042B4319004346DA000F4B99
:1079B0009B181C685D6802000B002000290001F084
:1079C000BBFE009001910098019922002B0003F06A
:1079D0004BF842464B005B08D60733431900B3E728
:1079E00001FCFFFFFFFF0F00EEFBFFFF50DE00007A
:1079F000EDFBFFFFF8B5274A4B005B0D9A180C0012
:107A00000700132A10DC002A36DB234B13410B42FC
:107A10003AD0802424031441002064189C430600BB
:107A2000250030002900F8BD332A0EDD8023060032
:107A3000DB000D009A42F4D102000B003800210057
:107A400001F07AFE06000D00EBE7144D0600AC468F
:107A5000012563446D42DD40AC4663460D000342A0
:107A6000DFD033239A1A323B93401818874200D94B
:107A70004C1C63469843D2E7C90FCC070020531C27
:107A8000CDD1074B1C43CAE706000D000028C0D12A
:107A9000C7E7C04601FCFFFFFFFF0F00EDFBFFFF44
:107AA0000000F03F30B5214A4B0087B05B0893429D
:107AB0001EDD1F4A934205DD02000B0002F0D4FFD9
:107AC00007B030BD02AA00F095F803231840049ACD
:107AD000059B012813D002281DD0002814D002983D
:107AE000039900F06FFB80231B069C466144E7E787
:107AF000002300220093002301F0DEF8E0E7029863
:107B0000039900F05FFBDBE70124029803990094DE
:107B100001F0D2F8D4E7012402980399009401F00F
:107B2000CBF880231B069C466144C9E7FB21E93F53
:107B3000FFFFEF7FF0B54746CE4680B58DB004001D
:107B40000D0000F067FA294B06001B780F005BB2AE
:107B50009846013310D022002B002000290003F0AA
:107B6000CBFA8146002807D10022002320002900FB
:107B700001F014FC002806D1300039000DB00CBC17
:107B800090469946F0BD01230293194B0694079540
:107B900003934B460A93434604940595002B15D056
:107BA000002300221900100002F0E2F8434608907A
:107BB0000991022B0ED103F0B9FB212303600A9B2C
:107BC0000193002B0CD1089E099FD5E700230024C8
:107BD0000893099402A801F0C1F90028EFD1EAE75F
:107BE00003F0A4FB0A9B01930360ECE77C000020F8
:107BF00060DE0000F0B54E464546DE465746E0B52D
:107C0000E14B4C008FB09046894664089C4200DCF2
:107C100087E0DE4B9C4222DCDD4A002900DC92E05A
:107C2000DC4B02F021FFDB4B06000F009C4200D131
:107C30007EE1D94AD94B02F017FF02000B00414602
:107C400030000A604B60390002F00EFFD34BD24A7D
:107C500002F00AFF434601259860D9606BE0D04BE3
:107C60009C4200DC8FE0CF4B9C4200DD55E1CE4AC8
:107C7000231592469A4451460905631A19001D00BE
:107C8000040003F055FA03F089FA02000B0020000B
:107C900029000892099302F0E7FE0022C34B02F08C
:107CA00071FC0F00060003F043FA03F077FA0400BA
:107CB0000D0002000B00300039000A940B9502F011
:107CC000D3FE0022B94B02F05DFC002200230C9091
:107CD0000D9101F05DFB002800D192E1002300220C
:107CE0002000290001F054FB434243410133B04AD4
:107CF00041460192022208A80092524600F07CFB05
:107D00004B460500002B16DA8022434612069446A5
:107D100042465B68454263445360D3686344D36022
:107D200009E00B00020041460A604B60002200237C
:107D300000258A60CB6028000FB03CBC9046994675
:107D4000A246AB46F0BD934B01F0F6FC914B06000A
:107D50000F009C4200D13DE18F4A904B01F0ECFCBA
:107D600002000B00414630000A604B60390002F00F
:107D70007BFE894A894B01F0DFFC012543466D42B9
:107D80009860D960D7E701F049F88A4A8A4B060023
:107D90000F0002F0F7FB0022884B01F0CDFC03F04E
:107DA000C7F9050003F0FAF9794A7A4B0490059176
:107DB00002F0E8FB02000B003000390002F054FE34
:107DC000754A06000F0004980599744B02F0DAFB1F
:107DD000029003911F2D00DCC7E0029A039B300044
:107DE000390002F041FE83468A4653465B00241563
:107DF0005B0DE31A102B6CDD04980599D322674BB9
:107E0000520502F0BFFB02000B0030003900029265
:107E1000039302F029FE0A00010013000691079265
:107E200002003900300002F01FFE029A039B02F0AC
:107E30001BFE06000F0004980599614A614B02F091
:107E4000A1FB32003B0002F00FFE069E079F0B00D5
:107E50000200390030000292039302F005FE4B004D
:107E60005B0D83468A46E41A312C32DD049805996D
:107E7000B822544B920502F085FB03000C0002006F
:107E8000029303940B000698079902F0EDFD02009F
:107E90000B0006000F000698079902F0E5FD029A14
:107EA000039B02F0E1FD484A029003910498059972
:107EB000464B02F067FB029A039B02F0D5FD0200DD
:107EC0000B00300039000292039302F0CDFD83468F
:107ED0008A465A465346414630000A604B60390094
:107EE00002F0C2FD029A039B02F0BEFD44460B0065
:107EF0000200A260E3604B46002B00DB1BE75B4601
:107F0000236080231B065344636080231B069C462A
:107F10006144A060E1606D420DE70B00020002F0D9
:107F2000A3FD434600259860D9601860596002E7B8
:107F3000D3221A4B520502F097FD214A214B0D0026
:107F4000040002F091FD02000B00414620000A608F
:107F50004B60290002F088FD1A4B194A02F084FD9B
:107F6000434601259860D960E5E602000B00300029
:107F7000390002F079FD6B1E154A9B009B58834621
:107F80008A46A342A5D130E7FB21E93F7BD90240D5
:107F900000004054FB21F93F3163621A61B4D03DC7
:107FA000FB213941FFFFEF7FEAFBFFFF000070413B
:107FB000E8DE000083C8C96D305FE43F0000E03FA9
:107FC0007370032E8A19A33BC14920259A837B39FC
:107FD00068DE0000D3220C4B520501F0ADFB0B4ACA
:107FE0000B4B04000D0001F0A7FB02000B00414603
:107FF00020000A604B60290002F036FD034A044B62
:10800000B9E6032373E6C04661B4D03D7370032E16
:108010008A19A33BF8B54746CE46674B80B50A00A0
:108020000F00190005003940994200D19BE004007F
:108030000100002F69DD3F1500D1B4E05F4B120352
:108040009C468023120B5B0313435B00CA0F6744FB
:108050009B184A00F80703D5D20F5B009B188A00D3
:1080600079108C46002180201624894680030D1843
:108070009D4202DC29185B1B8144D50F5B00013C4B
:108080005B1952004008002CF1D10020804680206E
:1080900020250027000609E08B425CD0D40F5B004E
:1080A000013DE31852004008002D16D0C4198B4240
:1080B000F2DD27180E00002C49DB5B1AA242894131
:1080C00049425B1A121BD40F5B00013D8044310012
:1080D000E31852004008002DE8D113434ED1434627
:1080E0005B0837494A468846494652104244C90708
:1080F00002D5802109060B4361460F05BD18180003
:1081000029000CBC90469946F8BD7B005B080343F0
:108110003900002BF5D0002F3CD1E30A153A640555
:10812000002BFAD08020400303423FD1002700E01B
:108130000F005B00791C0342FAD0250020208D40FF
:10814000401A2900D71B2200C2401A4376E7FE439B
:10815000F60F8E19B1E79442A0D82718002CF6DB51
:108160001E000023AEE702003B002800390002F0A9
:1081700009FA2A003B0001F0DFFAC2E74346013367
:1081800003D0434601335B08ABE701239846002345
:10819000C144A6E73B00020002F066FC02000B00AF
:1081A00001F0E6FDADE713000022BBE70127210047
:1081B00020207F42C6E7C0460000F07F01FCFFFFA1
:1081C0000000E03FF0B54746CE4680B587B000924C
:1081D0000193754B4F00814688467F089F4263DCC0
:1081E00002F0A6FF002800D1D4E04A4643464846A4
:1081F000414602F0C7F904000D006C4A6C4B02F0D6
:10820000C1F96C4A6C4B01F097FA22002B0002F086
:10821000B9F96A4A6A4B02F027FC22002B0002F0EF
:10822000B1F9684A684B01F087FA22002B0002F08E
:10823000A9F9664A664B02F017FC22002B0002F0F7
:10824000A1F9644A644B01F077FA22002B0002F096
:1082500099F9029003910022604B2000290002F05E
:1082600091F9029A039B06000F002000290002F0FA
:1082700089F9009A019B04000D004846414602F02E
:1082800081F902000B002000290002F0EDFB020042
:108290000B003000390002F0E7FB02000B00002069
:1082A0004F4902F0E1FB70E002000B0002F06AF9B6
:1082B00004000D003D4A3E4B02F064F93D4A3E4B3E
:1082C00001F03AFA22002B0002F05CF93B4A3C4BE9
:1082D00002F0CAFB22002B0002F054F9394A3A4B53
:1082E00001F02AFA22002B0002F04CF9374A384BF1
:1082F00002F0BAFB22002B0002F044F9354A364B5B
:1083000001F01AFA2B00220002F03CF9354B0290E2
:1083100003919F429FDD344B00229F423DDC334955
:1083200000207B182E4916001F0002F09DFB0490D0
:1083300005910022294B2000290002F023F9320088
:108340003B0002F091FB029A039B06000F00200005
:10835000290002F017F9009A019B04000D0048461D
:10836000414602F00FF902000B002000290002F044
:108370007BFB02000B003000390002F075FB0200AD
:108380000B000498059902F06FFB07B00CBC9046F7
:108390009946F0BD00201249F7E7154B00260492DC
:1083A0000593144FC5E7C046FFFF3F3ED43888BE53
:1083B000E9FAA8BDC4B1B4BD9EEE213EAD529C8089
:1083C0004F7E923E9015CB19A001FA3E7751C1160F
:1083D0006CC1563F4C5555555555A53F0000E03FE3
:1083E0000000F03F3233D33F0000E93F0000E0FFE0
:1083F0000000E73F0000D23FF0B5DE464E4645465E
:108400005746E0B5DC4CA5440D9114001900A49A20
:108410000993DA4B9200D6584D1E03901821E01EA6
:108420000696029500F0AAFEC3430100DB1719402F
:108430004B1C9A009B1ADB001B190B9105934C1BDC
:10844000771918D4A59BA5009C463F1922AE654418
:10845000013707E0286802F0A1FE013403C60435A5
:10846000BC4208D0002CF5DA00200021013403C6FC
:108470000435BC42F6D1069B002B01DA00F0FDFB6F
:10848000069B03990133DB009A46099BDA00944668
:1084900000920022914672AA0492B94A614493461E
:1084A00088469AAB63449B44029B002B00DABCE1F4
:1084B0005D4600260027039C4D442A686B6803CC68
:1084C00002F060F802000B003000390001F034F9CE
:1084D000083D06000F004445EFD1049B4B441E604D
:1084E0005F6008239C46E144D145DDD10EA80421FC
:1084F0008446494261448C46069A93009C446146F6
:1085000084460A910399083B63448C460C93009B74
:10851000009263449B46009A0498D10003008C4665
:10852000634408911E685F68002A33DD95498046E0
:108530008C466244D300984470AB9A460EAB994681
:108540000022914B3000390002F01CF802F0F0FDDF
:1085500002F024FE00228D4B04000D0002F012F800
:1085600002000B003000390002F07EFA02F0E0FD5C
:108570004B4601C39946434620001A685B682900B0
:1085800001F0DAF808235B429C46E04406000F0045
:10859000D045D5D1059B30001A003900984600F02F
:1085A000DFFCFF2300229B0504000D0001F0EAFF21
:1085B00000F038FC0022764B01F0E4FF02000B00D3
:1085C0002000290002F050FA0D00040002F0B0FD76
:1085D000814602F0E3FD02000B002000290002F0BA
:1085E00043FA060040460F00002800DCEEE0009B46
:1085F00018215A1E92000EAB9B58091A1D000D41FE
:10860000A9448D405D1B0EAB9D5017231B1A1D41C5
:10861000002D2DDD01239C46009BE144002B00DC56
:108620001CE20E9C0123002C00D0B5E0009A012A28
:1086300009D099000EAA54580133002C00D0ACE0A8
:10864000009A9A42F5D1059B002B0EDD012B00D13B
:10865000A8E1022B09D1009B0EA95A1E92000EAB75
:108660009B5807939B029B0A8B50022D00D1C1E0BF
:10867000002300223000390000F08AFE009B002811
:1086800000D194E2069A591E8A4210DC414A0A98A7
:1086900094460EAA6344944600229B0063441C68DF
:1086A000043B22438342FAD1002A00D0C0E0069B5B
:1086B0000EAA013B9B00D358002B00D0B3E001224F
:1086C0000C9B043B596801320029FAD0009B9C4660
:1086D0006244110007921A0001338B4246DC0B986A
:1086E00063468046A59C4344A046099C9B00A14646
:1086F0004A449844D30022AA9146049A9944944645
:10870000089BA59A63448446614494469A468B002C
:10871000634400934346586802F040FD4B4618609E
:108720005960029B002B24DB4D46039C002600274A
:1087300001E0286869680CCC01F024FF02000B00FE
:108740003000390000F0F8FF083D06000F005C45DE
:10875000EFD153469E60DF6004239C460433E0441F
:108760009C46009BE144E2449845D3D1079B00938B
:10877000D1E600260027ECE794FDFFFF30E0000083
:1087800018FEFFFFFFFFFF1F0000703E000070415A
:1087900000002040FFFFFF3F002180225204141BF5
:1087A0000EAA5450009999420EDD0EA884469B00F3
:1087B0000EAA8900D25861446344CF4800E01A6889
:1087C000821A04C38B42FAD101243CE7059B002B9B
:1087D00006D1009B0EAA013B9B00D558ED1517E76B
:1087E0000022C64B300000F0F7FD002800D024E145
:1087F00000253DE732003B000020C14902F034F97A
:1088000006000F00002C00D132E7059A0020BC4979
:1088100000F0A6FB02000B003000390002F024F942
:1088200006000F0024E7012250E70026002754E647
:108830004B46059A079388468B000EA9CB58183AE9
:1088400008950592002B0DD18C464146AD4B434413
:108850009B006344043B58680139183A0028F9D05A
:1088600088460592059A0020A54900F079FB434609
:1088700004000D00002B00DA05E29E000EAB9C46C2
:108880004346DB0066449C46059370AB9946049FC3
:1088900067440097306802F081FC22002B0001F051
:1088A00071FE002238607960974B2000290001F0AA
:1088B00069FE083F04000D00043EB945EAD14AAB09
:1088C00003939B4600239A46069B4246994643469D
:1088D0000132029204934B46002B00DAAAE080207A
:1088E0008A4B009D9846C005894900260027002430
:1088F00008E008239C460835E044544511DC434613
:10890000186859682A686B6801F03CFE02000B0089
:108910003000390000F010FF013406000F00A145BF
:10892000E7DA5B46C0C39B4601239C46009BE244BA
:10893000083B0093029B9A45CDD1049B9846A49B8B
:10894000022B00DD8EE0002B37DC1FD1059B0027BA
:108950001D00039B00249C461E006544083E2A68B7
:108960006B683800210000F0E7FE083D07000C00AE
:10897000AE42F4D1089B002B03D080231B069C46FB
:1089800064443A0023000D990A604B600720079B5E
:1089900018409B239B009D443CBC90469946A246B0
:1089A000AB46F0BD009B0EA95A1E92000EAB9B5821
:1089B00007935B025B0A8B5057E64346002B00DAB5
:1089C00070E100200021DB004AAAD61848AF3268C7
:1089D0007368083E00F0B0FEB742F8D1089B002B48
:1089E00000D025E10B0002004A984B990D9C2260B3
:1089F000636002F039F8434607000C00002B13DDDA
:108A000001254CAEB14638002E0021004C460136FF
:108A10000CCC00F091FEA146B045F7DA089B0700A8
:108A20000C00002B00D015E13A0023000D998A605C
:108A3000CB60ABE70026002773E701239C46009B31
:108A4000E1440225002B00DDEBE532003B00002075
:108A50002B4902F009F806000F0009E60024F2E5B0
:108A60004AAB0393A49B032B00D08FE74346002B14
:108A700000DC14E1039ADB009B46130091465B4443
:108A80001E685F68234B43440293DB00994448AB64
:108A90009A464B465C681B681800210032003B0078
:108AA0000090019100F048FE04000D0002000B0050
:108AB0000098019901F0D8FF3B00320000F03CFE25
:108AC0004B469860D9601C605D6008235B429C4601
:108AD000E14426002F00CA45DBD14346012B00DCD0
:108AE000E3E0039A13005B441E685F68029BDB00AF
:108AF00099464A44904610E0FFFFFF000000E03F27
:108B00000000F03FFFFFFF3F0000703EF0DF00007D
:108B1000FB21F93FFFFFFF1F984643465C681B6837
:108B20001800210032003B000090019100F004FE8B
:108B300004000D0002000B000098019901F094FF61
:108B400032003B0000F0F8FD4346039A9860D9607C
:108B50001C605D60083B26002F009A42DCD14D4628
:108B60009446002600244746083565442A686B6809
:108B70003000210000F0E0FD083D06000C00AF428F
:108B8000F4D1039B4A9F5D689968D868089B002BC5
:108B900065D08022120694460D9B6544604464446F
:108BA0001F605D609960D8601E615C61EEE69A4668
:108BB0004B460793059B30005A423900089500F058
:108BC000CFF900223A4B06000F0000F005FC002808
:108BD00024D0384B00223000390001F0D3FC02F0E1
:108BE000A7FA52460400950002F0D8FA0022304B52
:108BF00001F0C8FC02000B003000390001F034FF26
:108C000002F096FA0EAA50510122059B52441833E5
:108C10009046059393000EAAD45023E653463000A5
:108C200039009C0002F084FA0EAB1851D04619E6C8
:108C300080230D9A1B06CB18106053600B000200B6
:108C40004A984B9901F010FF434607000C00002B97
:108C500000DDD5E680231B069C466444E4E62B0039
:108C60003A000D9D2A606B600A000300AA60EB6069
:108C7000320023002A616B6188E6099BDB000093C8
:108C800072AB049332E4A49B022B00DDE8E6002BD8
:108C900000DD92E600D079E6002700246AE600268F
:108CA00000246EE70020002198E60026340068E7E3
:108CB000000070410000703EF0B5CE46474680B5DA
:108CC00087B000920193474A4B00814688465B0873
:108CD000934207DC4146484602F02AFA4146031E09
:108CE000484666D04A4643464846414601F04AFC5B
:108CF00004000D0002000B004846414601F042FC12
:108D0000394A3A4B06000F002000290001F03AFCD6
:108D1000374A384B01F0A8FE22002B0001F032FC4C
:108D2000354A364B00F008FD22002B0001F02AFCEA
:108D3000334A344B01F098FE22002B0001F022FC54
:108D4000314B324A00F0F8FC0E9B02900391002B4D
:108D500034D00098019900222D4B01F013FC029AA7
:108D6000039B049005913000390001F00BFC0200D8
:108D70000B000498059901F077FE22002B0001F00A
:108D800001FC009A019B01F06FFE224A04000D00D5
:108D9000214B3000390001F0F5FB02000B002000F0
:108DA000290000F0C9FC02000B004846414601F0D2
:108DB0005BFE07B00CBC90469946F0BD02000B006C
:108DC0002000290001F0DEFB124A134B01F04CFE9B
:108DD00032003B0001F0D6FB4A46434600F0ACFCB3
:108DE000E7E7C046FFFF3F3E7CD5CF5A3AD9E53D85
:108DF000EB9C2B8AE6E55A3E7DFEB157E31DC73E4C
:108E0000D561C119A0012A3F1111813FA6F81011A7
:108E10000000E03F495555555555C53F49004B08A1
:108E200019007047474AF0B54F4691464B005B0D1D
:108E300099444646D6464A46C0B505000C000E0089
:108E400088460700132A27DC002A4BDB3E4B1341E0
:108E50009A460B0052461340034318D03B4A3C4B02
:108E60002800210000F068FC0022002300F0AAFA8C
:108E7000002847D0002C04DA80234A465B031341C4
:108E800098444646534600279E43380031001CBC98
:108E900090469946A246F0BD332A08DD8023DB00C8
:108EA0009945F4D102000B0000F046FCEFE7294A97
:108EB0009446012263445242DA4092460242E6D08E
:108EC000224A234B2800210000F036FC0022002318
:108ED00000F078FA002815D0002C1EDB53464646D9
:108EE0009F430FE0194A1A4B2800210000F024FC90
:108EF0000022002300F066FA002803D0002C04DBD7
:108F00000027002638003100C1E7640064082543CB
:108F10000027002DF6D0104EF4E74B46142B0BD053
:108F20003422D21A012393405D19BD4208D2012395
:108F30009C462F00E044D1E7133B9C46E044CDE73C
:108F40002F00CBE701FCFFFFFFFF0F009C7500889F
:108F50003CE4377EEDFBFFFF0000F0BF00207047D0
:108F60004B0070B55B0D14000A00002B1AD14B00AA
:108F70005B08034315D0234B002201F003FB224B77
:108F80009C422DDB0A004B005B0D363B1F4DE31866
:108F9000AB422ADC002B0DDD1D4C1B0522401A4381
:108FA000110070BD1B4DAB42F0D102000B0000F070
:108FB000C3FBF6E71D00353519DA174B02009C425A
:108FC00009DD0B001548164900F032F8134A144B1E
:108FD00001F0D8FAE5E70B001248134900F028F831
:108FE000104A114B01F0CEFADBE70200E9E7084C2A
:108FF000363322401B051343190000220B4B01F0AE
:10900000C1FACEE700005043B03CFFFFFE0700006E
:10901000FFFF0F80FF07000050C300009C75008811
:109020003CE4377E59F3F8C21F6EA5010000903C66
:1090300030B54A00DB0FDB0752081A43110030BD80
:1090400002B4714649084900095C49008E4402BCDB
:109050007047C04603B47146490840004900095AA8
:1090600049008E4403BC7047002243088B4274D3EE
:1090700003098B425FD3030A8B4244D3030B8B4219
:1090800028D3030C8B420DD3FF22090212BA030C22
:109090008B4202D31212090265D0030B8B4219D303
:1090A00000E0090AC30B8B4201D3CB03C01A524123
:1090B000830B8B4201D38B03C01A5241430B8B426B
:1090C00001D34B03C01A5241030B8B4201D30B0354
:1090D000C01A5241C30A8B4201D3CB02C01A52417B
:1090E000830A8B4201D38B02C01A5241430A8B423E
:1090F00001D34B02C01A5241030A8B4201D30B0227
:10910000C01A5241CDD2C3098B4201D3CB01C01A40
:10911000524183098B4201D38B01C01A524143094A
:109120008B4201D34B01C01A524103098B4201D338
:109130000B01C01A5241C3088B4201D3CB00C01AA5
:10914000524183088B4201D38B00C01A524143081D
:109150008B4201D34B00C01A5241411A00D2014642
:10916000524110467047FFE701B5002000F0F0F8CB
:1091700002BDC0460029F7D076E7704703460B438F
:109180007FD4002243088B4274D303098B425FD300
:10919000030A8B4244D3030B8B4228D3030C8B422C
:1091A0000DD3FF22090212BA030C8B4202D3121212
:1091B000090265D0030B8B4219D300E0090AC30BE7
:1091C0008B4201D3CB03C01A5241830B8B4201D394
:1091D0008B03C01A5241430B8B4201D34B03C01A7D
:1091E0005241030B8B4201D30B03C01A5241C30AF5
:1091F0008B4201D3CB02C01A5241830A8B4201D366
:109200008B02C01A5241430A8B4201D34B02C01A4F
:109210005241030A8B4201D30B02C01A5241CDD2F4
:10922000C3098B4201D3CB01C01A524183098B423F
:1092300001D38B01C01A524143098B4201D34B0128
:10924000C01A524103098B4201D30B01C01A52418B
:10925000C3088B4201D3CB00C01A524183088B4212
:1092600001D38B00C01A524143088B4201D34B00FB
:10927000C01A5241411A00D201465241104670476D
:109280005DE0CA0F00D04942031000D34042534072
:1092900000229C4603098B422DD3030A8B4212D332
:1092A000FC22890112BA030A8B420CD38901921164
:1092B0008B4208D3890192118B4204D389013AD0A1
:1092C000921100E08909C3098B4201D3CB01C01A76
:1092D000524183098B4201D38B01C01A5241430989
:1092E0008B4201D34B01C01A524103098B4201D377
:1092F0000B01C01A5241C3088B4201D3CB00C01AE4
:10930000524183088B4201D38B00C01A5241D9D2FB
:1093100043088B4201D34B00C01A5241411A00D27C
:109320000146634652415B10104601D34042002B78
:1093300000D54942704763465B1000D3404201B5F7
:10934000002000F005F802BD0029F8D016E77047AC
:109350007047C046D0400B1C1141203A03D49C46B4
:109360001341184363465242934018437047C04626
:109370008446101C62468C46191C634600E0C046B9
:109380001FB501F097F8002801D40021C8421FBD85
:1093900010B500F0EFFF4042013010BD10B501F0F4
:1093A00089F8002801DB002010BD012010BDC04657
:1093B00010B501F07FF8002801DD002010BD01206C
:1093C00010BDC04610B501F011F8002801DC0020E6
:1093D00010BD012010BDC04610B501F007F80028EF
:1093E00001DA002010BD012010BDC046F0B5CE4608
:1093F000474615042D0C2E0080B50704140C3F0CB5
:109400009946030C7E435D43674363437F19340CE5
:10941000E4199C46A54203D980235B029846C444C4
:109420004B4643435143250C36046544360C240413
:10943000A4195B19591820000CBC90469946F0BD40
:10944000F0B54E4657464546DE46E0B543025B0A58
:10945000450083B00F1C99462D0EC60F002D57D026
:10946000FF2D24D08020DB00C00418430023814658
:109470009A469B467F3D7C027A00FB0F640A120EDF
:10948000984623D0FF2A4BD0E30080240020E40438
:109490007F3A1C43AD186B1C4746019353467740F7
:1094A0003A000F2B48D87D499B00CB589F46002B94
:1094B00000D085E008339A46063B9B467C027A0042
:1094C000FB0FFF25640A120E9846DBD1002C00D05A
:1094D00090E0524601231A4392460120DBE74C46B6
:1094E00058461700022824D0032800D1CFE00022DC
:1094F000002301284DD15802D205400AFF0710432E
:10950000384303B03CBC90469946A246AB46F0BDFA
:10951000002B5BD104239A46033B00259B46AAE718
:10952000FF35002C60D1524602231A439246022096
:10953000B1E7FF220023DEE74B461B0C9C464B465F
:109540002604360C180461463300220C6446000CD5
:1095500043434E435043544380191A0C1218964209
:1095600003D9802149028C4664441B041B0C10045F
:10957000C01883015E1EB341800E1843130C1B19E3
:109580009B0103431C00230179D5012362081C4081
:109590001443019A7F32002A4DDD630704D00F2364
:1095A0002340042B00D00434230103D53C4B019A03
:1095B0001C408032FE2ABCDCA3015B0AD2B29AE7CF
:1095C0000C239A46093BFF259B4654E7180001F0FF
:1095D00071FE4A46431F76259A4000236D4291460C
:1095E0002D1A9A469B4646E7524603231A43924653
:1095F000032050E7200001F05DFE431F2D1A9C4020
:10960000763D002047E780230027DB03FF2272E737
:10961000424666E74C463200584662E780234A4697
:10962000DB031A4222D01C4220D123435B025B0A97
:109630004746FF225FE701239A1A1B2A21DC2300F9
:109640000199D3409E318C401A0023005C1EA34137
:1096500013435A0704D00F221A40042A00D00433BF
:109660005A0111D49B015B0A002244E780234A4639
:10967000DB0313435B025B0A3700FF223BE70195E4
:1096800087E70022002336E70122002333E7802307
:10969000DB0323435B025B0AFF222CE740E0000070
:1096A000FFFFFFF770B500283DD0C317C5185D4018
:1096B000C40F280001F0FEFD9E22121A962A07DC34
:1096C000D2B2082833DD083885406802400A23E01A
:1096D000992A0BDD052329001B1AD94003001B33EF
:1096E0009D402B005D1EAB4119430D00052801DD97
:1096F000431F9D402B000F490B406E0709D00F26DA
:109700003540042D05D004335D0102D59F220B4066
:10971000121A9B01580AD2B24002D205400AE4074D
:109720001043204370BD002400220020F4E76802AB
:10973000400AF1E7FFFFFFFBF0B54F464646D6462D
:109740000C000903C0B5490A470F5E0039431F03E7
:10975000DB0F9C4665007B0A570F1F436D0DE40F1E
:10976000760DA146C000B846D200AB1B64457BD045
:10977000002B5FDD002E00D0A4E03E00164300D198
:1097800012E15E1E002E00D09EE1871A4346B842C9
:1097900080410125C91A4042091A0B0200D431E167
:1097A00049024E0A002E00D16EE1300001F082FD28
:1097B0000300083B1F2B00DD61E120223900D21A93
:1097C0009E40D1409F400E439D4200DD51E15D1B14
:1097D0006B1C1F2B00DD7CE12021C91A3D003000ED
:1097E0008F408840DD40791E8F4131000722284399
:1097F000D940002507433A40002A09D00F233B40B7
:10980000042B05D03B1DBB42BF417F42C9191F003D
:109810000B0200D426E26A1CC64B55056D0D9A4218
:1098200000D106E1C44AFF080A40530752023B43F5
:10983000120B8EE0002B00D0B8E06B1C5B055B0DBB
:10984000012B00DC30E1871A4346B842B641CB1AFF
:1098500076429E1B330200D54CE13B003343A1D13D
:1098600000220024002570E0002B00DCE5E0002E43
:1098700000D183E0AF4EB54260D080263604374336
:10988000B846382B00DC3EE1434613431F007A1EE6
:1098900097413F1887428041404209180B0200D48B
:1098A000B0E0A44B01359D4200D1C3E0A24A7B0841
:1098B0000A4001210F401F435108D30707221F43CD
:1098C0003A4099E79B4EB54238D08026360437435C
:1098D000B846382B00DDDCE01F2B00DC30E11E0039
:1098E0004746203EF740BC46202B04D04026F31AC2
:1098F00046469E403243170063467A1E97411F43F7
:10990000CCE0002B00D104E24346134300D159E1DF
:109910004B07C00818438023C9081B03194208D00D
:109920004546ED081D4204D14346D0085907084377
:109930002900420FC9007F4D1143C0004B07CA08E0
:109940007C49C00803438D4268D012036D05120B99
:109950006D0D002112031800130B0A0D12051A4396
:10996000764B2D0513402B435B00E4075B08234334
:1099700019001CBC90469946A246F0BD3E00164315
:1099800012D05E1E002E00D000E187188742804171
:1099900041444042091801250B0233D5022585E7D1
:1099A00064463300414610001D00C7E7002D00D07B
:1099B000DAE00C000443F3D05C1C00D19FE15D4C65
:1099C000A64200D12FE1DB43382B00DD66E11F2BDF
:1099D00000DD83E120240500E41A0F00DD40D940BA
:1099E000A0404346A7405B1A441EA04198462F431F
:1099F0003843171ABA42924143465242991A644672
:109A00003500CAE607223A40002A00D0F6E64B07A6
:109A1000CA084849FF083B438D4296D119001143BB
:109A200000D19EE1802109030A431203120B414D2C
:109A30008FE71500002200238BE7002B00D0C7E042
:109A40006B1C5F057F0D012F00DCF1E0394DAB424F
:109A500000D1B9E085180A00854289414244494253
:109A600051180722CF076D082F4349083A401D00BF
:109A7000C2E607223049ED1A31403A40BCE63E00CA
:109A80002838864000279FE6380001F013FC20307C
:109A90008EE6434613431F007A1E9741C71BB84208
:109AA00080414042091A78E60E003B00064313430A
:109AB000002D61D1002E00D0F4E0002B00D11BE17D
:109AC00064463900100039E71A4FBB427AD03300A0
:109AD000FFE630001F3DE840202B03D04021CB1A89
:109AE0009E4037437B1E9F41072207433A40002197
:109AF000002589E7171A4346BA42B641591A7642F9
:109B00008E1B64464EE61F2B00DDADE02026474647
:109B1000F61AB740B9461700B246DF404E463E43FC
:109B200037005646B240561EB24117434246DA400D
:109B30008918AEE6FF070000FFFF7FFFFFFF0F80E1
:109B400020264746F61AB740B9461700B246DF400E
:109B50004E463E4337005646B240561EB24117436A
:109B60004246DA40891A99E77F4CA6425BD08024AE
:109B700024045B42214327E7002E0CD1002B00D1A7
:109B8000CBE0644639001000774DD7E6764FBB42F4
:109B900018D0330075E6002B14D04B07C0081843CB
:109BA0008023C9081B03194207D0FC081C4204D1BA
:109BB0007907D0080843E14621004C46420FC9000E
:109BC0001143C000684DB9E61D0000220023C0E625
:109BD000002D5BD10D00054300D1E2E65D1C00D1F4
:109BE000B0E0614DAE421FD0DB43382B71DC1F2B40
:109BF00000DD96E020250F00ED1AAF40B9460700C2
:109C0000AA46DF404D463D432F005546A840D94067
:109C1000451EA84188440743BF18974292415142CC
:109C2000414435003AE6644635004146100085E679
:109C30000B000343002D00D063E6002BF5D0434614
:109C4000134300D17AE687188742804107224144B6
:109C5000404209183A400B0200D4D5E6434B013587
:109C60001940C9E5380069E61E004746203EF74026
:109C7000BC46202B04D04026F31A46469E40324371
:109C8000170063467A1E97411F4302E6364DAE42E7
:109C9000CAD080252D045B422943A6E70843411E14
:109CA0008841A6E6002B00D148E6871A4346B84211
:109CB000B641CB1A76429E1B33024BD5171A434648
:109CC000BA429241591A5242891A072264463A40CE
:109CD00092E501430F00791E8F419DE71C000F00A4
:109CE000203CE740202B03D04024E31A994008434E
:109CF000411E884138437CE60022002425E6171ADD
:109D00004346BA429241591A5242891A6446350072
:109D100043E541461000144D10E680220024120352
:109D200080E61D000F00203DEF40BC46202B03D0F5
:109D30004025EB1A9940084307006346781E874187
:109D40001F4369E7871897429B4141445B42C9180A
:109D50003500A3E53B003343CED0072231003A4023
:109D600052E600231A00F4E5FF070000FFFF7FFF23
:109D7000F0B55746DE464E464546E0B583460700F9
:109D80000E03480085B092461C00360B400DCD0FE7
:109D9000002800D19DE0954B984239D08023F600F1
:109DA0001B041E43924A7B0F33439946944603009B
:109DB0006344009300230026FF00029323031B0B40
:109DC00098466300E40F52465B0D019400D1B3E066
:109DD00086498B4200D19EE04246D1008022120487
:109DE0000A435146490F11438B46814952468C46DE
:109DF00000996344CB1A0021D20000932B006340EA
:109E00009A460F2E00D905E17A4BB6009B599F4622
:109E10005B463343994600D0B8E00223082600276A
:109E200000900293CAE7CB463A0002990195019B44
:109E30009A46022927D0032900D180E2012944D083
:109E40006D49009B8C4663441C00002C38DD530791
:109E500000D013E2D2085B46DB0109D55946674BB7
:109E600019408B468021C9008C46009B63441C002E
:109E7000634B9C4207DC5B4664055F075B0217434C
:109E80001B0B620D02E000230027584A00211B0330
:109E90001C0B0B0D1B05234314055A4A38001340B5
:109EA0001C4353466400DB0764081C43210005B0D3
:109EB0003CBC90469946A246AB46F0BD01225242B8
:109EC00001231B1B382B00DCADE1002200230027FF
:109ED000DCE75B46334399465ED0002E00D18AE131
:109EE000300001F0E7F903000B3B1C2B00DD7BE1A8
:109EF0001D22D31A5A460100DA4008398E40130059
:109F00005F46334399468F403F4B00261B1A009310
:109F10000023029352E7414653460B433B499B467D
:109F20008C46009B634400935B46002B3BD102238D
:109F300000221E43022161E7434613439B4637D06C
:109F40004346002B00D162E1404601F0B3F9030023
:109F50000B3B1C2B00DD53E102004146083A9140C7
:109F600088461D21CB1A5146D9400B0041460B4370
:109F70009B46534693401A00009B25499C466044EB
:109F800003008C4663440093002137E70323B14666
:109F900000900C26029311E700230093013304265E
:109FA000002702930AE70323C3461E43032125E744
:109FB00001331E430022012120E700239A4680231B
:109FC00000271B03094A61E7802349461B03194206
:109FD00000D1E2E05946194200D0DEE00B431B03FA
:109FE00017001B0BA246014A50E7C046FF070000BE
:109FF00001FCFFFF80E00000FF030000FFFFFFFE09
:10A00000FE070000FFFF0F800DFCFFFF01F8FFFFC0
:10A01000F3030000D94500D9CBE000D1C6E03C00F5
:10A0200048460027009B013B00935B46160E1B022F
:10A030001E431302984633041B0C9946310C0191C0
:10A04000FFF798F84A4642430B04210C05001943D8
:10A050008A4207D98919013D8E4203D88A4201D923
:10A06000851E8919881A0199FFF784F809048C461E
:10A070004A46210464464243090C030021438A42B4
:10A0800004D98919013B8E4200D8F1E02D041D430B
:10A09000AB464346891A4246280C12041D0C5B4607
:10A0A000140C22001B041B0C5A4303946B434443BF
:10A0B000029568431B19150CEB189C4203D98024A8
:10A0C0006402A44660441C0C15041B042D0C2018CB
:10A0D0005D19814277D373D00C1AA24A7D1BAF421F
:10A0E000BF419446009B7F426344E01B1C008642B4
:10A0F00000D1DBE00199FFF73DF84A4642430B04EB
:10A10000290C070019438A4207D98919013F8E4259
:10A1100003D88A4201D9871E8919881A0199FFF745
:10A1200029F809044A46894629044D464243090C48
:10A13000030029438A4207D98919013B8E4203D87B
:10A140008A4201D9831E89193F04891A3A00039F64
:10A150001A43380013041B0C584381460298150C0F
:10A160006F43434345434846000C8446DB19634430
:10A170009F4203D9802040028446654448461F0C14
:10A1800000041B04000C7D191818A94200D284E0B9
:10A1900000D17FE001231A4357E680234A461B0380
:10A1A00013431B031B0BAA466F4A6FE6BA4200D942
:10A1B00035E74B46DC0758087B081C43FF0734E7AC
:10A1C0000024AF4289D247444745A4415B466442DC
:10A1D000A4196418013BA6421ED2A0426DD800D13A
:10A1E000B6E0241A9B4678E703005A46283B9A407B
:10A1F0000027914688E6584601F05CF8203072E668
:10A2000003005246283B9A4093460022B4E650464B
:10A2100001F050F820309AE6A642E2D1B845DCD9E8
:10A22000341A9B4659E71F2B65DC504C0099A44615
:10A230005C46614408008C4011008240D940501EA9
:10A2400082410C4314435A46DA401300620709D096
:10A250000F222240042A05D02200141D9442894175
:10A2600049425B181A0262D50122002300270DE63D
:10A270008A4200D80AE7831E891907E70F23134093
:10A28000042B00D1E6E5171D9742924153429B44AF
:10A29000FA08E0E5002800D1D7E57118531EB14255
:10A2A00027D3A94215D358D01A0073E7002B00DC3E
:10A2B00004E6012300229B44CDE5022347444745A1
:10A2C00089415B429C46494289190C19E344241A8E
:10A2D00003E743465F0047459B41B8465B429E19F2
:10A2E000023A8919A94200D054E7404500D051E70D
:10A2F000ABE51A00F6E71F215F4649420C1BE74019
:10A30000202B07D01A49009B8C46634418005B46FB
:10A3100083401A43501E82413A43072700231740C7
:10A3200009D00F21002311401400042995D12200E7
:10A330005F075B021B0BD20817430022A6E58023B0
:10A3400059461B030B431B0317001B0B064A9DE5D5
:10A35000BD42B2D89B460024BFE68045B9D31A005F
:10A36000C3E7C046FF030000FF0700001E04000013
:10A370003E040000F0B54F464646D6468446C0B57A
:10A380008046194E18030F034D00000B5C008246F7
:10A390003F0B6D0DC90F9146640DDB0F0120B542D7
:10A3A0000AD0B44203D0A54201D157450CD01CBC01
:10A3B00090469946A246F0BD66463E43F7D1AC4270
:10A3C000F5D154461443F2D10120C845EFD199424A
:10A3D00007D0002DEBD163461F433800471EB8411C
:10A3E000E5E70020E3E7C046FF070000F0B54F4671
:10A3F0004646D6464D00C0B50E03C90F8A462C49C5
:10A400001F035C008046360B6D0D91463F0B640DBB
:10A41000DB0F8D421ED08C4216D0002D1ED1304352
:10A420008446002C01D13A4323D06246002A1AD038
:10A430009A4529D0514602200139084001381CBCF8
:10A4400090469946A246F0BD39001143E5D002205E
:10A450004042F4E73043FAD1AC420FD0002C0FD188
:10A460003A43E7D00CE00122013B9343180001304E
:10A47000E5E763460020002BE1D0DBE73A43E6D175
:10A480009A45D7D1A542D5DCA54205DBBE42D1D83D
:10A4900008D00020BE42D2D2504601230138984352
:10A4A0000130CCE7C845C5D80020C845F4D3C6E77D
:10A4B000FF070000F0B54F464646D6464D00C0B5F2
:10A4C0000E03C90F8A462E491F035C008046360BD7
:10A4D0006D0D91463F0B640DDB0F8D4218D08C4201
:10A4E00011D0002D18D130438446002C1ED13A43A0
:10A4F0001CD163460020002B30D051460220013988
:10A50000084001382AE039001143EAD0022025E052
:10A510003043FBD1AC4226D0002C26D13A4324D183
:10A520005146022001390840013817E06246002AEE
:10A530000FD09A45E1D1A54205DBBE42DDD819D046
:10A540000020BE420AD25046012301389843013010
:10A5500004E00122013B9343180001301CBC9046EB
:10A560009946A246F0BD3A43D0D19A45C5D1A542FD
:10A57000C3DCE0E7C845C0D80020C845E3D3EDE719
:10A58000FF070000F0B55746DE464E464546E0B5AB
:10A59000834606000F03480087B092461D003F0B1C
:10A5A000400DCC0F002800D16FE0DE4B984238D030
:10A5B0008023FF001B041F43730F3B430193DA4BBF
:10A5C0000027994600239B46F60081442B0369002F
:10A5D0001B0B52469846490DED0F002900D185E02E
:10A5E000D04B994200D173E04346DA0080231B042C
:10A5F00013435246CC48520F844613435246002020
:10A600006144D20089442100694000918C460121B7
:10A6100049448A460F2F00D990E0C449BF00CF5962
:10A62000BF465B463B43019300D06AE10223082703
:10A63000002681469B46C9E732005846019B614689
:10A640000091022800D175E0032800D1FEE1012825
:10A6500000D02CE100230027002600253F032A0D0F
:10A660003F0BB34812053A4302401B051343009ABF
:10A670005B00D1075B080B433000190007B03CBCFE
:10A6800090469946A246AB46F0BD5B463B430193DC
:10A6900000D12FE1002F00D1A5E1380000F00AFE23
:10A6A00003000B3B1C2B00DD96E11D22D31A5A46FA
:10A6B0000100DA405E4608398F4013008E403B436C
:10A6C00001939C4B00271B1A994600239B467DE76C
:10A6D000414653460B4393498C46E144002B00D03E
:10A6E0001AE102220220174300228CE7134300D113
:10A6F0000DE14346002B00D181E1404600F0DAFD38
:10A7000002000B3A1C2A00DD72E1010043460839C1
:10A710008B4098461D239A1A5346D3401A0043464D
:10A72000134352468A404946081A82498946814461
:10A73000002068E77B4B002700268EE7140C1204EC
:10A74000120C1100370C3604350C794328008C4666
:10A750002E0060436044834656432100300C8046FF
:10A760005846794340440291844506D98846802161
:10A7700049028C46E044414602913604010C360CF5
:10A7800000048B4681191E0C1B041B0C039119003D
:10A7900079438C46280075436544A8465843050C08
:10A7A00045447743A94203D9802149028C46674436
:10A7B000290C8C4639000004000C2D042D1861442E
:10A7C000AB4405915946049101990F043F0C080CC4
:10A7D000390051434243904602008C46090C8B4697
:10A7E00062437C4344445C44A04503D98021490230
:10A7F00088464244210C884661460904090C8C466F
:10A8000039005943434370437E430F0CF618240428
:10A81000BE19644442448C46B34203D980235B0290
:10A8200098464044029B61469846049B3704434443
:10A830009B46AB45AD416B420D0405992D0C8C46F2
:10A840007F196744FD18A8465D462D19A542A4410D
:10A8500093466442A446C344DC448F42BF419845BA
:10A860009B4193459241A445A4415B427F421F43D3
:10A87000360C52426442BF192243BF186246381850
:10A880004302D20D039913436A020A43501E8241C8
:10A890006146ED0D2A434E023243D90100D4B3E0A4
:10A8A0000126500832400243DE0732435B08224C47
:10A8B0005444002C62DD510709D00F2010400428B9
:10A8C00005D0101D9042924152429B180200D901BE
:10A8D00004D580241948E4000340544418488442B5
:10A8E00000DD27E75E075B02D2081F0B63051643F6
:10A8F0005B0DB2E6002399460133042700269B46F0
:10A9000064E60323019781460C279B465EE60122FD
:10A9100001201743002276E6032303201F4343460A
:10A9200071E6C046FF07000001FCFFFFC0E0000029
:10A93000FFFF0F800DFCFFFFFF030000FFFFFFFE86
:10A94000FE0700000023802700933F030026434BAF
:10A9500083E6019B3200A446584670E6AC466EE69C
:10A96000802701993F0339422DD03B422BD11F4311
:10A970003F033F0B00951600384B6EE601252D1B5B
:10A98000382D00DD66E61F2D40DC35481C005044A4
:10A99000160082408440EE40501E824134431443EE
:10A9A000EB40620709D00F222240042A05D0220082
:10A9B000141D9442804140421B181A023ED50123C7
:10A9C0000027002649E68027019B3F031F433F03E2
:10A9D0003F0B0094214B40E603005A46283B9A4027
:10A9E000002601926DE6584600F064FC203057E6E0
:10A9F00003005246283B9A401300002293E650463B
:10AA000000F058FC20307BE6CA4650E71F201E00AD
:10AA10004042041BE640202D03D0124C5444A34076
:10AA20001A43501E8241324307260027164009D0A0
:10AA30000F200023104014000428B9D122005E0723
:10AA40005B021F0BD2081643002306E680273F0354
:10AA50001F433F033F0B1600004BFEE5FF070000BE
:10AA60001E0400003E040000F8B557464E46454619
:10AA7000DE460C000903E0B5490A460F5F0031438A
:10AA80001E03DB0F760A9B46530F3343C84E650007
:10AA9000C000E40FD2006D0DA24681467F0D9C469A
:10AAA0009046B74200D1B9E05B46012673409B4611
:10AAB000EE1BA34500D183E0002E63DD002F00D004
:10AAC000B1E06346134300D123E1731E002B00D095
:10AAD000BAE1861A6346B04280410125C91A404254
:10AAE000091A0B0200D447E149024B0A9846434633
:10AAF000002B00D189E1404600F0DCFB0300083B5D
:10AB00001F2B00DD7CE120223000D21A4146D040CC
:10AB1000994002009E400A439D4200DD6AE15D1BB0
:10AB20006B1C1F2B00DD94E1202110003500C91A99
:10AB30008E40DA408840DD40711E8E4111000722B0
:10AB40002843002506433240002A09D00F23334012
:10AB5000042B05D0331DB342B641764289191E003D
:10AB60000B0200D43DE26A1C914B55056D0D9A42D3
:10AB700000D119E18F4AF6080A40570752023743BD
:10AB8000120B9BE0002E00D0C5E06E1C7605760D02
:10AB9000012E00DC48E16746861ACB1BB042BF415C
:10ABA0007F42B8461F004346FF1A3B00B8461B02CF
:10ABB00000D55FE137439AD100220024002579E0D7
:10ABC000002E00DCFAE0002F00D18DE0784B9D4292
:10ABD00067D0802367461B041F43BC46382E00DC29
:10ABE00052E1634613435A1E93411E188642804128
:10ABF000404209180B0200D4BEE06D4B01359D4266
:10AC000000D1D2E06B4A73080A4001210E401E4376
:10AC10005108D30707221E43324095E71E00164312
:10AC200000D045E740E7624B9D423AD0802367461B
:10AC30001B041F43BC46382E00DDEBE01F2E00DC5A
:10AC40003AE133006746203BDF403B00202E05D031
:10AC50004027BF1B6646BE40324390464646721EA2
:10AC600096413343DAE0002B00D114E263461343EC
:10AC700000D168E180234E07C008C9081B030643C2
:10AC8000194208D06046C008184204D1634601004A
:10AC9000D2085E071643F3009946C900720F444D6F
:10ACA00011434B46DE08424B4F073743CA089D42CB
:10ACB00000D16EE012036D05120B6D0D0021120321
:10ACC000130B0A0D12051A433B4B2D0513402B4362
:10ACD0005B00E4075B082343380019003CBC904646
:10ACE0009946A246AB46F8BD6346134311D0731E86
:10ACF000002B00D007E18618864280416144404223
:10AD0000091801250B0237D502257BE73E00614675
:10AD100091463500C5E75C46002D00D0E1E00B0010
:10AD20000343F3D0731C00D1ACE1214B9F4200D10F
:10AD30003AE1F343382B00DD6FE11F2B00DD8CE19E
:10AD400020250E00ED1AAE40B0460600AA46DE40B1
:10AD5000454635432E005546D940A8406346451E1A
:10AD6000A8415B1A9C463043161AB2429241634690
:10AD70005242991A3D00B4E607223240002A00D020
:10AD8000E4E60B4BF6084F073743CA089D4200D054
:10AD900090E73B00134300D1A6E180231B031A4335
:10ADA0001203120B024D89E715000022002785E7E8
:10ADB000FF070000FFFF7FFFFFFF0F80002E00D086
:10ADC000C7E06B1C5E05760D012E00DCF0E0C84D7F
:10ADD000AB4200D1B9E085180A008542894162443E
:10ADE000494251180722CE076D082E4349083240C8
:10ADF0001D00A9E6BF49ED1A114007223240A3E623
:10AE0000320028388240002686E6300000F052FAF0
:10AE1000203073E6634613435A1E9341C61AB0426C
:10AE200080414042091A5CE60E006746064317431C
:10AE3000002D5ED1002E00D0F3E0002F00D11EE1E6
:10AE40005C46614691462CE7A94FBE427BD01E006E
:10AE5000F1E610001F3DE840202B03D04021CB1A23
:10AE60009A401643731E9E4107220643324000213A
:10AE7000002583E7161A6346B2428041591A4042C0
:10AE80000B1A98465C4632E61F2E00DDABE0202709
:10AE9000BB1B9A4663465746BB40994613004F4634
:10AEA000F3401F433B005746BA40571EBA41134375
:10AEB0006246F240891898E62027BB1B9A466346F3
:10AEC0005746BB40994613004F46F3401F433B0093
:10AED0005746BA40571EBA4113436246F240891A98
:10AEE0009CE7834B9F425FD080252D04734229430A
:10AEF00020E7002E0CD1002F00D1D0E05C46614647
:10AF000091467B4DCDE67A4FBE421CD01E0065E6D1
:10AF1000002F18D0C0084E0706438020C908000340
:10AF2000014208D06346DC08044204D12100DA461D
:10AF3000D2085E071643F300994601245346C90020
:10AF4000720F11431C406A4DABE61D000022002722
:10AF5000B4E6002D59D10B00034300D1D6E6731C93
:10AF600000D1B2E0624B9F421ED0F343382B6FDC1E
:10AF70001F2B00DD97E020250E00ED1AAE40B046F5
:10AF80000600AA46DE40454635432E005546A840F9
:10AF9000D940451EA8418C440643B61896429241BA
:10AFA000514261443D0025E63D006146914678E608
:10AFB0000B000343002D00D055E6002BF5D063466F
:10AFC000134300D16DE686188642804161444042B9
:10AFD000091800220B0200D4D0E6464B0135194077
:10AFE000B2E5B1465DE633006746203BDF403B00FB
:10AFF000202E05D04027BF1B6646BE4032439046F8
:10B000004646721E96413343EFE5394B9F42CBD003
:10B0100080252D0473422943A8E70843411E884137
:10B02000A2E6002F00D13CE66346861ACF1AB04252
:10B030009B415B42FB1A98461B024ED5161A63468B
:10B04000B2429241591A5242891A5C4600227BE56B
:10B0500001430E00711E8E419FE71D000E00203D32
:10B06000EE40B046202B04D04025EB1A994008430F
:10B07000814648464346411E8841184374E60022F3
:10B08000002417E6161A6346B2429241591A5242F8
:10B09000891A3D0025E561469146154D01E680225D
:10B0A0000024120379E61D000E00203DEE40B0465C
:10B0B000202B04D04025EB1A9940084381464E4688
:10B0C0004346711E8E411E4367E7861896429B4198
:10B0D00061445B42C9183D008CE547463743CED0FA
:10B0E00007224146324049E600273A00E6E5C046DD
:10B0F000FF070000FFFF7FFF70B50C4E0D031C0320
:10B1000049005B002D0B490D240B5B0DB14208D0AB
:10B11000064900208B4203D114432000441EA04165
:10B1200070BD05430120002DFAD1F1E7FF070000B3
:10B1300030B5144D0A034B00120B5B0DC90F0024F0
:10B14000AB4211DD104CA34210DC80246403224387
:10B150000E4CE41A1F2C0CDD0D48C31ADA40130004
:10B160005C42002900D11C00200030BD094BCC18E6
:10B17000FAE7094DE040AC4663449A4013000343AC
:10B18000EEE7C046FE0300001D040000330400008B
:10B1900013040000FFFFFF7FEDFBFFFF70B50028E9
:10B1A0002DD0C317C5185D40C40F280000F082F8E9
:10B1B000154B1B1A5B055B0D0A2815DD0B38854006
:10B1C00000222D032D0B002110002D030A0D2D0B45
:10B1D00012052A430D4D1B052A4013435B00E4076B
:10B1E0005B082343190070BD02002900153291400D
:10B1F0000A000B21081AC5402D032D0BE3E700249C
:10B20000002300250022DEE71E040000FFFF0F8060
:10B210004100090E4B1C70B5DBB24602750AC40F23
:10B22000012B14DDE0239B006D07360BCB180021AA
:10B230000A0D280012051C4D32435B052A405B08AD
:10B2400013435B00E4075B082343190070BD00292A
:10B2500014D1002D1ED0280000F02CF80A281CDC88
:10B260000B232A001B1ADA40030015339D400F4BB5
:10B2700012031B1A5B05160B5B0DD8E7002D06D0D9
:10B28000320B802636036D071643094BCFE7084B78
:10B290000026CCE700230026C9E703002A000B3B69
:10B2A0009A400025E3E7C046FFFF0F8089030000B6
:10B2B000FF0700001C2101231B04984201D3000C4E
:10B2C00010391B0A984201D3000A08391B09984219
:10B2D00001D30009043902A2105C40187047C0462F
:10B2E000040302020101010100000000000000004F
:10B2F00030B51C00094B05001B6885B0D868084BA9
:10B30000002A01D1074B1A000292019300912B00F1
:10B310002200054900F026F800F0A6FD800000207C
:10B3200000E1000038CF00000DE10000014B18687B
:10B330007047C04680000020084B10B50400002B69
:10B3400002D0002100E000BF054B1868836A002B83
:10B3500000D09847200001F05DFBC04600000000CF
:10B360003CE100000EB403B5010003AB044804CB7C
:10B370000068019300F076F802B008BC03B01847EB
:10B380008000002070B500260C4D0D4C641BA410ED
:10B39000A64209D1002601F03FFB0A4D0A4C641B6E
:10B3A000A410A64205D170BDB300EB5898470136F2
:10B3B000EEE7B300EB5898470136F2E75002002061
:10B3C000500200205002002060020020002310B52F
:10B3D0009A4200D110BDCC5CC4540133F8E710B5DB
:10B3E000884202D98B18984203D3002307E08B5C74
:10B3F0008354013AFBD210BDCC5CC45401339A4251
:10B40000FAD1F8E703001218934200D1704719707F
:10B410000133F9E7936810B5013B9360002B04DA20
:10B420009469A34207DB0A2905D01368581C1060F1
:10B430001970080010BD00F04BFC0100F9E7F8B5E9
:10B4400006000F001400D518AC4201D1002007E01F
:10B4500021783A003000FFF7DDFF0134431CF3D1BF
:10B46000F8BD0000F0B59FB002900F0016000593E4
:10B47000002805D083690493002B01D100F0F4FD6E
:10B480007B4B9F425BD1029B5F68BB891B0762D5E8
:10B490003B69002B5FD0002306AC636120336376E9
:10B4A0001033A37635002B78002B01D0252B5CD1EF
:10B4B000AB1B04930CD0320039000298FFF7BFFF9A
:10B4C000431C00D1C4E06269049B944663446361F9
:10B4D0002B78002B00D1BBE0012200235242626096
:10B4E00002A9543252186E1C2360E360A3601370EB
:10B4F000A365317805225F4800F0D4FE751C002852
:10B5000035D12268D30604D5532302A95B18202124
:10B510001970130704D5532302A95B182B21197046
:10B5200033782A2B2CD0350000210A20E3682A78B2
:10B530006E1C303A092A64D900292ED026E04E4BE1
:10B540009F4202D1029B9F689FE74C4B9F429CD138
:10B55000029BDF6899E73900029800F00FFC002891
:10B5600099D0012040421FB0F0BD01359BE7414B0F
:10B570002268C01A01238340134323602E00B8E7DA
:10B58000059B191D1B680591002B01DB099304E045
:10B590005B42E3600223134323602B782E2B0AD1F6
:10B5A0006B782A2B35D1059B02351A1D1B68059235
:10B5B000002B2BDB0793324E29780322300000F05A
:10B5C00071FE002806D04023801B8340226801358D
:10B5D00013432360297806222A486E1C217600F046
:10B5E00061FE00283AD0284B002B25D10722059B6D
:10B5F00007339343083305936369039A9B18636188
:10B6000050E7434301219B18350090E701235B423B
:10B61000D0E700230A201A000135636029786E1CE8
:10B620003039092903D9002BC5D00792C3E742431B
:10B63000012352183500F1E705AB00933A00134B94
:10B640002100029800E000BF0390039B0133D3D197
:10B65000BB895B0600D584E70B9884E705AB0093B4
:10B660003A000A4B2100029800F080F8ECE7C0464F
:10B6700094E1000040E10000B4E1000074E100004A
:10B6800046E100004AE10000000000003FB4000075
:10B69000F7B5150001938A680B6900900C0093427E
:10B6A00000DA130022002B6043321278002A01D006
:10B6B00001332B6023689B0602D52B6802332B6075
:10B6C000062723681F4027D0230043331B785A1EC8
:10B6D00093412268920630D42200019943320098A7
:10B6E000089EB047431C25D0062320682A68E168DD
:10B6F00003400025042B03D18D1AEB43DB171D40BB
:10B70000A3682269934201DD9B1AED180027BD4210
:10B7100020D1002010E00137E3682A689B1ABB4261
:10B72000D2DD22000123193201990098089EB0470A
:10B73000431CF0D101204042FEBD3020E1184331CE
:10B74000087021005A1C45310978A218433202338F
:10B750001170C1E7220001231A3201990098089E56
:10B76000B047431CE6D00137D1E70000F0B589B0FF
:10B7700004920A0043320593039002920A7E0C0061
:10B780000E9B6E2A00D186E01FD8632A33D008D8DA
:10B79000002A00D18CE0582A4DD0250042352A706D
:10B7A00030E0642A01D0692AF7D1196825680A1D9A
:10B7B000280629D508681A60002803DA2D23029A82
:10B7C000404213706B4E0A274FE0732A74D008D89A
:10B7D0006F2A1FD0702AE0D1202209680A43226014
:10B7E00003E0752A16D0782AD7D122007821453275
:10B7F0001170614E22E025001A684235111D196052
:10B8000013682B70012365E008681A606906D3D5B8
:10B8100000B2D1E719682568081D186008682E066F
:10B8200005D5544E08276F2A1BD00A2719E06D064C
:10B83000F7D580B2F5E745314E4E0A701868226898
:10B84000011D00681960150621D5D30702D52023F4
:10B850001A4322601027002803D1202322689A432C
:10B8600022602300002243331A706368A360002B18
:10B8700058DB0422216891432160002854D1029DA5
:10B88000002B5AD02500337842352B7055E05506F1
:10B89000DBD580B2D9E71A680D68101D49691860B8
:10B8A00013682E0601D5196002E06D06FBD51980DC
:10B8B0000023029D23614FE01A68111D196015686D
:10B8C00000216268280000F0EDFC002801D0401B38
:10B8D0006060636823610023029A13703CE023696F
:10B8E0002A0004990398059DA847431C3ED023686D
:10B8F0009B0715D4079BE068984239DA180037E0B7
:10B9000022000123193204990398059EB047431C75
:10B910002CD00135E368079A9B1AAB42F0DCE9E7CB
:10B920000025F7E70028ADD0029D3900FDF722FC85
:10B93000735C013D2B700028F7D1082F09D12368D3
:10B94000DB0706D563682269934202DC3023013DA0
:10B950002B70029B5B1B2361059B07AA00932100B0
:10B96000049B0398FFF794FE431CB8D1012040428A
:10B9700009B0F0BD51E1000062E100000D4B70B56F
:10B980001C680500A36B002B0FD1182000F06EFC83
:10B99000094BA0630360094B01224360084B83609D
:10B9A0000B2383810023026143610022A36B1D618D
:10B9B0005A6170BD800000200E33CDAB34126DE6AD
:10B9C000ECDE0500124B10B51C68A36B002B0FD1E9
:10B9D000182000F04BFC0F4BA06303600E4B0122BC
:10B9E00043600E4B83600B2383810023026143611C
:10B9F000A46B0B4A206961690A4BFDF7F7FC012231
:10BA0000002380185941206161614800400810BD41
:10BA1000800000200E33CDAB34126DE6ECDE050065
:10BA20002D7F954C2DF451580CB430B5164B9DB06C
:10BA30000C1E1D6808DA8B2301202B6040421DB0CC
:10BA400030BC08BC02B01847822302A99B008B813E
:10BA50000023029008619C4200D0631E8B604B6102
:10BA600001235B42CB81209A21AB2800019300F097
:10BA700055FD431C01DA8B232B60002CDFD0002303
:10BA8000029A1370DBE7C046800000200EB400B5B8
:10BA90000B499CB01DAB0290069007910491094898
:10BAA000094904CB0591006802A9019300F036FD15
:10BAB0000023029A13701CB008BC03B01847C0469C
:10BAC000FFFFFF7F800000200802FFFF020010B58B
:10BAD0001378541C002B05D1CC5CD4540133002CBA
:10BAE000FAD110BD2200F3E7C9B20378002B04D0CD
:10BAF0008B4200D170470130F7E74B425941494230
:10BB00000840F7E702780B78002A03D001300131B2
:10BB10009A42F7D0D01A70470023C25C0133002A42
:10BB2000FBD1581E7047002330B59A420AD0013A23
:10BB3000C45CCD5CAC4204D1934202D00133002CF2
:10BB4000F6D1631B180030BD30B50500002A00D1C6
:10BB500030BD0C78013A6B1C2C700131002C05D1E2
:10BB60009A189A42F4D01C700133FAE71D00EDE7F1
:10BB700010B50378002B0FD10B785A4253415B422A
:10BB8000184010BD0023CA5C002AFAD0C45C94425D
:10BB900001D10133F7E701300378002BF2D118000F
:10BBA000EFE70000F0B51F000E0087B0059001918F
:10BBB00002920C98347800F0EAFA082200194378CF
:10BBC000751C134036D12D2C36D1B51C7478012646
:10BBD000002F62D0102F09D1302C07D120222B78D2
:10BBE0009343582B54D110276C7802352D4B3900D4
:10BBF000F31818000393FDF7BDFA04910121002307
:10BC0000494202008C4618002100303909291AD80F
:10BC10000C00A74223DD591C09D06346824206D39B
:10BC200002D10499A14202DB0123784320182C7829
:10BC30000135E9E72E00BCE72B2C01D01E00C7E739
:10BC4000B51C7478FAE721004139192901D8373C2D
:10BC5000DFE721006139192901D8573CD9E75A1C7F
:10BC600008D1059A23331360029B0398002B09D156
:10BC700007B0F0BD002E00D04042029A002AF7D053
:10BC8000002B01D06B1E0193029B019A1A60EFE713
:10BC90003024002FAAD10827A8E7302C9ED00A27ED
:10BCA000A4E7C046FFFFFF7F37B51300064A050033
:10BCB0001068046A002C00D1044C0A00009429008A
:10BCC000FFF770FF3EBDC04680000020E40000206A
:10BCD000F8B505000E001400002804D08369002B7D
:10BCE00001D100F0C1F9224B9C422DD16C68A369AF
:10BCF000A360A3891B0731D52369002B2ED02368AD
:10BD00002269F7B2981A6369F6B2834205DC210012
:10BD1000280000F03BF9002826D1A3680130013B40
:10BD2000A36023685A1C22601F706369834204D099
:10BD3000A389DB071AD50A2E18D12100280000F0AC
:10BD400025F9002812D00FE00A4B9C4201D1AC68C3
:10BD5000CDE7094B9C42CAD1EC68C8E72100280016
:10BD600000F00CF80028CAD0012676423000F8BD59
:10BD700094E10000B4E1000074E10000364B70B5BE
:10BD80001D6806000C00002D05D0AB69002B02D108
:10BD9000280000F069F9314B9C420FD16C680C23EC
:10BDA000E25E93B219072DD4D90611D409230120DC
:10BDB000336037331343A381404270BD284B9C420C
:10BDC00001D1AC68EBE7274B9C42E8D1EC68E6E791
:10BDD0005B0713D5616B002908D0230044339942D7
:10BDE00002D0300000F06AFA002363632422A389A2
:10BDF0009343A38100236360236923600823A289FE
:10BE00001343A3812369002B0BD1A0218022A38996
:10BE1000890092000B40934203D02100300000F0D3
:10BE2000E1F90123A289134011D00023A3606369C3
:10BE30005B42A361002023698342BED10C23E25EF2
:10BE40001306BAD540231343A3810138B5E79207FF
:10BE500000D46369A360EDE78000002094E1000056
:10BE6000B4E1000074E1000010B5062000F090FC81
:10BE7000012000F0CFFD0000F7B58A8905000C0015
:10BE8000130760D44B68002B04DC0B6C002B01DC27
:10BE90000020FEBDE76A002FFAD000232E682B6039
:10BEA00080235B01216A1A4034D0606DA3895B074F
:10BEB00006D56368C01A636B002B01D0236CC01ACF
:10BEC0000200216A00232800E76AB847A189431CC1
:10BED00006D12B681D2B30D82B4ADA40D3072CD53E
:10BEE0000023636023692360CB0405D5431C02D182
:10BEF0002B68002B00D16065616B2E600029C7D0D4
:10BF000023004433994202D0280000F0D7F90020E2
:10BF10006063BEE701232800B847431CC6D12B68E5
:10BF2000002BC3D01D2B01D0162B01D12E60AFE703
:10BF30004023A2891343A381ABE740230B43012095
:10BF4000A3814042A5E70F69002FA1D00B680F60C5
:10BF5000DB1B01930023920700D14B69A360019B77
:10BF6000002B00DC94E7019B3A00216A2800A66AB6
:10BF7000B047002803DC4023A2891343DFE7019B7D
:10BF80003F181B1A0193EAE7010040200B6970B5C6
:10BF900005000C00002B01D1002070BD002804D04A
:10BFA0008369002B01D100F05FF80B4B9C4209D153
:10BFB0006C680C22A35E002BEED021002800FFF756
:10BFC0005BFFEAE7054B9C4201D1AC68F1E7044B0B
:10BFD0009C42EED1EC68ECE794E10000B4E1000093
:10BFE00074E10000002310B5040003604360836027
:10BFF00081814366C2810361436183611900082224
:10C000005C30FFF7FFF9054B24626362044BA362C7
:10C01000044BE362044B236310BDC046D1C700004C
:10C02000F9C7000031C800005DC8000010B5024922
:10C0300000F08CF810BDC0468DBF000070B56825BB
:10C040004A1E55430E002900743100F081F9041E88
:10C0500008D000212A00016046600C30A0606832E0
:10C06000FFF7D0F9200070BD836913B50400002BE1
:10C0700028D18364C3640365134B144A1B6882622E
:10C080000193984201D101238361200000F020F840
:10C090006060200000F01CF8A060200000F018F89C
:10C0A0000022E06004216068FFF79CFF0122092163
:10C0B000A068FFF797FF02221221E068FFF792FFC6
:10C0C0000123A36113BDC0463CE100002DC0000068
:10C0D000F8B51C4B07001E68B369002B02D1300075
:10C0E000FFF7C2FF4836B4687368013B04D5336874
:10C0F000002B07D03668F6E70C22A55E002D0DD088
:10C100006834F2E704213800FFF798FF3060002818
:10C11000F0D10C2304003B602000F8BD20000A4B46
:10C12000656625606560A560E36025616561A56160
:10C13000082229005C30FFF765F96563A563A564F3
:10C14000E564E9E73CE100000100FFFFF7B504000A
:10C150000700002601914834002C01D13000FEBDBB
:10C160006368A5680093009B013B009301D5246898
:10C17000F2E7AB89012B08D90E22AB5E013304D064
:10C1800029003800019B984706436835EBE7EC30FF
:10C190000068704770B50E001D000E23C95E96B092
:10C1A0001400002907DA00232B60B3891B0611D481
:10C1B0008023DB000FE06A4600F088FB0028F2DBFA
:10C1C000F022019B12021340054A9B185A42534128
:10C1D0002B60EDE740230020236016B070BDC04601
:10C1E00000E0FFFFF7B502268B8905000C00334203
:10C1F00006D0230047332360236101236361F7BD29
:10C2000001AB6A46FFF7C6FF00990700280000F05F
:10C210009FF8002808D10C22A35E9A05EFD40322D0
:10C2200093431E43A681E4E70F4BAB628023A289B0
:10C2300020601343A381009B20616361019B002B5D
:10C240000DD00E23E15E280000F052FB002806D03E
:10C250000322A38993431A0001231343A381A089D6
:10C260003843A081CBE7C0462DC0000010B5034B7A
:10C270000100186800F06CF810BDC0468000002076
:10C2800082B0002900D101A9101E06D0002B06D0D3
:10C2900013780B601078431E984102B0704702205B
:10C2A0004042FAE7C9B28218904201D1002070479B
:10C2B00003788B42FBD00130F6E7000070B5050033
:10C2C000002910D00C1F2368002B00DAE418280086
:10C2D00000F034FB1D4A1368002B05D16360146025
:10C2E000280000F02CFB70BDA34209D9216860181A
:10C2F0008342F3D118685B6841182160EEE71300B0
:10C300005A68002A01D0A242F9D919685818A042E7
:10C310000BD120680918581819608242E0D11068C2
:10C320005268411819605A60DAE7A04202D90C231A
:10C330002B60D5E721686018824203D110685268EB
:10C340004118216062605C60CAE7C046201C002082
:10C35000032370B5CD1C9D43083506000C2D1ED25D
:10C360000C25A9421DD8300000F0E8FA254A1468CF
:10C370002100002919D1244C2368002B03D130005F
:10C3800000F0CAF920602900300000F0C5F9431C14
:10C390002BD10C233000336000F0D1FA03E0002DE4
:10C3A000DFDA0C233360002070BD0B685B1B19D4EF
:10C3B0000B2B03D90B60CC18256003E04B688C4233
:10C3C0000DD11360300000F0BAFA200007220B30C4
:10C3D000231D9043C31AE7D05A42E250E4E763605A
:10C3E0000C00EFE70C004968C3E70323C41C9C431F
:10C3F000A042E1D0211A300000F08EF9431CDBD1BD
:10C40000C7E7C046201C0020241C0020F8B5070008
:10C410000D001600002905D11100FFF799FF040057
:10C420002000F8BD002A03D1FFF748FF3400F7E7EA
:10C4300000F086FA2C00B042F2D231003800FFF74B
:10C4400087FF041EECD029003200FEF7BFFF290051
:10C450003800FFF733FFE3E7F0B58E6885B00700DB
:10C460000C00039201939E423CD890238A89DB0002
:10C470001A4234D00325096923685B1A0293636961
:10C4800002985D43EB0F5D19019B6D1001331B1882
:10C49000AB4200D91D00530532D529003800FFF703
:10C4A00057FF061E09D10C233B6040230120A289BF
:10C4B00040421343A38105B0F0BD029A2169FEF703
:10C4C00085FFA389144A1A4080231343A381029B4A
:10C4D0002661F61826606561019EED1AA560019B34
:10C4E0009E4200D9019E320003992068FEF777FF33
:10C4F000A36800209B1BA36023689E192660DAE7CF
:10C500002A003800FFF782FF061EE0D121693800BB
:10C51000FFF7D4FEC7E7C0467FFBFFFFF0B59FB033
:10C52000029005938B890F0016001B0611D50B692D
:10C53000002B0ED14021FFF70BFF38603861002837
:10C5400005D10C23029A013813601FB0F0BD4023BF
:10C550007B61002306AC6361203363761033A376DE
:10C5600035002B78002B01D0252B46D1AB1B049333
:10C570000CD0320039000298FFF76EFF431C00D147
:10C58000AEE06269049B9446634463612B78002BA0
:10C5900000D1A5E0012200235242626002A9543278
:10C5A00052186E1C2360E360A3601370A36531789A
:10C5B00005225448FFF776FE751C00281FD122681B
:10C5C000D30604D5532302A95B1820211970130741
:10C5D00004D5532302A95B182B21197033782A2B19
:10C5E00016D0350000210A20E3682A786E1C303A04
:10C5F000092A4ED9002918D010E00135B1E7414B86
:10C600002268C01A01238340134323602E00CEE723
:10C61000059B191D1B680591002B01DB099304E0A4
:10C620005B42E3600223134323602B782E2B0AD155
:10C630006B782A2B35D1059B02351A1D1B68059294
:10C64000002B2BDB0793304E297803223000FFF7B5
:10C6500029FE002806D04023801B83402268013534
:10C66000134323602978062228486E1C2176FFF7A1
:10C6700019FE00283CD0264B002B25D10722059B14
:10C6800007339343083305936369039A9B186361E7
:10C6900066E7434301219B183500A6E701235B426F
:10C6A000D0E700230A201A000135636029786E1C48
:10C6B0003039092903D9002BC5D00792C3E742437B
:10C6C000012352183500F1E705AB00933A00114BF6
:10C6D0002100029800E000BF0390039B0133D3D1F7
:10C6E000BB890B985B0600D42FE7012040422CE762
:10C6F00005AB00933A00074B21000298FFF736F88C
:10C70000EAE7C04640E1000046E100004AE10000DF
:10C710000000000059C40000002370B5064C05005D
:10C720000800236000F060F9431C03D12368002B4C
:10C7300000D02B6070BDC046B42F002070B504003F
:10C740000D001F2904D9162303600120404270BD4B
:10C75000436C002B04D08A009B181A68002A08D169
:10C76000200000F031F82A000100200000F01AF843
:10C77000EDE70020012AEAD0511C03D11623013035
:10C780002360E4E7002428001C6090472000DEE7D7
:10C7900010B5034B01001868FFF7D0FF10BDC0466D
:10C7A00080000020002370B5064C05000800110031
:10C7B000236000F001F9431C03D12368002B00D053
:10C7C0002B6070BDB42F002010B500F0E5F810BD4F
:10C7D00070B50C000E25495F00F0BAF8002803DBA5
:10C7E000636D1B18636570BDA389024A1340A38162
:10C7F000F9E7C046FFEFFFFFF8B51F008B89050082
:10C800000C001600DB0505D50E23C95E00220223AD
:10C8100000F080F8A389054A28001340A381320064
:10C820000E23E15E3B0000F02BF8F8BDFFEFFFFFA9
:10C8300070B50C000E25495F00F06CF8A389421C0E
:10C8400003D1054A1340A38170BD802252011343D6
:10C85000A3816065F8E7C046FFEFFFFF10B50E2328
:10C86000C95E00F021F810BD0B1E04D0FF2A04D9C8
:10C870008A2303608B3B180070470A700123FAE794
:10C8800070B50500080011000022064C22601A0055
:10C8900000F0B8F8431C03D12368002B00D02B60B4
:10C8A00070BDC046B42F0020002370B5064C0500B3
:10C8B0000800236000F060F8431C03D12368002BBC
:10C8C00000D02B6070BDC046B42F0020002370B58F
:10C8D000064C050008001100236000F055F8431CC9
:10C8E00003D12368002B00D02B6070BDB42F002033
:10C8F000002370B5064C05000800236000F054F8D2
:10C90000431C03D12368002B00D02B6070BDC046B0
:10C91000B42F002070B50500080011000022064C5D
:10C9200022601A0000F050F8431C03D12368002B4A
:10C9300000D02B6070BDC046B42F002070477047F8
:10C940000B1F1B68181F002B01DA0B58C01870470B
:10C9500070B50500080011000022064C22601A0084
:10C9600000F03AF8431C03D12368002B00D02B6061
:10C9700070BDC046B42F002058220120014B404218
:10C980001A607047B42F002058220120014B40420A
:10C990001A607047B42F002058220120014B4042FA
:10C9A0001A607047B42F00205822024B00201A60F2
:10C9B0007047C046B42F002058220120014B40424E
:10C9C0001A607047B42F002058220120014B4042CA
:10C9D0001A607047B42F002058220120014B4042BA
:10C9E0001A607047B42F0020044A1368002B00D14E
:10C9F000034B1818106018007047C046281C002010
:10CA0000B82F002058220120014B40421A60704785
:10CA1000B42F0020FEE7C046F8B5C046F8BC08BCFD
:10CA20009E467047F8B5C046F8BC08BC9E467047A5
:10CA30006461746100000000B4CA0000EF010000EE
:10CA4000BDCA0000E3020000C5CA000009090000D9
:10CA5000CCCA0000190A0000D1CA0000310500004C
:10CA6000DCCA000053030000E1CA0000710C0000A2
:10CA7000EDCA00001F020000F7CA00001108000004
:10CA800005CB0000BD06000012CB0000F104000041
:10CA900072616E646F6D00616C6C006C6173740028
:10CAA00066616C7365007472756500252E3135738F
:10CAB0002E2E2E006D616B654C6973740061646489
:10CAC0004C6173740064656C657465006A6F696EAF
:10CAD00000636F707946726F6D546F0066696E64A3
:10CAE000006A6F696E537472696E677300756E6960
:10CAF000636F6465417400756E69636F6465537438
:10CB000072696E67006E6577427974654172726111
:10CB10007900667265654D656D6F72790000000081
:10CB200085CB0000D91000008ACB0000F710000070
:10CB3000C5CA0000FB10000090CB0000DD10000013
:10CB40009ACB0000FF100000A3CB000003110000EF
:10CB5000ADCB000007110000B8CB00000B110000A6
:10CB6000C4CB0000E1100000CDCB0000EF100000AE
:10CB7000D7CB0000E5100000E2CB0000F31000006E
:10CB800066696C65006F70656E00636C6F7365003D
:10CB9000656E644F6646696C6500726561644C69D8
:10CBA0006E650072656164427974657300617070CE
:10CBB000656E644C696E6500617070656E64427983
:10CBC0007465730066696C6553697A650073746196
:10CBD00072744C697374006E657874496E4C697335
:10CBE000740073797374656D496E666F00000000A0
:10CBF000381300004813000062130000E013000027
:10CC0000181400004E14000086140000AC1400003C
:10CC1000E81400002A15000080150000C41500006B
:10CC200030160000781600009E160000D616000090
:10CC30001C17000042170000701700009E1700002C
:10CC4000D4170000581800002019000096190000A1
:10CC5000061A0000521A0000721A0000941A00000E
:10CC6000461B00008C1B0000041C00003813000051
:10CC700038130000321C00009A1C0000021D000046
:10CC8000601D0000A81D00001E1E0000941E000074
:10CC9000DC1E0000221F0000581F00009E1F000025
:10CCA000E41F00002C20000080200000D4200000A1
:10CCB0001C21000086210000BC210000042200008D
:10CCC0004C22000094220000CE2200001623000017
:10CCD0005E230000C0240000381300003813000059
:10CCE000C623000038130000FC23000028240000A5
:10CCF0005E2400008A24000038130000381300006E
:10CD0000381300003813000042250000842500007D
:10CD10003813000038130000CA2500001A2600004E
:10CD200040260000381300003813000038130000BC
:10CD30006E2600009E260000CE260000042700007C
:10CD40002E270000642700008E270000B627000071
:10CD5000DE2700000E2800003E28000068280000A2
:10CD600092280000F02800001A2900003813000063
:10CD70003813000038130000381300003813000087
:10CD80004A29000076290000A2290000CE290000CF
:10CD9000FA290000302A0000662A00009C2A0000C0
:10CDA000D22A0000FE2A00002A2B0000602B00007F
:10CDB0003813000038130000381300003813000047
:10CDC0003813000038130000381300003813000037
:10CDD0003813000038130000381300003813000027
:10CDE00038130000381300008C2B0000C22B000009
:10CDF0005B2564206974656D206C6973745D00281F
:10CE000025642062797465732900286F626A6563FE
:10CE10007420747970653A20256429005374616325
:10CE20006B20756E646572666C6F7700626F6F6CF5
:10CE300065616E006E756D62657200737472696E05
:10CE400067006C6973740062797465206172726145
:10CE5000790000000700000003000000AECE0000D3
:10CE6000E52C0000B6CE0000952D0000BFCE0000DE
:10CE70003F2E0000C8CE0000E92C0000D1CE0000FB
:10CE8000432E0000D9CE00002D2E0000000000002F
:10CE90000100000002000000030000000400000088
:10CEA0000A0000006D6963726F3A6269740068611C
:10CEB00073546F6E6500706C6179546F6E650068B5
:10CEC0006173536572766F00736574536572766F24
:10CED00000646163496E69740064616357726974C8
:10CEE0006500474320746F6F6B2025642075736560
:10CEF00063733B206672656520256420776F7264DA
:10CF000073003C496E74656765723E003C4C697302
:10CF1000743E003C4F626A6563743E003C42797423
:10CF20006541727261793E000D0A564D2050616E66
:10CF300069633A2025730D0A006D69736300000070
:10CF400075CF0000093B00007ECF0000993A000039
:10CF500082CF0000ED3900008ACF00009339000035
:10CF600094CF000029390000A0CF00002B3800002A
:10CF70006E756C6C00686578546F496E74007369E7
:10CF80006E006A736F6E476574006A736F6E436FED
:10CF9000756E74006A736F6E56616C7565417400CE
:10CFA0006A736F6E4B6579417400000008D0000011
:10CFB000753B000010D00000793B00001AD0000043
:10CFC000973B000023D00000A13B00002ED00000C2
:10CFD000AB3B00003AD00000B53B00004FD0000052
:10CFE000BF3B000064D00000C93B000070D00000CF
:10CFF000D33B000080D00000833B00008CD00000B9
:10D000008D3B00006E657400686173576946690066
:10D010007374617274576946690073746F705769ED
:10D0200046690077696669537461747573006D7938
:10D030004950416464726573730068747470536519
:10D0400072766572476574526571756573740072A6
:10D050006573706F6E64546F487474705265717547
:10D060006573740068747470436F6E6E65637400EA
:10D07000687474704973436F6E6E656374656400A1
:10D080006874747052657175657374006874747037
:10D09000526573706F6E7365001A1B1C03040607DC
:10D0A000090A171819000000000008080800080AFB
:10D0B0004A4000000A5FEA5FEA0ED92ED36E1932A9
:10D0C0004489330C924C924D0808000000048808F3
:10D0D00008040804848488000A448A4000048EC43A
:10D0E00080000000048800000EC00000000008005E
:10D0F00001224488100C9252524C048C84848E1C61
:10D10000824C901E1EC244924C06CA525FE21FF02F
:10D110001EC13E02448ED12E1FE24488100ED12E35
:10D12000D12E0ED12EC4880008000800000480040F
:10D13000880244880482000EC00EC008048244881D
:10D140000ED126C0040ED135B36C0C925ED2521CA7
:10D15000925C925C0ED010100E1C9252525C1ED04B
:10D160001C901E1ED01C90100ED013712E12525EF9
:10D17000D2521C8808081C1FE242524C12549814C8
:10D1800092101010101E113B75B131113935B37169
:10D190000C9252524C1C925C90100C92524C861C79
:10D1A000925C92510ED00C825C1FE48484841252F3
:10D1B00052524C1131312A44113135BB7112524C4B
:10D1C0009252112A4484841EC488101E0EC8080876
:10D1D0000E10080482410EC242424E048A400000F2
:10D1E000000000001F0804800000000ED2524F1003
:10D1F000101C925C000ED0100E02424ED24E0C92C9
:10D200005C900E06C81C88080ED24EC24C10101C32
:10D2100092520800080808024002424C1014981468
:10D22000920808080806001B75B131001C92525282
:10D23000000C92524C001C925C90000ED24EC20028
:10D240000ED010100006C8049808080EC807001277
:10D2500052524F0011312A4400113135BB00124C9B
:10D260008C9200112A4498001EC4881E06C48C8427
:10D2700086080808080818080C881800000C836045
:10D280000000000001000000020000000300000098
:10D290000400000005000000060000000700000078
:10D2A00008000000090000000A0000000B00000058
:10D2B0000C0000000D0000000E0000000F00000038
:10D2C0001000000012000000140000001600000012
:10D2D000180000001A0000001C0000001E000000E2
:10D2E00020000000230000002600000029000000AC
:10D2F0002C0000002F00000032000000360000006B
:10D300003A0000003E00000042000000460000001D
:10D310004B00000050000000550000005A000000C3
:10D3200061000000680000006F000000760000004F
:10D330007D000000840000008B00000092000000CF
:10D3400099000000A0000000A7000000AE0000004F
:10D35000B5000000BC000000C3000000CA000000CF
:10D36000D1000000D8000000DF000000E60000004F
:10D37000ED000000F4000000FB000000FF000000D2
:10D38000D0D30000F53B0000DBD300004541000096
:10D39000E5D30000B13D0000F2D30000B53F00002E
:10D3A000F9D300000540000002D400005540000001
:10D3B0000ED400004D3F00001FD40000213E0000AD
:10D3C0002CD40000DD3E0000646973706C6179004C
:10D3D0006C696768744C6576656C006D624469734E
:10D3E000706C6179006D62446973706C61794F662D
:10D3F00066006D62506C6F74006D62556E706C6F7C
:10D4000074006D62447261775368617065006D628B
:10D410005368617065466F724C6574746572006E16
:10D42000656F506978656C53656E64006E656F500A
:10D430006978656C53657450696E004E6F74206531
:10D440006E6F75676820726F6F6D206576656E20F0
:10D45000616674657220636F6D70616374696F6E6D
:10D4600000436F6D70616374656420466C6173681E
:10D4700020636F64652073746F72650A256420628F
:10D4800079746573207573656420282564252529C2
:10D49000206F6620256400426164207265636F72AC
:10D4A0006420666F756E6420647572696E672069AA
:10D4B0006E697469616C697A6174696F6E00256464
:10D4C0002025642025642028256420776F726473EA
:10D4D00029002564207265636F7264732C202564B3
:10D4E00020776F7264732C206D6178494420256425
:10D4F0002C20636F6D70616374696F6E2063796354
:10D500006C657320256400526573746F72656420C6
:10D51000256420736372697074730053746172744C
:10D52000656400726164696F00000000BCD5000092
:10D530000D4B0000C9D50000A94D0000D9D5000051
:10D54000294D0000E7D500003D4F0000F2D5000056
:10D55000354B000002D60000BD4B000016D600007F
:10D56000A54B000025D600001F51000031D6000059
:10D570009D5000003AD600004150000045D6000002
:10D58000894F000050D60000C54F000059D600005A
:10D59000F94F000062D60000454B000071D6000034
:10D5A000254B00007AD60000554B00006E6F6E656B
:10D5B000006F7468657200706169720064697361FC
:10D5C000626C65526164696F006D65737361676554
:10D5D0005265636569766564007061636B6574525A
:10D5E000656365697665007061636B657453656E2C
:10D5F00064007265636569766564496E7465676524
:10D60000720072656365697665644D657373616701
:10D6100065547970650072656365697665645374F5
:10D6200072696E670073656E64496E7465676572D2
:10D630000073656E64506169720073656E64537443
:10D6400072696E67007365744368616E6E656C0025
:10D6500073657447726F757000736574506F77658A
:10D6600072007369676E616C537472656E6774687B
:10D67000006465766963654944006C6173744D6547
:10D680007373616765494400556E6B6E6F776E20EA
:10D690007072696D6974697665205B25733A2573CC
:10D6A0005D00000000000000963007772C610EEE50
:10D6B000BA51099919C46D078FF46A7035A563E9E9
:10D6C000A395649E3288DB0EA4B8DC791EE9D5E010
:10D6D00088D9D2972B4CB609BD7CB17E072DB8E70F
:10D6E000911DBF906410B71DF220B06A4871B9F364
:10D6F000DE41BE847DD4DA1AEBE4DD6D51B5D4F49D
:10D70000C785D38356986C13C0A86B647AF962FD01
:10D71000ECC9658A4F5C0114D96C0663633D0FFA4E
:10D72000F50D088DC8206E3B5E10694CE44160D554
:10D73000727167A2D1E4033C47D4044BFD850DD23E
:10D740006BB50AA5FAA8B5356C98B242D6C9BBDB51
:10D7500040F9BCACE36CD832755CDF45CF0DD6DC4C
:10D76000593DD1ABAC30D9263A00DE518051D7C8F3
:10D770001661D0BFB5F4B42123C4B3569995BACF7E
:10D780000FA5BDB89EB802280888055FB2D90CC69F
:10D7900024E90BB1877C6F2F114C6858AB1D61C118
:10D7A0003D2D66B69041DC760671DB01BC20D29837
:10D7B0002A10D5EF8985B1711FB5B606A5E4BF9FC4
:10D7C00033D4B8E8A2C9077834F9000F8EA80996B7
:10D7D00018980EE1BB0D6A7F2D3D6D08976C649122
:10D7E000015C63E6F4516B6B62616C1CD83065853B
:10D7F0004E0062F2ED95066C7BA5011BC1F4088218
:10D8000057C40FF5C6D9B06550E9B712EAB8BE8B58
:10D810007C88B9FCDF1DDD62492DDA15F37CD38CE1
:10D82000654CD4FB5861B24DCE51B53A7400BCA3DF
:10D83000E230BBD441A5DF4AD795D83D6DC4D1A411
:10D84000FBF4D6D36AE96943FCD96E34468867ADE8
:10D85000D0B860DA732D0444E51D03335F4C0AAA87
:10D86000C97C0DDD3C710550AA41022710100BBE8A
:10D8700086200CC925B56857B3856F2009D466B9D1
:10D880009FE461CE0EF9DE5E98C9D9292298D0B006
:10D89000B4A8D7C7173DB359810DB42E3B5CBDB7B3
:10D8A000AD6CBAC02083B8EDB6B3BF9A0CE2B60334
:10D8B0009AD2B1743947D5EAAF77D29D1526DB04E9
:10D8C0008316DC73120B63E3843B64943E6A6D0D34
:10D8D000A85A6A7A0BCF0EE49DFF099327AE000A7F
:10D8E000B19E077D44930FF0D2A3088768F2011E12
:10D8F000FEC206695D5762F7CB67658071366C19A9
:10D90000E7066B6E761BD4FEE02BD3895A7ADA10C9
:10D91000CC4ADD676FDFB9F9F9EFBE8E43BEB717AA
:10D92000D58EB060E8A3D6D67E93D1A1C4C2D83834
:10D9300052F2DF4FF167BBD16757BCA6DD06B53F9A
:10D940004B36B248DA2B0DD84C1B0AAFF64A0336D9
:10D95000607A0441C3EF60DF55DF67A8EF8E6E3158
:10D9600079BE69468CB361CB1A8366BCA0D26F25A1
:10D9700036E2685295770CCC03470BBBB9160222EE
:10D980002F260555BE3BBAC5280BBDB2925AB42B03
:10D99000046AB35CA7FFD7C231CFD0B58B9ED92C18
:10D9A0001DAEDE5BB0C2649B26F263EC9CA36A757D
:10D9B0000A936D02A906099C3F360EEB8567077234
:10D9C00013570005824ABF95147AB8E2AE2BB17B9B
:10D9D000381BB60C9B8ED2920DBED5E5B7EFDC7C22
:10D9E00021DFDB0BD4D2D38642E2D4F1F8B3DD6879
:10D9F0006E83DA1FCD16BE815B26B9F6E177B06F74
:10DA00007747B718E65A0888706A0FFFCA3B066660
:10DA10005C0B0111FF9E658F69AE62F8D3FF6B61ED
:10DA200045CF6C1678E20AA0EED20DD75483044E8F
:10DA3000C2B30339612667A7F71660D04D4769491D
:10DA4000DB776E3E4A6AD1AEDC5AD6D9660BDF4030
:10DA5000F03BD83753AEBCA9C59EBBDE7FCFB247E3
:10DA6000E9FFB5301CF2BDBD8AC2BACA3093B353C8
:10DA7000A6A3B4240536D0BA9306D7CD2957DE54D1
:10DA8000BF67D9232E7A66B3B84A61C4021B685DAA
:10DA9000942B6F2A37BE0BB4A18E0CC31BDF055A23
:10DAA0008DEF022D416C6C207461736B7320737465
:10DAB0006F7070656400763038340020257320253F
:10DAC00073004D656D6F727920636C65617265647A
:10DAD000004E6F2066726565207461736B20656E01
:10DAE000747269657300000030DB0000A9640000F7
:10DAF0003DDB0000E560000049DB000079640000C8
:10DB00004FDB00008964000055DB000099640000D1
:10DB10005BDB00001961000065DB000005650000AB
:10DB20006DDB00005962000073656E736F727300E5
:10DB3000616363656C65726174696F6E0074656DB5
:10DB400070657261747572650074696C74580074E4
:10DB5000696C74590074696C745A00746F756368E9
:10DB600052656164006932635265616400693263C1
:10DB70005772697465000000ECDB000091650000DD
:10DB8000FADB00009565000003DC0000A1650000E1
:10DB90000DDC0000A565000016DC0000A965000092
:10DBA0001BDC0000AD65000020DC0000B16500005A
:10DBB0002CDC0000B565000033DC0000B965000016
:10DBC0003CDC0000BD65000041DC0000C1650000D8
:10DBD0004CDC0000C565000056DC000099650000C3
:10DBE00060DC00009D65000074667400656E616213
:10DBF0006C65446973706C6179006765745769641A
:10DC00007468006765744865696768740073657453
:10DC1000506978656C006C696E65007265637400AC
:10DC2000726F756E646564526563740063697263D4
:10DC30006C6500747269616E676C650074657874F8
:10DC400000746674546F7563686564007466745418
:10DC50006F7563685800746674546F756368590013
:10DC6000746674546F75636850726573737572650A
:10DC7000007661727300000098DC0000556A0000B5
:10DC8000A2DC0000356A0000ABDC0000116A000075
:10DC9000B7DC00009D690000766172457869737495
:10DCA00073007661724E616D6564007365745661D0
:10DCB000724E616D6564007661724E616D65466F8E
:10DCC00072496E6465780057656C636F6D6520748A
:10DCD0006F204D6963726F426C6F636B73210070CC
:10DCE0005F73706920213D204E554C4C002F686FAA
:10DCF0006D652F6769742F2E706C6174666F726D1D
:10DD0000696F2F7061636B616765732F6672616DF8
:10DD100065776F726B2D61726475696E6F6E6F726D
:10DD20006469636E7266352F6C69627261726965CF
:10DD3000732F5350492F5350492E63707000535026
:10DD400049436C6173733A3A535049436C6173733E
:10DD5000284E52465F5350495F547970652A2C20F3
:10DD600075696E74385F742C2075696E74385F74D1
:10DD70002C2075696E74385F742900000000000063
:10DD800000000000616C00001D6C0000436C00008E
:10DD90004D6C0000576C0000416C00000300000057
:10DDA0000200000001000000040000000500000067
:10DDB000110000000C0000000B0000001200000029
:10DDC0000A000000060000001A0000001400000015
:10DDD00017000000160000001500000010000000F1
:10DDE000FFFFFFFFFFFFFFFF000000001E0000001D
:10DDF00019000000180000000700000008000000E3
:10DE0000090000000D0000000E0000000F000000DF
:10DE10001C0000001B0000001D000000130000009B
:10DE200000000000000000001171000041780000B7
:10DE300091710000A57100009B7100000D71000040
:10DE400001710000B17100002D710000FD70000033
:10DE5000000000000000304300000000000030C35C
:10DE60007371727400000000FB21F93FFB2109402F
:10DE70007CD91240FB2119407A6A1F407CD922408C
:10DE8000BBFD2540FB2129403A462C407A6A2F40B1
:10DE90005C4731407CD932409C6B3440BBFD3540FF
:10DEA000DB8F3740FB2139401BB43A403A463C40B7
:10DEB0005AD83D407A6A3F404C7E40405C474140E2
:10DEC0006C1042407CD942408CA243409C6B444041
:10DED000AC344540BBFD4540CBC64640DB8F474098
:10DEE000EB584840FB21494083F9A200444E6E00A4
:10DEF000FC291500D1572700DD34F50062DBC00096
:10DF00003C999500419043006351FE00BBDEAB009D
:10DF1000B761C5003A6E2400D24D42004906E000C8
:10DF200009EA2E001C92D100EB1DFE0029B11C0055
:10DF3000E83EA700F535820044BB2E009CE9840032
:10DF4000B4267000417E5F00D691390053833900BA
:10DF50009CF439008B5F840028F9BD00F81F3B005A
:10DF6000DEFF97000F980500112FEF000A5A8B0073
:10DF70006D1F6D00CF7E360009CB2700464FB700DE
:10DF80009E663F002DEA5F00BA277500E5EBC700EB
:10DF90003D7BF100F739070092528A00FB6BEA00E3
:10DFA0001FB15F00085D8D00300356007BFC46000A
:10DFB000F0AB6B0020BCCF0036F49A00E3A91D0043
:10DFC0005E619100081BE60085996500A0145F0062
:10DFD0008D40680080D8FF0027734D000606310091
:10DFE000CA561500C9A873007BE260006B8CC000A4
:10DFF00000000040FB21F93F000000002D44743E6A
:10E00000000000809846F83C0000006051CC783B4E
:10E0100000000080831BF0390000004020257A3882
:10E02000000000802282E336000000001DF3693505
:10E0300002000000030000000400000006000000D1
:10E0400038950000E2940000E29400001096000071
:10E05000DE940000DE94000006960000109600009A
:10E06000DE94000006960000DE940000109600008A
:10E070001496000014960000149600001C960000F0
:10E0800014A00000869E0000CA9E00002E9E000084
:10E09000CA9E0000BA9F0000CA9E00002E9E00008B
:10E0A000869E0000869E0000BA9F00002E9E000003
:10E0B000269E0000269E0000269E0000C89F0000AD
:10E0C0003CA700003EA600003EA600005CA90000A0
:10E0D00038A6000038A6000044A900005CA9000092
:10E0E00038A6000044A9000038A600005CA9000082
:10E0F00052A9000052A9000052A9000060A9000026
:10E100002C2066756E6374696F6E3A2000617373BC
:10E11000657274696F6E2022257322206661696CB6
:10E1200065643A2066696C6520222573222C206C78
:10E13000696E65202564257325730A00840000201C
:10E14000232D302B2000686C4C00656667454647E0
:10E150000030313233343536373839414243444563
:10E1600046003031323334353637383961626364D2
:10E1700065660000000000000000000000000000D4
:10E18000000000000000000000000000000000008F
:10E19000000000000000000000000000000000007F
:10E1A000000000000000000000000000000000006F
:10E1B000000000000000000000000000000000005F
:10E1C000000000000000000000000000000000004F
:10E1D000000000004300504F534958000020202009
:10E1E0002020202020202828282828202020202007
:10E1F00020202020202020202020202020881010D7
:10E200001010101010101010101010101004040432
:10E2100004040404040404101010101010104141F0
:10E2200041414141010101010101010101010101DE
:10E2300001010101010101011010101010104242F2
:10E2400042424242020202020202020202020202AE
:10E25000020202020202020210101010200000004E
:10E2600000000000000000000000000000000000AE
:10E27000000000000000000000000000000000009E
:10E28000000000000000000000000000000000008E
:10E29000000000000000000000000000000000007E
:10E2A000000000000000000000000000000000006E
:10E2B000000000000000000000000000000000005E
:10E2C000000000000000000000000000000000004E
:10E2D000000000000000000000000000000000003E
:04E2E000000000003A
:08E2E400241EFF7F0100000071
:10E2EC00FFFFFFFF4006000001000000E803DC0513
:10E2FC00DC05DC05DC050000FFFFFFFFFFFFFFFF77
:10E30C001800000019FCFFFFFFFFFFFFFF000000DB
:10E31C000200000003000000FFFFFFFF00000000F0
:10E32C00010000000000020001000000FFFFFFFFE1
:10E33C0000000000020000000000040002000000C9
:10E34C00FFFFFFFF000000000300000000000800BA
:10E35C00030000000A00000008000000010000009B
:10E36C00840000200000000094E10000B4E10000F3
:10E37C0074E100000000000000000000000000003C
:10E38C000000000000000000000000000000000081
:10E39C000000000000000000000000000000000071
:10E3AC000000000000000000000000000000000061
:10E3BC000000000000000000000000000000000051
:10E3CC0000000000430000000000000000000000FE
:10E3DC000000000000000000000000000000000031
:10E3EC0000000000430000000000000000000000DE
:10E3FC000000000000000000000000000000000011
:10E40C0000000000430000000000000000000000BD
:10E41C0000000000000000000000000000000000F0
:10E42C00000000004300000000000000000000009D
:10E43C0000000000000000000000000000000000D0
:10E44C00000000004300000000000000000000007D
:10E45C0000000000000000000000000000000000B0
:10E46C00000000004300000000000000000000005D
:10E47C000000000000000000000000000000000090
:10E48C00000000004300000000000000000000003D
:10E49C000000000000000000000000000000000070
:10E4AC000000000069C8000081C2000000000000EC
:10E4BC00DCE10000B2CA000038CF000038CF000009
:10E4CC0038CF000038CF000038CF000038CF000024
:10E4DC0038CF000038CF000038CF0000FFFFFFFF1F
:10E4EC00FFFFFFFFFFFFFFFFFFFF00000100415395
:10E4FC00434949000000000000000000000000003B
:10E50C00000000000000000000000000000041536B
:10E51C00434949000000000000000000000000001A
:10E52C0000000000000000000000000000000000DF
:10E53C00E9000000ED6B0000356F00005D74000019
:04E54C00C10000000A
:0400000300006FD1B9
:00000001FF
